:020000040800F2
:1000000000800020693A0008E5460008453A0008EB
:10001000E7460008E9460008EB460008000000003B
:1000200000000000000000000000000041910008F6
:10003000ED46000800000000D1910008159200086C
:10004000EF460008F1460008F3460008F5460008B0
:10005000F7460008F9460008794600087F46000880
:10006000854600088B46000891460008FB460008BC
:10007000FD460008FF460008014700080347000846
:100080000547000807470008094700080B47000814
:100090000D4700080F470008114700089746000861
:1000A00013470008154700081747000819470008BC
:1000B0001B4700081D4700081F470008214700088C
:1000C000234700082547000827470008294700085C
:1000D0002B470008B94D0008854F00082D47000840
:1000E000BB460008654700082F4700083147000855
:1000F000334700080000000000000000000000007E
:1001000000000000000000005FF808F110B5054C89
:10011000237833B9044B13B10448AFF300800123B3
:10012000237010BD700200200000000050BD0108C7
:1001300008B5034B1BB103490348AFF3008008BD6A
:10014000000000007402002050BD010808B50348FB
:1001500006F0BAFEBDE8084004F044BF2969010872
:1001600004F040BF70B515460022C0E901150270C9
:10017000C0E90332C0E90522C0E907224262DDE995
:100180000412044600F11C0610F008F838B929469C
:10019000074806F099FE2B21064803F0D1FBDDE964
:1001A0000423314620460FF0E6FF204670BD00BF15
:1001B000476901087269010810B50446C06910B1A9
:1001C000012111F0AFFA206910B1012111F0AAFA52
:1001D000204610BD2DE9F04100259DF81860C0E9CA
:1001E00001120570C0E90335C0E90555C0E907559E
:1001F000456231460446174600F11C080FF020FE08
:1002000038B93946074806F05FFE2021064803F05A
:1002100097FB3246414620460FF000FE2046BDE8DF
:10022000F08100BF4769010872690108F8B500252F
:10023000C0E901120570C0E90335C0E90555C0E900
:100240000755456206990446164600F11C070FF053
:10025000E7FE38B93146074806F036FE2021064849
:1002600003F06EFB069A394620460FF0C2FE204688
:10027000F8BD00BF4769010872690108F8B500259B
:10028000C0E901120570C0E90335C0E90555C0E9B0
:100290000755456206990446164600F11C070FF003
:1002A00065FF38B93146074806F00EFE20210648A2
:1002B00003F046FB069A394620460FF027FF2046FA
:1002C000F8BD00BF47690108726901082DE9F041D6
:1002D0008F4B9EB0D3E9001214331B6881EA0204ED
:1002E0005C400EAF00948B4806F0EEFD2146384688
:1002F0000BF038FF00F0A8FE02463B4652F8300FE4
:10030000012651684FF0080803C310F099FB054619
:1003100004AC814B814A314600962046FFF75AFFD4
:100320002146284610F038FC2046FFF745FF7C4B5D
:10033000CDE900781A4604212046FFF713FF214635
:10034000284610F029FC2046FFF736FFCDF8048040
:100350004FF0100814AB0093724B04211A4620464C
:10036000FFF700FF2146284610F016FC2046FFF755
:1003700023FF10AB00936C4BCDF804801A46042188
:100380002046FFF7EFFE2146284610F005FC674F98
:100390002046FFF711FF16AB654A0093CDF80480A5
:1003A0003B4604212046FFF7DDFE2146284610F09B
:1003B000F3FB2046FFF700FF1AAB5E4A0093CDF82F
:1003C00004803B4604212046FFF7CCFE2146284608
:1003D00010F0E2FB2046FFF7EFFE04210FAB564A78
:1003E0000191009320463B46FFF7BCFE214628467C
:1003F00010F0D2FB2046FFF7DFFE0B234F4A00939D
:1004000002214F4B2046FFF711FF2146284610F0EE
:10041000C3FB2046FFF7D0FE0E230027494A009376
:100420000221494B2046FFF701FF2146284610F0E4
:10043000B3FB2046FFF7C0FE444B454A31460096C9
:100440002046FFF7C7FE2146284610F0A5FB2046B0
:10045000FFF7B2FE3F4B404A314600972046FFF778
:10046000B9FE2146284610F097FB2046FFF7A4FE70
:100470003A4B3B4A009303213A4B2046FFF7FEFEDE
:100480002146284610F088FB2046FFF795FE364BA4
:10049000364A314600972046FFF79CFE2146284603
:1004A00010F07AFB2046FFF787FE314B314A314688
:1004B00000962046FFF78EFE2146284610F06CFB82
:1004C0002046FFF779FE2C4B2C4A009303212C4B3E
:1004D0002046FFF7D3FE2146284610F05DFB20465C
:1004E000FFF76AFE2846274B274A284910F01CFAD6
:1004F000274B0493274B0593274B0693274B0093D9
:1005000094E80700052310F0F5FC1EB0BDE8F0816B
:100510005000F81FD8660108FB6601080E67010845
:10052000136701081A670108216701080A670108B3
:100530002867010830670108386701086767010804
:100540003F670108936701086A6701089B67010814
:10055000D8A00108B6670108DF6701082D68010807
:1005600021680108E86701083C680108666801081D
:100570007768010899680108BE6F0108F1680108F1
:10058000A668010861010008FF68010823690108E5
:10059000E93F0008713F00084D010008000008080D
:1005A00008B500F043FC00F05BFC00F011FC014BCF
:1005B000187808BDB804002008B500F045FDBDE876
:1005C000084000F077BD07B58DF8041001A98DF83B
:1005D00005208DF8063001F031FE03B05DF804FB14
:1005E0002DE9F04F85B0FFF771FEFA200AF0C2F84E
:1005F00010F040FA0FF02CFE5C4806F065FC10F09D
:1006000039FA5B4E054633685A4C13F0010F04D19A
:1006100001F02EFD012320603360266800F014FDF8
:1006200000F12801304601F0E7FB5349206801F052
:10063000E5FB52492846266810F0BFF850490246AB
:1006400001A801F0C3FB01A9304601F019FC6127A4
:100650004C4B01A902934C4B8346206801970393AE
:1006600001F020FD494A4A4B02924A4A187001A9FA
:1006700020680197039201F015FD474A474E029208
:10068000474A307001A920680197039201F00AFDE2
:1006900070220192434A444F0292002201A938700D
:1006A00020688DF80C2001F0FDFCDFF8148188F83B
:1006B0000000206802F058FD3C498246206802F0A4
:1006C00059FC3B498146284610F054F8304B394DCF
:1006D0001978F0B120682A7880F828103378FFF76D
:1006E00072FF31782A780B462068FFF76CFF20688C
:1006F00001F0C4FF304806F0E7FB01224FF4FA7125
:10070000206801F029FF002009F0AEFD05B0BDE82A
:10071000F08F2068534680F828102A78FFF753FF9F
:1007200033782A7851462068FFF74DFF3B782A78C6
:1007300031782068FFF747FF204A4B461278397816
:100740002068FFF740FF3B782A7849462068FFF78A
:100750003AFF98F800302A7839782068FFF733FF9D
:1007600033785A4698F80010BEE700BF656A010862
:100770008C020020D4020020B9050008216801087D
:10078000826A01081A7C0108A10500088E6A010826
:10079000D8020020CD080008936A0108D902002081
:1007A000050A0008837B0108DB0200209A6A010821
:1007B000DF670108B8040020A36A0108B70400201D
:1007C000DA0200202DE9F04F85B01F46904606461C
:1007D0000D4610F04FF904463A464146684610F07F
:1007E00025FF374B6846197810F04AFF35492046F7
:1007F0000FF0C0FF814600F027FC347800F1110AA9
:100800000CBB05F101082B78A3421CDD4046514684
:1008100000F0A8F94FEAC40B08F1080868B3B9F171
:10082000000F06D00BF1020106222944684610F0A1
:1008300009FF05EB4404B4F90211684610F02FFFDC
:10084000337801333370B9F1000F0CBF0223082352
:100850003478FF1A2B78A34209D9684610F01DFF9F
:10086000B8420CD329781848091B06F02DFB6846BE
:1008700010F013FF05B0BDE8F08F0134C3E74FEA75
:10088000C40808F101005146284400F06BF998B9FA
:10089000B9F1000F06D008F102010622294468468A
:1008A00010F0D0FE05EB4403B3F90211684610F0D6
:1008B000F6FE3378013333700134E4B2CAE700BF87
:1008C0002204002099680108446A010870B52D4B84
:1008D000C0B21B788EB0984203D100F0A7FA00F0A6
:1008E000BFFA04F055F8284BC3E9000100F070FA94
:1008F00000F0AAFB044610F0BDF824490FF03AFFBF
:1009000020B904F11101224811F01EFA00F0F4F9A7
:1009100000F044FAE36904F11C051B682846002135
:100920009847012203211B4803F022FDE369284672
:100930005B680021984702221648114603F018FD13
:1009400000230124124D144E8DF803302B789DF8AE
:100950000320934211D921460132304606F0B4FA01
:10096000322301AA29460DF10300FFF72BFF0146B0
:1009700001A806F00FFB0134E8E7084B18780EB029
:1009800070BD00BFDA020020100000206668010878
:10099000E002002000000240AB690108B80400201A
:1009A0001FB50A221449684610F040FE002168462F
:1009B00010F066FE0321684610F062FE04216846CE
:1009C00010F05EFE0D4B6846B3F9001010F067FEA4
:1009D0000B4B6846198810F06EFE684610F05BFEFF
:1009E0000446684610F059FE2146C2B2012002F0CA
:1009F000E5FC04B010BD00BFC7020020DC020020EF
:100A0000DE0200202DE9F843254BC0B21B78254DAE
:100A1000984204D1244806F057FA00232B7023494A
:100A20002C78D1E90023B3F1004F08BF002A894692
:100A3000DFF89C8009D0D8E900108E1A60EB03071C
:100A400000231B4AB242BB410DDA2146194806F089
:100A50003BFAD8E90023C9E90023FFF7A1FF164BB1
:100A60001878BDE8F883154E3378A34212D9314681
:100A70003223134A0B48FFF7A5FE07462A78611C6C
:100A80003378104806F020FAFAB20D49022002F03D
:100A900095FCE4E721460C4806F016FA0B4BDFE71D
:100AA000D9020020C6020020DB69010808000020EE
:100AB00008510100F6690108B7040020E002002097
:100AC00094020020086A0108276A0108B80400207F
:100AD0001000002037B500F0B7FA0125044603687E
:100AE0009B689847114B4FF496720193104900236D
:100AF0000095104809F0CAFA23682946DB682046A9
:100B000098474FF4FA7003F011FA23680021DB686C
:100B100020469847084806F0D7F9084806F0D4F967
:100B2000C82003F003FA09F08BFCFEE790020020D6
:100B3000BD6A0108E1050008C66A0108D96A010812
:100B4000FF23044A1370044A1370044A1370044AC2
:100B500013707047D8020020DB020020D902002069
:100B6000DA02002008B5082213F042F8B0FA80F04B
:100B7000400908BD2DE9F04FA3B00FF07BFF002521
:100B800006464FF48070CDE9055507958DF8205045
:100B900006F026FA5249044630460FF00EFE014692
:100BA000204613F03DFF662665274FF064084FF09E
:100BB00063094FF0620A4FF0610B204613F038FFD3
:100BC000A84219DD635D413B052B06D8DFE803F041
:100BD00003070A0D101204F805B00135EDE704F81B
:100BE00005A0FAE704F80590F7E704F80580F4E7B4
:100BF0006755F2E76655F0E725785DB9394806F0A4
:100C000063F92946384811F0EDF8204606F0D2F98C
:100C1000012026E004AA3549204613F0A0FF09AFC1
:100C200000233E46DFF8C4800990019356F8045B28
:100C3000D5B1019B04AA013341460020019313F072
:100C40008EFF3060054613F0F3FE0C28EED02B78B3
:100C5000002BEBD0264806F037F9204606F0AAF91B
:100C6000002023B0BDE8F08F2E46019BAB4234D06C
:100C70004FF00008DFF870901B4B1B78434526DDD2
:100C80004FF0000B09F102030DF1140A13F8012BC8
:100C900050460BF1010B1749CDE9023313F096FED4
:100CA000BBF1060F0AF1020A029BEFD10C2205A943
:100CB000386813F0C5FE09F1080958B9F2B206F117
:100CC00001095FFA88F1084811F070F84E460135C5
:100CD0000437CAE708F10108CEE7314692E700BFC2
:100CE000F1680108766B0108E0020020A06B0108A2
:100CF000A26B0108D79B010838B5064C25683DB9A1
:100D0000042010F001FD40F6E443057043802060AC
:100D1000206838BD240400200378F7B504466BBB77
:100D200002F0F2FF194912F08BFA12F075FC85B24D
:100D3000284612F031FA154912F036FB11F010FE78
:100D4000064660880F4612F027FA104912F02CFB75
:100D500011F006FE3B46CDE9000132460C4806F094
:100D6000B3F86388AB420BD90A4806F0ADF800F03F
:100D70006BF9012100F08AF90123237003B0F0BD63
:100D8000054803B0BDE8F04006F09EB800007A4484
:100D9000C56B0108FB6B0108146C0108037810B5E2
:100DA00004464BB1054806F08FF800F04DF90021DC
:100DB00000F06CF90023237010BD00BF2C6C0108FB
:100DC00008B5FFF799FFBDE80840FFF7E7BF00004F
:100DD000002310B5124C2370FFF78EFFFFF79CFF26
:100DE00000F032F9C36901215B681C3098470D4857
:100DF00010F0EAFE0B4810F039FF0A4810F0B4FE7C
:100E000048B1FFF7B7FE074811F01AF80123237025
:100E1000FFF7D6FF10BD044806F056F8F8E700BF0C
:100E200022040020E00200204D6B010810B5FFF7FE
:100E3000C7FF02F069FF074912F002FA12F0ECFB5B
:100E400084B22146044806F03FF8044B20461C803B
:100E500010BD00BF00007A44326B0108DE020020A2
:100E600010B500F0F1F8C36900215B681C309847A9
:100E7000FFF742FFFFF750FF10F03CFE0446FFF77C
:100E80009FFF2146034806F01FF8034B20461C80B5
:100E900010BD00BF0A6B0108DC0200207047000093
:100EA00038B50A4C05460121204603F0E5FA002337
:100EB00020461A46012103F01DFA85F00102204662
:100EC000BDE83840012103F0E3BA00BF0000024052
:100ED00008B50120FFF7E4FFBDE80840032004F057
:100EE00091B80846FFF7DCBF10B504463C2110F06E
:100EF00019FC204610BD084603F018B8024B01212A
:100F0000186803681B68184750040020021C18BFAB
:100F100001220321014803F0BBBA00BF00040240D4
:100F20000321014803F0BDBA0004024010B5094C8A
:100F3000094805F0C9FF20460B2103F09DFA002364
:100F400020461A460B2103F0D5F9BDE8104002F007
:100F5000D3BF00BF00000240BF6F010808B50220E8
:100F600002F02EFF02F090FF00F088FB02F0B6FFC7
:100F700000F068FD03F016FD0A4802F0A7FC4FF4EC
:100F8000E13003F0F3FF084B1A680AB9074A1A6008
:100F9000074B1A680AB9054A1A600648BDE80840B6
:100FA00005F092BFD10E000888070020214E0008EE
:100FB0008C070020AE6C010810B5044611F0F0F962
:100FC00022460D4B0D4842F8113B0023C4F8113066
:100FD00053600B4A84F82430E2610A4AC4E90C33B6
:100FE0002262094A84F83830A262084AE26205F0B7
:100FF0006BFF204610BD00BF10700108F36F0108A1
:10100000F8700108487101087871010864710108DD
:1010100010B5094CFFF7A2FF2368DB0709D4074886
:10102000FFF7CAFF0123064A06490448236011F06E
:10103000DEF9024810BD00BF2C040020540400203B
:10104000000000209D0E000838B5064D064C2B68A8
:1010500013F0010F04D1FFF7DBFF012320602B60A9
:10106000206838BD300400209004002008B50B2112
:10107000054803F01BFA28B1BDE808400B210248DF
:1010800003F028BA08BD00BF0000024008B519B13E
:10109000BDE80840FFF74ABF044805F015FFBDE86A
:1010A000084002220B21024803F062B9DB6F0108FD
:1010B0000000024070B504462C4804F11C0505F000
:1010C00003FF2846002100F0E5FC0021284600F03F
:1010D000F7FC204611F06EF90BF088F9204600214C
:1010E000FFF7D4FF0AF02EFB01220C21204803F069
:1010F0003FF903F06FFD23682046DB6804F12C05FF
:10110000002198471B4E0021284600F05FFD03F0A8
:101110003DFA194805F0D8FE03F020FE02F0DEFE8D
:10112000304601220D2103F023F9012230460E2121
:1011300003F01EF90021084603F00AFD04F1200027
:1011400000F0D4FC0121284600F040FD4FF4E130CE
:1011500003F00CFF094805F0B7FE0AF019FA03F096
:1011600037FD2046BDE8704011F031B98D6F0108A0
:101170000004024000000240B16F01088A9A010891
:1011800038B50546FFF772FF044628B1002128460E
:10119000FFF77CFF02F0B0FE02F0B6FD05460CB191
:1011A000FFF7C4FE284638BD70B50C460646154903
:1011B000204612F001FA20B90021204612F0DEF993
:1011C00070B11149204612F03BF812F0FFF90146C8
:1011D0000E4805F079FE40F263110D4802F0B0FBB5
:1011E0003046FFF743FF054648B93046FFF7C8FFD2
:1011F0000146204612F0E0F908B1FFF797FE2846B5
:1012000070BD00BF3333534000007A44C46C010802
:10121000F36C010870B52F4AD6B013680546DB079A
:1012200005D42D4900F12C030B60012313602B49D9
:101230002846FFF7B9FF0646294805F045FE00217C
:1012400005F11C0000F03CFC264C274BE360274BCB
:101250002361274BA360274B6360274B2360274BF9
:101260006361274BA361274BE36104F110030FCBAC
:101270008DE80F0094E80F0010F01EFD002305A874
:10128000C5F81130C5F8153010F09EFC9DF81430EB
:1012900005F11104012B16D1DDF8153005A8C5F8AC
:1012A0001130DDF81930C5F8153010F05DFC164826
:1012B00005F00AFE0821204605F06CFEBDF9161166
:1012C000124805F001FE31462846FFF7DFFE56B012
:1012D00070BD00BF280400205004002000004040E2
:1012E000476C0108984E00202D3F0008B53E0008CD
:1012F000FD0E0008210F00080D0F0008C96E000840
:1013000065910008A5910008686C01088E6C0108C1
:101310007FB5F82300F12005064628468DF80F30EA
:1013200000F0EAFB02230DF10F0100930122A0233C
:10133000284600F0E5FB4FF400430822009306F135
:101340003001A0230446284600F004FC0440E4B227
:10135000284600F0D3FB204604B070BD30B50446EB
:101360008BB05A4805F0B0FD204600F021FB00F09C
:101370005FFA00F00BFA564805F0A6FD04F12005CF
:101380005448554905F0A0FD284600F0AFFB38B998
:10139000524805F099FD40F22111514802F0D0FA6F
:1013A00002F0AAFD2046FFF7B3FF20B94FF4937176
:1013B0004B4802F0C5FA94F837304A48049394F841
:1013C0003630039394F83530029394F83430019317
:1013D00094F83330009394F8323094F8312094F834
:1013E000301005F071FD284600F0D2F9284600F0D3
:1013F00031FA04F11C0584F838000021284600F079
:1014000049FB012000F032FC0021284600F058FB87
:10141000012000F049FC2046FFF7FCFE00F066FAD0
:10142000314805F051FD4FF4FA7012F0D1FB04463B
:10143000002844D12D4805F047FD2D4805F044FD16
:101440002C4805F041FD2C4805F03EFD2B4805F0E9
:101450003BFD2B4805F038FD2A4805F035FD2A48AC
:1014600005F032FD294805F02FFD294A29492A486F
:1014700005F02AFD29492A4805F026FD294805F0EE
:1014800023FD294B294A1B6829490093294B1268DF
:101490001B68294813F09AFA2749284805F014FDDB
:1014A00007A803F017FA07A805F064FC01462448D2
:1014B00005F00AFD0F4805F007FD0BB030BD2148CF
:1014C00005F002FD204612F08BFBB6E7336D0108F4
:1014D000456D01085A6D0108A0860100756D01086F
:1014E000F36C01088B6D0108C06D0108EE6D0108F9
:1014F000BC6F01082C6E01085D6E01086C6E01085E
:101500008E6E0108B16E0108D56E0108BD6F01082D
:10151000F86E0108FE6E01081C6F01082C6F0108AF
:10152000336F01083E6F01086400F81F5000F81F78
:101530005E6F01085400F81F34040020706F01082A
:101540007B6F0108226E0108024B186803685B6814
:10155000184700BFA0040020024B186803689B686E
:10156000184700BFA00400200023F0B513701446F4
:10157000022205460C4E85B030688DF80F100368C6
:101580000092DF6801222B460DF10F01B84748B1E8
:101590004FF4004230682146036800921E69012220
:1015A0002B46B04705B0F0BDA004002030B585B093
:1015B0008DF80D200022074B8DF80C101C6803A934
:1015C00023680092DD68022203462046A84705B042
:1015D00030BD00BFA004002037B54FF40045064BD6
:1015E0001C68236800951D6913460A46014620467B
:1015F000A84703B030BD00BF9C04002037B50025CC
:10160000054B1C6823680095DD6813460A460146B1
:101610002046A84703B030BD9C04002037B5022502
:10162000054B1C6823680095DD6813460A46014691
:101630002046A84703B030BD9C040020024B186828
:1016400003681B68184700BF9C040020024B186801
:1016500003685B68184700BF9C040020024B1868B1
:1016600003689B68184700BF9C0400204FF47A73FE
:101670005843B0FBF3F009F07DB8000010B5424CC0
:101680000AF0B2F820460222002102F071FE012287
:101690002046114602F06CFE20460122022102F093
:1016A00067FE20460222032102F062FE204600224D
:1016B000042102F05DFE20460222082102F058FEBD
:1016C00020460122092102F053FE204601220A2170
:1016D00002F04EFE204602220B2102F049FE02F0EB
:1016E000FDFB002320461A460C2102F003FE204693
:1016F00000220C2102F0CCFE2046002204F580647A
:101700000F2102F035FE20460122002102F030FEBA
:1017100020460022022102F02BFE20460022032157
:1017200002F026FE20460222062102F021FE20467B
:101730000022082102F01CFE20460022092102F0AE
:1017400017FE204601220C2102F012FE2046022242
:101750000D2102F00DFE204602220E2102F008FEAD
:10176000204602220F2102F003FE002304F58064CC
:1017700020461A460D2102F0BDFD2046BDE810406E
:1017800000220D2102F084BE0000024003F00AB9DD
:101790001C4B00B51A6889B0D2075FBF1A4A1060A7
:1017A00001221A60194B0493194B0593194B0393AB
:1017B000194B0293194B0793194B069308AB13E986
:1017C00003008DE8030002AB0FCB10F023F990B1BA
:1017D000144805F079FB00221348114602F0C8FDB9
:1017E0000F2302220021104802F062FC09B05DF8CC
:1017F00004EB10F0A9B869210C4809B05DF804EBBE
:1018000002F09EB898040020A004002049150008AA
:101810005915000869150008AD150008C96E0008C3
:101820006D1600089D70010800000240AE700108AE
:10183000002307B5ADF8043001238DF80630019878
:1018400009F02EFF02F04AFB03B05DF804EB09F04B
:1018500079BF0000194B10B51A688CB0D2075FBF72
:10186000174A106001221A60164B0793164B059316
:10187000164B0693164B0893164B0993164B0A9377
:10188000164B0B930CAB13E907008DE8070005AB73
:101890000FCB0FF0E3FF044601220F21104802F0A6
:1018A00067FD3CB10F4805F00FFB0FF0B5FF204678
:1018B0000CB010BD0C4805F007FBF8E794040020BD
:1018C0009C040020D9150008FD1500081D1600080D
:1018D0003D1600084D1600085D160008C96E000888
:1018E0000000024024700108577001082DE9F047FC
:1018F0009AB00AF043FBDFF8B490244C244E254FF5
:1019000012AD50B9CDE91544CDE91376CDF8489024
:10191000009495E80F000AF037FB1F4B4FF0000AC8
:1019200013931E4B4FF0010812931D4B06A91493FD
:101930001C4B284615931C4BCDE91876CDE916347F
:101940000423CDE9063A8DF81D8006F009F805F06C
:10195000FBFF12F09FFF514610220EA812F07EF9F5
:101960000323CDE908440D938DF83D8001AC0DAD06
:101970000FCDCDE90A970FC42B682360009608AB02
:101980000FCB0AF035FC1AB0BDE8F087C96E00082D
:10199000B56F0008E16F0008C9B6000891B50008EE
:1019A000A1B4000839B400084DB4000891490008FA
:1019B0002DE9F047044602F0A7F91E49054611F04B
:1019C0003FFC11F003FE01461B4805F07DFA4FF085
:1019D0008041284611F0D2FD48B30025DFF8609021
:1019E000DFF85080154E02F08FF94946074611F096
:1019F000D9FDA8B94146384611F022FC11F0E6FDA8
:101A00000146304605F060FA236885F0010520465E
:101A1000DB68294698474FF47A7002F087FAE2E7CC
:101A200023682046BDE8F047DB6800211847BDE881
:101A3000F08700BF00007A447570010882700108C9
:101A40000000204008B50D49012002F003FE0C49BA
:101A50000B2002F0FFFD0B490A2002F0FBFD0A49B2
:101A6000042002F0F7FD0949072002F0F3FDBDE86C
:101A700008400749052002F0EDBD00BF8D8C00082D
:101A80009D8F0008298E0008B59000080990000875
:101A900091900008002310B50C461A460D21074806
:101AA00002F028FC14B1012C00D010BD2246BDE884
:101AB00010400D21014802F0EBBC00BF00080240BD
:101AC000002310B50C461A460C21074802F012FC00
:101AD00014B1012C00D010BD2246BDE810400C21ED
:101AE000014802F0D5BC00BF00000240014802F0EE
:101AF0003BBD00BFA086010002F006BD02F020BD84
:101B00002DE9F041069F1E4607F00303032B804694
:101B10000C46154603D119210D4801F011FF20464E
:101B2000BC07324629460AD502F058FD10B1012003
:101B3000BDE8F0810123002088F80430F8E7FB07B6
:101B400002D502F059FDF1E702F03AFDEEE700BFE1
:101B5000007101082DE9F041069C0D46E107804621
:101B600016461F4603D536210D4801F0E9FEA207AF
:101B700003D539210A4801F0E3FE23043A463146F1
:101B800028460AD502F046FD10B10120BDE8F081DB
:101B90000123002088F80430F8E702F003FDF3E7A2
:101BA0000071010808B50321034802F07AFC0030F7
:101BB00018BF012008BD00BF000402400A460248C9
:101BC000032102F065BC00BF0004024008B581B1EA
:101BD000012303211A460A4802F08CFB032108481E
:101BE00002F04AFCBDE8084003220548114602F015
:101BF00061BB0122BDE808400321014802F0B8BBE7
:101C00000004024002F0C4BE084611461A469DF880
:101C1000003002F05DBF02F009BF02F021BF0846AC
:101C200002F09ABDDFB50023CDE90133ADF80C30E9
:101C300001238DF807308DF808306FF01D038DF803
:101C400009300723044601A88DF80A3005F079F819
:101C5000236806461B6820460F469847864277EB66
:101C60000103B4BF0120002004B0D0BD042817D860
:101C7000DFE800F00309100E1200002303211A46CA
:101C8000084802F037BB00220321064802F070BB6F
:101C90000222F9E70122F7E70321024802F08EBB96
:101CA000704700BF00000240042817D8DFE800F0AA
:101CB0000309100E1200002302211A46084802F000
:101CC00019BB00220221064802F052BB0222F9E7AA
:101CD0000122F7E70221024802F070BB704700BF03
:101CE000000002401FB553680293137801934B68BC
:101CF00000930B6842680178024805F0E5F805B0EA
:101D00005DF804FB9071010810B50446C06908B184
:101D100005F050F9206908B105F04CF9606808B188
:101D200005F048F9204610BD10B50446006808F0DB
:101D3000CDF8204610BD0000CA21014801F000BEC8
:101D4000AE710108FE2307B58DF80430054B01A9DB
:101D50001868002300681A4607F0A4FD03B05DF878
:101D600004FB00BFB0040020D0B51F467423C0E9B7
:101D70000031002304468360082016460FF0C4FC9F
:101D8000C0E90067A0602046D0BD0000036837B5F9
:101D9000632B05460C4601D0FFF7CEFF002301AAB6
:101DA000A9682046019304F075FE019A3AB12146D4
:101DB000044805F089F83821034801F0C1FD03B05B
:101DC00030BD00BFF07101081D72010870B56323BA
:101DD0000025C0E90031044685601A2016460FF040
:101DE00093FC1A22294611F039FF3146A0602046A3
:101DF000FFF7CCFF204670BD81647047C164704717
:101E00002DE9F843D0E90173884600254FF00C090D
:101E1000DB1B0A4E9B105E43ECB2B4420BD209FBB3
:101E200004724146506812F0F1FD01350028F3D1EB
:101E30002046BDE8F8834FF0FF30FAE7ABAAAAAA24
:101E40002DE9F843D0E90473884600254FF00C09CA
:101E5000DB1B0A4E9B105E43ECB2B4420BD209FB73
:101E600004724146506812F0D1FD01350028F3D1CB
:101E70002046BDE8F8834FF0FF30FAE7ABAAAAAAE4
:101E80002DE9F0470E4649680446FFF7B9FFC0B296
:101E9000FF2807D071682E4805F016F87C212D48E0
:101EA00001F04EFDD4E901232B4F9B1A9B107B437D
:101EB0007E2B03D97F21274801F042FDD4E901128E
:101EC0000C25E068531A9B10121A7B4392107A4338
:101ED0000133934205FB03F80ED84144A160D4E9D5
:101EE000013496E80700E31A04E907001A489B103A
:101EF00058430138BDE8F087404605F071F80546C3
:101F000018B96921154801F01BFDD4E901C3002768
:101F10004FF00C0AA3EB0C030F4A9B1002FB03F9D2
:101F2000A9EB0703002B0ADD0AFB07F305EB030E01
:101F3000634493E8070001378EE80700F0E7604646
:101F400005F038F865604544C4E90255C7E700BFAD
:101F5000567701081D720108ABAAAAAA7677010874
:101F60001FB56E23CDE90131002301A90393FFF7CB
:101F700087FF05B05DF804FB0023FF2270B54FF02A
:101F80000041C0E90033C0E90233C0E90433C0E9CD
:101F90000633C0E9083380F82820044600206FF09B
:101FA0007F42C4E90C01C4E90E014FF0FF31C4E9DE
:101FB0001233C4E91012002305221E4DC4E9142374
:101FC0002A6812F0010212D101211B4E084632602C
:101FD00007F08EFB306018B91121184801F0B0FCF1
:101FE0000123174A174914482B6010F000FA164BCA
:101FF0001A680AB9104A1A6014492046FFF7B0FF60
:10200000134B144918702046FFF7AAFF124B1349CF
:1020100018702046FFF7A4FF114B12491870204694
:10202000FFF79EFFFE22104B1870104B20461A70CF
:1020300070BD00BFAC04002020050020A37801087B
:1020400000000020291D0008B0040020DD780108F0
:10205000B8040020E5780108B6040020ED780108F6
:10206000B4040020F2780108B7040020B504002071
:1020700010B5084C2368DB0709D40748FFF77CFF3D
:102080000123064A06490448236010F0B0F90248CB
:1020900010BD00BFA8040020C804002000000020DC
:1020A000091D00082DE9F0470E4649680446FFF770
:1020B000C7FEC0B2FF2807D071682E4804F004FFA5
:1020C00087212D4801F03CFCD4E904232B4F9B1AB7
:1020D0009B107B437E2B03D98A21274801F030FCDB
:1020E000D4E904120C25A069531A9B10121A7B43E1
:1020F00092107A430133934205FB03F80ED8414412
:102100006161D4E9043496E80700E31A04E90700A2
:102110001A489B1058430138BDE8F087404604F048
:102120005FFF054618B96921154801F009FCD4E99B
:1021300004C300274FF00C0AA3EB0C030F4A9B10BB
:1021400002FB03F9A9EB0703002B0ADD0AFB07F3E7
:1021500005EB030E634493E8070001378EE80700A0
:10216000F0E7604604F026FF25614544C4E90555C3
:10217000C7E700BFAE7701081D720108ABAAAAAA83
:102180007677010838B5D0E901239B1A074A9B10DE
:102190005343CDB29D42044603D3A621044801F027
:1021A000CFFB0C20636800FB053038BDABAAAAAAA0
:1021B0001D72010838B5CCB2114905460B6813F001
:1021C000010307D10F4A70201372012310600E48DB
:1021D0000B605060FF2C10D0D5E904239B1A0B4AEA
:1021E0009B1053439C4203D3B221094801F0A8FB42
:1021F0000C23286903FB040038BD0248FCE700BF3C
:10220000A4040020BC0400209D720108ABAAAAAA65
:102210001D72010810B5D0E90730C9B2D2B28342AD
:1022200009D01C788C4204D15C78944201D1987812
:1022300010BD0333F3E74FF0FF30F9E72DE9F0412C
:10224000D0E904239B1A534A9B1053430D46097847
:102250000446994203D393214F4801F071FBD4E91E
:1022600001239B1A4B4A9B1053436978994203D32D
:102270009421494801F064FBD4E904239B1A454AA0
:102280009B105343A978994205D3FE2903D0952189
:10229000414801F055FB6A7829782046FFF7BAFFDC
:1022A000C3B2FF2B06462CD03C4804F00DFE297823
:1022B0002046FFF77FFF697807462046FFF762FF59
:1022C000314680462046FFF775FF414602463846B4
:1022D000FFF708FD29782046FFF76CFF697806466E
:1022E0002046FFF74FFFA97807462046FFF762FF19
:1022F000394602463046FFF7F5FC9C21264801F09E
:102300001FFBD4E90723234F9B1A7B437E2B03D962
:102310009F21214801F014FBD4E90721606A8B1A40
:102320007B43091A4F430133BB4203EB43080AD8EE
:10233000424422622A88236A23F8032CAA7803F8ED
:10234000012CBDE8F081404604F04AFE064618B96B
:102350006921134801F0F4FAD4E907010B1A0D4979
:1023600059430023CA1A002A0DDD03EB43028718E4
:10237000B7F800E006EB020C26F802E0BA78013369
:102380008CF80220EEE704F015FEE6614644C4E94D
:102390000866CFE7ABAAAAAA1D72010882720108DB
:1023A0007677010813B5FF24074B8DF804401B68AE
:1023B0000A46186801A907F019FB012814BF204636
:1023C0009DF8040002B010BDB004002038B581684B
:1023D00000681D46144604F04FFE0346201845EBE6
:1023E000E37138BD2DE9F0410E681046722E1F468C
:1023F00027D0742E08D0632E12D000244FF0004551
:1024000020462946BDE8F0818B68D3E90023B3F16B
:10241000004F08BF002A19D0841847EB0305EFE7E7
:10242000886804F0F7FB002871F1000304460D46AC
:10243000E6DA084804F048FDDD21074801F080FA9B
:10244000DEE78868BDE8F041FFF7C0BF14461D46CF
:10245000D6E700BFA47301081D7201082DE9F047FB
:102460000F460646FFF7A6FE0024DFF85C904268A0
:102470000178FFB2124804F027FDD6E90758454518
:1024800016D02B78BB4211D169783046FFF77AFE1F
:10249000016869290AD1D0E9012A484604F014FDEF
:1024A000DAF8003003B198470134E4B20335E6E7C7
:1024B0002146044804F008FD2046BDE8F08700BF2F
:1024C000CA73010813740108F17301082DE9F34779
:1024D00007468846FFF76EFE0025426801781B48D4
:1024E00004F0F2FCFC693E6ADFF8689003340336BE
:1024F0005FFA88F8A64220D0234633F8032D9B7854
:10250000ADF804208DF8063014F8033C984512D13C
:102510009DF805103846FFF735FE016869290AD194
:10252000D0E9012A484604F0CFFCDAF8043003B1C0
:1025300098470135EDB20334DCE72946044804F03E
:10254000C3FC284602B0BDE8F08700BF3174010823
:102550007E7401085A740108836C73B504460D46F5
:10256000164623B94FF48C710D4801F0E9F90D4975
:10257000CDE9006423462A460B4807F087FD012871
:1025800001460AD0094804F09FFC4FF48F710448BB
:1025900002B0BDE8704001F0D3B902B070BD00BF19
:1025A0001D72010824770108C92D00082F77010842
:1025B00038B590F847300446032B0D4604D940F255
:1025C0003111064801F0BCF994F847305A1C84F8E0
:1025D00047201C4484F8425038BD00BF1D720108DA
:1025E00010B590F84730044623B94FF49B71064864
:1025F00001F0A6F994F84730013BDBB284F847308C
:102600001C4494F8420010BD1D720108CBB2FE2B91
:1026100037B5054605D1104803B0BDE8304004F099
:1026200053BCFFF7C7FD016804466D290DD1017A3F
:102630002846FFF7BFFD436800930368D4E9001202
:10264000064804F041FC03B030BD4268044803B0C2
:10265000BDE8304004F038BC4F78010857780108D5
:102660008475010808B5FFF78DFDBDE80840D0E985
:102670000012014804F028BCCE7701082DE9F74F7D
:1026800004462A4804F020FC4FF00008284FDFF8E9
:10269000B0A0DFF8B090D4E90431C91A89107943A9
:1026A0005FFA88F6B14231D9504604F00DFC20465D
:1026B0003146FFF7ABFF94F82830DFF88CB0B34217
:1026C0000CBF1C48484604F0FFFBD4E907531A4AE4
:1026D000AB4218D02978B14213D11046019304F0CF
:1026E000F3FB69782046FFF7BDFF584604F0ECFB8A
:1026F000A9782046FFF78AFF484604F0E5FB019BD6
:102700000D4A0335E4E708F10108C4E7D4E90723DB
:102710009B1AD4E90102121A92107B437A430748AC
:1027200003B0BDE8F04F04F0CFBB00BFD67701087F
:10273000ABAAAAAAEE770108FA7701080B7801087C
:10274000E5770108BD6F0108077801082DE9F84316
:102750000422054690F84710114804F0B5FB002408
:10276000DFF848900F4F05F1420695F84730A34235
:1027700010DD16F8011B2846FFF71CFDD0F8048079
:1027800014B1484604F0A0FB4146384604F09CFBD7
:102790000134EAE70448BDE8F84304F095BB00BF04
:1027A0003F780108497801084C780108477801080A
:1027B00000232DE9F04FC0E90433884619464FF055
:1027C00000430446C0E90213C0E90013FF2085B0AE
:1027D000CDE90013DDE90E6720745FFA82F9D8E9CC
:1027E00007500390039BD4E900AB9D4220D02B7887
:1027F0004B451BD169784046FFF7C4FC32463B4647
:1028000001464046FFF7EEFDDDE90023994208BF8F
:1028100090420BD09B4508BF924503D0504571EBC9
:102820000B0303DA6B78C4E9000123740335D9E79D
:10283000BBF1004F08BFBAF1000F05D0BAEB060696
:102840006BEB0707C4E90267204605B0BDE8F08FCF
:10285000F8B50D460E4B896806464B434FF47A7126
:10286000B3FBF1F1FFF79EFD0446C7B2B06C0368FD
:102870001B689847C6E90E0104F0A6FA0146054810
:1028800004F022FBFF2F0CBF287C2046F8BD00BFC0
:1028900040420F005F72010870B5C36C86B00446F9
:1028A0000D464BB9224804F00FFB2946204606B0DE
:1028B000BDE87040FFF7CCBF806C1E4903681B6900
:1028C0009847A06C03689B689847D5E9002303A844
:1028D00004F012FAA06C9DF80C20036800929DF899
:1028E0000F109DF80E205E689DF80D30B047A06C6B
:1028F0000368DB689847E36C9847A06C03689B68A3
:102900009847A06C03681B689847C4E90E0104F05F
:102910005BFA0146084804F0D7FA00212046FFF789
:1029200041FDC0B2FE2808BF287C06B070BD00BFC4
:1029300065780108451D0008837801082DE9F84FE6
:102940009046D1E90023B3F1004F08BF002A0546A5
:102950000C4677D0DFF830B1DFF830A1D4E90201BE
:10296000012871F100030DDA50EA010302D03B485F
:1029700004F0AAFA3A4804F0A7FA94F810904846EE
:10298000BDE8F88FB8F1000F1AD0504604F09CFA59
:1029900021462846FFF75CFF5FFA80F9B9F1FF0F87
:1029A0001ED1304804F090FA40F20E212E4800F07B
:1029B000C7FF2E4B2E4A40F20F212B4811F006F88C
:1029C000D5E91423904271EB030301DA5846DDE7A1
:1029D000284804F079FA21462846FFF75DFFDBE737
:1029E000237C4B452AD1D5E90E01D4E9002390423E
:1029F00071EB030C12DA204804F066FAD5E90E23D5
:102A0000D4E90001801A61EB0301C4E9020104F07A
:102A1000F1F90146194804F057FA9FE7861A61EB6D
:102A20000307022E77F10003A9DB3946304604F094
:102A3000E1F90146124804F047FAA0E7114804F012
:102A400043FA9CE7B8F1000F03D0BDE8F84FFFF759
:102A5000FFBEBDE8F84FFFF71FBF00BFFB750108C1
:102A600020760108907601081D720108B6760108EB
:102A70001F79010876760108BC760108DB7601082B
:102A8000EE7601080D7701085876010838760108BE
:102A90002DE9F04188B004460E46FFF78BFB036832
:102AA0000546702B04D04FF49E71344800F048FF67
:102AB000A06C03681B6898473246C4E90C01CDE955
:102AC0000001214602A8FFF773FE31462046FFF7BA
:102AD000C5FC9DF818300746FF2B0AD148B9297864
:102AE00027486A6804F0F0F940F24711234800F0E3
:102AF00027FFD4E90C0104F067F90146214804F0EE
:102B0000E3F93946204804F0DFF99DF81810FF2951
:102B100015D11E4804F0D8F900224FF00043CDE94A
:102B200004232A7A02A92046FFF708FF054631460A
:102B30002046FFF7CBFC284608B0BDE8F0812046D0
:102B4000FFF720FBD0E90078DDE9020104F03CF951
:102B50004246034639460E4804F0B6F9D4E90C3231
:102B600002980399C01A61EB0201CDE9040104F057
:102B700041F90146074804F0A7F9D2E71D720108A0
:102B8000DC7201080F7301082E73010849730108F4
:102B9000627301088673010870B504460D46FFF79D
:102BA00009FB03686D2B11D0702B09D0612B0DD15F
:102BB000836894F8411094F84000BDE870401847CD
:102BC00029462046BDE87040FFF762BF40F22B1156
:102BD000024800F0B5FE4FF0FF3070BD1D720108D5
:102BE0002DE9F74F0446684804F06EF9674804F091
:102BF0006BF9674804F068F9644804F065F994F8E3
:102C00002830FF2B04D14FF4D071624800F098FEB9
:102C100094F828102046FFF7CDFA426801785E4804
:102C200004F052F994F82830DFF898B1DFF85891A1
:102C300084F8463094F846102046FFF7BBFA036844
:102C400080466D2B1BD14168544804F03DF994F83F
:102C500046102046FFF7ACFC98F80810204684F890
:102C60004610FFF7A7FA426801784D4804F02CF9A6
:102C70002046FFF76BFD484604F026F9DAE794F8A2
:102C800046102046FFF788FFC3B2FF2B07460ED140
:102C9000444804F019F940F2B5113E4800F050FEE6
:102CA00040F2B511404B414A3A4810F08FFE0246BF
:102CB00094F846102046FFF7ADFAC5B2FF2D0CD1AF
:102CC0003B4804F001F940F2BB11324800F038FEF5
:102CD000354B364A40F2BB11E6E794F84610FE2D1C
:102CE000204630D1FFF77CFC014606462046FFF720
:102CF00061FAD8F8042098F8001082462D4804F0B4
:102D0000E3F83A4631462046FFF784FAC5B2FF2D74
:102D10000CD1294804F0D8F84FF4E3711D4800F0B5
:102D20000FFE214B214A4FF4E371BDE7DAF804109E
:102D3000584604F0C9F82046FFF708FD484604F05D
:102D4000C3F83146CBE7FFF735FA39460646204649
:102D5000FFF718FA294680462046FFF72BFA019024
:102D6000164804F0B1F8164804F0AEF8019A41464E
:102D70003046FEF7B7FF94F8463084F8417084F887
:102D8000403084F8465055E7BD6F01089E74010835
:102D9000BD7401081D720108DC740108FA74010891
:102DA0001975010830750108B6760108FA7801082E
:102DB000537501086D7501088C750108D5750108FA
:102DC000EB750108BF75010808B5FFF751F9FFF76A
:102DD00007FF00002DE9F8431F461646FFF7D2F91A
:102DE000B7F1004F08BF002ED0E9005884681AD010
:102DF000742D01D0FEF7A0FFD4E9000103F0FAFF23
:102E000039468146304603F0F5FF4A4603464146BF
:102E10000A4804F059F8742D01D0FEF78DFFC4E97B
:102E20000067BDE8F883742D01D0FEF785FFD4E973
:102E3000000103F0DFFF024B0246E8E7AB72010836
:102E4000D0720108FF23054A1370054A1370054A22
:102E50001370054A1370054A13707047B8040020B8
:102E6000B6040020B4040020B7040020B5040020FC
:102E700010B50446006807F029F8204610BD10B5CB
:102E80000446006807F022F8204610BD1FB509F07F
:102E900003FB0023ADF80C300E4B5A7812B101221F
:102EA0008DF80C201B7813B101238DF80D30002311
:102EB000094A0A490A4800931278039B0978006876
:102EC00009F06AFC20B1074B187805B05DF804FBE7
:102ED000054BF9E7480500204B0500204A05002076
:102EE00044050020B4040020B604002008B50023E7
:102EF0001A4606F0D7FC431E5842584108BD000050
:102F000007B50B78012B11D05AB22AB1022B11D080
:102F10000A4803F0D9FF06E00192094B01A91B689A
:102F20001868FFF7E3FF03B05DF804FB4FF0FF33D1
:102F30000193F2E7024B04311B68F1E71B7B0108A8
:102F40003C0500201FB56123CDE9013101A90392A1
:102F5000FFF7A8F805B05DF804FB1FB57023CDE9B5
:102F60000131002301A98DF80C30FFF79BF805B063
:102F70005DF804FB30B5044685B00D4600F010F84E
:102F80006D22064B01A91B782046CDE901258DF85D
:102F90000C30FFF787F805B030BD00BF4E050020AC
:102FA0002DE9F04F554B85B01A780446002A40F0C1
:102FB000A180012652491E70FEF7D2FF514B5249A3
:102FC00018702046FEF7CCFF504B51491870204630
:102FD000FEF7C6FF4F4900230A2208704E4901A898
:102FE000FEF7C2FE01A801462046FEF749FF4B4FFF
:102FF0004B4938702046FEF7B3FF4A4D4A4A2870C5
:103000004A492046FFF79EFFDFF854B1484A8BF843
:10301000000048492046FFF795FF474905462046EE
:10302000FFF79BFF70238046019301A8434B0146A5
:10303000204602938DF80C60FFF734F8404A824630
:1030400040492046FFF77EFF3F4E40493070204602
:10305000FFF790FF81463E482B4602789BF8001010
:103060002046FDF7B0FA294A434629461278204601
:10307000FDF7A9FA274953460A7820462946FDF765
:10308000A2FA2B463A7841462046FDF79CFA2B4699
:103090003A7851462046FDF796FA2E4A2B462946A5
:1030A0002D4F12782046DFF8BC80FDF78CFA2946B8
:1030B0001C4D3B7898F800202046FDF784FA4B46DB
:1030C0002A7831782046FDF77EFA337898F8002088
:1030D00049462046FDF777FA204A3B781278317846
:1030E0002046FDF770FA1A483B780278317820467E
:1030F000FDF769FA05B0BDE8F08F00BF4206002079
:10310000747B01084C0500207E7B01084F050020E0
:10311000897B010830050020957B010831050020DE
:10312000A27B0108500500208D2E0008AE7B01080F
:10313000BD350008B87B0108CC7B0108DF7B0108A6
:1031400031360008F37B010840050020047C0108AB
:10315000B4040020B7040020B5040020510500206D
:103160004E050020B80400202DE9F8432B4B0446FF
:103170001A682B4E12F0010F4AD1FF223270012241
:103180001A602046FFF70CFF264A27492046FFF722
:10319000D9FE264A307026492046FFF7D3FE254D3A
:1031A000254928702046FFF7D8FE2449814620464D
:1031B000FFF7D3FE0746224A2B7831782046127853
:1031C000FDF701FA1F4A3378297820461278FDF777
:1031D000FAF91D4ADFF878804B46297820461278A4
:1031E000FDF7F1F92B7898F8002049462046FDF7C5
:1031F000EAF9164A3B46297820461278FDF7E3F9AA
:103200002B7898F8002039462046FDF7DCF902E0DB
:103210003378FF2BB5D03078BDE8F8832C0500203B
:1032200043060020E1360008157C010875320008CD
:103230001F7C01084D050020297C0108377C01080E
:103240004C050020B80400204F050020B6040020E3
:103250003105002070B50D460446FEF709FF04490C
:1032600022462B46BDE870400978FFF7B3BD00BF8A
:1032700031050020F7B5414C26689EB904200EF0B8
:1032800043FA3246054606600421012006F030FA72
:10329000286018B911213A4800F052FB39482560DE
:1032A00009F01AF9384F394E396839480131396017
:1032B00003F00AFE09F0F0F833781BB901233370EC
:1032C00009F020F9002301932368324A01A9186804
:1032D00006F08CFB012806D02F4803F0F5FDFB21FA
:1032E0002E4800F02DFB019D6B1C24D12C4803F0CF
:1032F000EBFD3C681E21013CE4B21E2C28BF1E24BD
:10330000002001FA04F4B4F5E15F307028BF4FF4F7
:10331000E15403F0B1FE0025261845EBE077314675
:10332000204803F0D1FD30463946FFF793FF1E4B8E
:10333000187803B0F0BD4DB129461C4803F0C4FD18
:1033400001980021FFF786FF194BF1E719483D600E
:1033500003F0BAFD09F04AF823686BB1284609F07A
:10336000BBF8256835B1286806F0B0FD0421284671
:103370000EF0D8F9002323600F4BD9E73C0500205D
:10338000A3780108012F0008600500205C050020DB
:1033900074790108A086010087790108A1790108E4
:1033A000ED790108047A0108B60400201B7A0108AF
:1033B0004F050020307A0108B8040020054B187032
:1033C000054B1A700022054B1960054B1A705A7094
:1033D000704700BF4B0500204A050020440500202F
:1033E000480500204FF47A7337B5002403FB00F240
:1033F0000749B2FBF3F20D6801A92868019406F0B1
:1034000037FC012814BF2046019803B030BD00BF2F
:10341000380500204FF47A7337B5002403FB00F21F
:103420000749B2FBF3F20D6801A92868019406F080
:10343000DDFA012814BF2046019803B030BD00BF5B
:1034400034050020034B93F82A30022B0CBF0220D6
:10345000002070479000002070B51D4600230446F0
:1034600003604171164602B115B92371204670BD43
:1034700028460EF053F92A462060314610F0C6FB6C
:103480002571F3E710B50446006808B10EF048F95D
:10349000204610BDF7B5184D04462A6822B94FF4EE
:1034A0009171164800F04CFA24B3637F13B3237F65
:1034B00003B308200EF028F9237FA26C617F064633
:1034C0006789FFF7C9FF002328681A4601A9006829
:1034D000F780019606F030F901280BD0084803F078
:1034E000F3FC019C34B12046FFF7CCFF08212046B5
:1034F0000EF018F903B0F0BD38050020A1790108DD
:10350000497B010810B50446FFF7C4FF24B12046EB
:10351000BDE810400BF0E6B810BD00007FB542F2E8
:10352000107008F0DFFF04461F4803F0CDFC002CAC
:1035300037D0A06FFFF7AEFF2578022D2DD1606840
:103540000021FFF787FEA36FF3B1D3E914231343E0
:103550001AD0164B1E6806F0BBFF01461448B04750
:10356000A36FD3E9140103F02FFCA36F01461A6D7A
:10357000104803F0A9FCA36F01A8D3E9142303F0BA
:10358000BBFB01A801F096F90B4803F09DFC204617
:1035900009F066FE284604B070BD032DD3D100208B
:1035A000CEE70125F6E700BF407A01089000002031
:1035B0005E7A01086B7A01089C7A0108002310B535
:1035C000144C84F82E3008F045FF08B108F064FF71
:1035D000FFF7A4FF032815D8DFE800F005020A086A
:1035E0000D4803F071FC0D4B187810BD0C4BFBE738
:1035F000FFF728FF022809BF01230A4B84F82E3069
:10360000094BF1E709484FF4FA7100F099F94FF0CE
:10361000FF30EAE790000020017B0108B804002099
:10362000B70400204F05002030050020A1790108D3
:1036300070B500200021FFF7D5FE28B1194803F02E
:1036400043FC194B187870BD00200021FFF7E2FE03
:10365000044620B302794179144803F035FC2279FD
:10366000134BDE2A28BFDE222168184610F0CEFA5E
:10367000034666790F48257906700F48A1790570D1
:103680000E48E27903600E4B204619705A70FFF71E
:10369000F9FE082120460EF045F80A4BD2E70A4B06
:1036A000D0E700BFB57A010851050020CC7A0108A7
:1036B000640500204B0500204A0500204405002039
:1036C0004805002050050020B404002010B5044631
:1036D000006810B101210EF025F8204610BD000051
:1036E00070B54F4BC0B21B788AB0984201D14D4B98
:1036F0007DE00DF0BFF94C4904460DF03BF805465E
:10370000002877D0494A214601A80DF03CF8484AE4
:10371000214604A80DF037F8464A214607A80DF0C7
:1037200032F8079A0499019809F06EF907A8FFF793
:10373000CDFF04A8FFF7CAFF01A8FFF7C7FF3E4966
:1037400020460DF031F840B20AF02EFE09F0DEF806
:103750003A4920460DF028F8C0B20AF0F3FD09F00E
:10376000CBF837492046374C0DF004F809F01EF924
:10377000226812F0010212D10421334E0846326051
:1037800005F0B6FF306018B91121304800F0D8F8C4
:1037900001232F4A2F492C4823600EF028FE2E4B80
:1037A0001A680AB9284A1A602C4C226812F00102E1
:1037B00012D104212A4E0846326005F099FF30608C
:1037C00018B91121214800F0BBF80123204A2549EE
:1037D000234823600EF00BFE234B1A680AB9204AD7
:1037E0001A60224809F0F8F8002D80D0204B187894
:1037F0000AB070BD214601A81E4A0CF0C4FF214644
:1038000004A81D4A0CF0BFFF214607A81B4A0CF074
:10381000BAFF049A0799019809F0E4F886E700BF17
:103820004D050020B80400200E6701081A67010842
:10383000136701082167010893670108676701089A
:10384000D8A001082805002058050020A378010809
:10385000000000207F2E00083805002024050020ED
:1038600054050020712E000834050020053500089D
:103870004C050020386701083067010828670108F7
:10388000FF23094A1370094A1370094A1370094A41
:103890001370094A1370094A1370094A1370094AD0
:1038A0001370094A137070474E0500204D05002023
:1038B0004005002051050020500500204C05002047
:1038C0004F0500203005002031050020014B186015
:1038D000704700BFD006002073B5134C064623780E
:1038E0000D46124A1BB913780BB172B6FEE70123DD
:1038F000002113700E48642210F0B0F92B46009698
:103900000C4A64210A4811F02DF80B4B1B6803B1D7
:1039100098470125064E304603F01AFB72B6074B56
:103920002570013BFDD1F6E7B006002044060020DB
:1039300046060020597C0108D0060020FFFF0F003A
:10394000F7B5164C064623780D46154A1BB9137871
:103950000BB172B6FEE701230021137011486422F7
:1039600010F07CF92B4600960F4A64210D4810F0A8
:10397000F9FF0E4B1B6803B198470125094E0C4F08
:10398000304603F0E5FA384603F0E2FA72B64FF03B
:10399000FF332570013BFDD1F2E700BFB1060020E7
:1039A0004506002046060020817C0108D006002044
:1039B000907C01080368DFF888C080B5CCF800303F
:1039C000164F4368164E3B608368164D3360C368DC
:1039D00015492B600369154A0B604369144C136049
:1039E0008369C0692360134B1860DCF800003868F5
:1039F000306828680968104812680021226864222B
:103A00001B6810F02BF923680C4A64210A4810F057
:103A1000A9FF094803F09CFAFEE700BFC00600209A
:103A2000C8060020CC060020C4060020AC060020FA
:103A3000B4060020B806002046060020467C010897
:103A4000BC060020074B1B6803B198471EF0040F0B
:103A50000CBFEFF30880EFF309808169004A10473B
:103A6000B5390008D0060020002103E00A4B5B585E
:103A70004350043109480A4B42189A42F6D3094A86
:103A800002E0002342F8043B074B9A42F9D300F0CE
:103A90000DF8FDF71FF870475CBD0108000000201D
:103AA0007002002070020020C84E0020314B82B00E
:103AB0001A6842F480721A6099682F4A0A409A6024
:103AC0001A6822F0885222F001121A601A6822F451
:103AD00080221A609A6822F47D029A600022DA60DD
:103AE00001921B6813F4007318BF01230193019B1B
:103AF000012B37D14FF48051204B1A68A3F5806316
:103B000022F00102C3F80024D3F8002422F00202BC
:103B1000C3F80024D3F8002422F00402C3F80024E0
:103B20005A6A42F080525A62154A11605168C906B9
:103B3000FCD49A689A609A689A609A689A605A68FF
:103B400022F460425A605A6842F440425A609A68CD
:103B500022F003029A609A689A60064A936813F00A
:103B60000C0FFBD14FF00062064B9A60064ADA60F8
:103B700002B07047003802400CC0FF88003C024091
:103B80000070004000ED00E00003FA0570B5064645
:103B900088B02D4801F080FA2C4B1A680092009AE8
:103BA00091073AD501214FF4007001F0CFFC0120BC
:103BB00001F0C0FA264A536843F400335360A2F57B
:103BC000374253681B07FCD50024012502A801F0E9
:103BD0009DFA02A91C4806948DF81C50ADF80C40C3
:103BE00001F06EFA2A4606233146174801F0AEFA74
:103BF0002946154801F095FA0221134801F038FBD7
:103C0000114801F027FB134D01940F4C022120466F
:103C100001F028FB58B108B070BD1A6842F00102EB
:103C20001A60009A9207BDD41A680092F9E7019BC6
:103C300001330193019BB3F5805FE7DB3821284610
:103C4000FFF77EFEE2E700BF00240140003802409B
:103C500000270140AC7C010808B5002001F06AFA99
:103C60000021074801F05DFA00214FF4007001F0D7
:103C70006DFC044A136823F00103136008BD00BF04
:103C8000002401400038024013B5072301220146F9
:103C9000114801F05BFA02210F4801F0E9FA0E48E1
:103CA00001F0D8FA00230D4C019302210A4801F0DB
:103CB000D9FA28B1084802B0BDE8104001F0CFBAE7
:103CC000019B01330193019BB3F5805FEDDB4C2138
:103CD0002046FFF735FEE8E700240140AC7C0108F0
:103CE00070B506460825FFF751FF00243046FFF760
:103CF000CBFF013D0444F9D1FFF7AEFFC4F3CF0081
:103D000070BD00000000000008B51120FFF7E8FFBB
:103D10000FF03EFA014608480FF046FB0EF020FE79
:103D200003A3D3E900230EF073FE0FF02BF908BDB7
:103D30002FDD24068195F33F00F07F450F4A536A3B
:103D400043F0805353620E4B1A465968C906FCD49F
:103D50001B68022823F4C05306D143F4C0531360F8
:103D60005368DB06FCD47047012802D143F480532A
:103D7000F5E70028F3D143F40063F0E70038024090
:103D80000070004010B50C4B5A68D206FCD41C6879
:103D900014F4C05F0BD114F480500AD114F4006401
:103DA00004D106482A21FFF7CBFD204610BD022092
:103DB000FCE70120FAE700BF00700040F27C010838
:103DC00038B50546012001F063FA022D01BF144AFF
:103DD000136843F001031360124B1A6842F48072B7
:103DE0001A601A689205FCD55A6822F4604242F4BF
:103DF00040425A6000229A600A4B9C6814F00C04FE
:103E0000FBD14FF480721A60074B084A28461A60AB
:103E1000FFF794FF2046BDE8384001F02DBA00BFFF
:103E2000003C02400038024018000020D0FE3F0055
:103E30000C4B5A6B900513D45A6A42F080525A6266
:103E4000094A116841F480711160596B41F4807125
:103E50005963596B8905FCD5136823F4807313608B
:103E6000704700BF0038024000700040054B5A6B9D
:103E7000910706D45A6B42F001025A635A6B9207BB
:103E8000FCD5704700380240094B5A6A42F02002C4
:103E90005A629A6942F020029A619A6922F02002DD
:103EA0009A610022A3F509331A801A855A62704775
:103EB000003802401521002202384143064B1A8582
:103EC000D962012199825A621A8219801A8AD2070C
:103ED000FCD500221A80704700140040002349F6E8
:103EE000FE7282B00193019B934201DD02B07047E4
:103EF000019B01330193F6E7002340F6FE7282B086
:103F00000193019B934201DD02B07047019B013395
:103F10000193F6E7002382B00193019BB3F5CC7FB8
:103F200001DD02B07047019B0133F5E7D0B10128F4
:103F300001D1FFF7EFBF0C4B00211A684FF47A73E1
:103F4000B2FBF3F2094B013A92B21A850122013811
:103F5000D8629A82596219821A801A8AD207FCD5CD
:103F600000221A80704700BF180000200014004093
:103F700000F1774303F57803B3F5804F2DE9F04165
:103F800006460C4617462DD202F1F73303F6080316
:103F90000344B3F5804F25D2FFF7F4FE804610B1FD
:103FA0000020FFF7CBFE01F08BF901252744361BDB
:103FB000A7420AD101F094F9B8F1000F02D04046AF
:103FC000FFF7BCFE2846BDE8F08141F6027001F023
:103FD0008FF9301914F8011B01F0E6F9042818BF15
:103FE0000025E5E70025EDE710B50C4600F1774127
:103FF00001F57801B1F5804F0DD202F1F73303F6E8
:1040000008030344B3F5804F05D2014620460FF064
:10401000FDFD012010BD0020FCE7000008B5114B9C
:10402000984215D003F58063984213D003F580635E
:10403000984211D003F5806398420FD003F50063D6
:1040400098420DD0084B094A142109480FF0BEFCD4
:10405000002008BD0120FCE70220FAE70320F8E772
:104060000520F6E700000240817D01083B7D010844
:104070009A7D01080F2808B505D9094B094A3B214B
:1040800009480FF0A3FC012303FA00F0C043074ADC
:1040900051680140516013681840106008BD00BFAE
:1040A000E37D0108457D01089A7D01080004014077
:1040B0000F292DE9F84F82460D4693461F4605D934
:1040C0005A4B5B4A54215B480FF080FC4FF00109CA
:1040D00009FA05F900F0B8F86FEA0903564E032D06
:1040E0007268564C02EA03027260326803EA020305
:1040F000534A3360136A43F0010313622ED80F2230
:10410000A3684FEA850802FA08F223EA0203A360D3
:104110005046FFF783FFA36800FA08F01843A06039
:104120001BF0020F18BFB368464A1CBF43EA0903DD
:10413000B3601BF0040F1EBFF36843EA0903F3608A
:10414000336843EA090333603B01DBB2002D45D1FC
:1041500082F8063340231360BDE8F88F072D13D88B
:104160000F22A5F10408E3684FEA880802FA08F272
:1041700023EA0203E3605046FFF750FFE36800FACA
:1041800008F01843E060CBE70B2D13D80F22A5F100
:10419000080823694FEA880802FA08F223EA0203B2
:1041A00023615046FFF73AFF236900FA08F01843ED
:1041B0002061B5E70F22A5F10C0863694FEA880872
:1041C00002FA08F223EA020363615046FFF726FF72
:1041D000636900FA08F018436061A1E7012D03D17B
:1041E00082F807338023B6E7022D04D182F8083322
:1041F0004FF48073AFE7032D04D182F809334FF4F5
:104200000073A8E7042D04D182F80A334FF48063C9
:10421000A1E7092D04D882F817334FF400039AE779
:1042200082F828334FF48073536095E7EF7D0108DF
:10423000607D01089A7D01080004014000000140F2
:104240000038024000E100E0144B984205D1144AC6
:10425000D36943F00103D3617047124B984204D1F4
:104260000F4AD36943F00203F5E70F4B984204D19C
:104270000B4AD36943F00403EDE70C4B984204D199
:10428000074AD36943F00803E5E7094B9842E3D1B5
:10429000034AD36943F02003DDE700BF000002407A
:1042A000003802400004024000080240000C0240B6
:1042B000001402400323490010B584688B4024EAAF
:1042C000030484600124022A04FA01F407D0032ABB
:1042D0000DD0012A07D183682343836003E08368FC
:1042E0008A401A43826083681C43846010BD8268E0
:1042F0001343F2E70F29F8B504460F4615461E464C
:1043000003D940211948FFF71BFB2046FFF79CFF0C
:1043100003237A009340DB43216819402160012187
:10432000D4F800C001FA02F04CEA000CB940C4F81D
:1043300000C009B266B1A688314389B2A180E168A4
:10434000012D03EA0103E36006D0022D08D0F8BD79
:10435000A68826EA0101F1E7E3680343E360F6E794
:10436000E36805FA02F21A43E260F0E73F7E0108D3
:104370000F2970B505460C46164603D960210E4834
:10438000FFF7DEFA2846FFF75FFF032361008B404B
:10439000DB43EA68012E02EA0302EA6005D0022E3E
:1043A00003D02A6813402B6070BDEA6806FA01F159
:1043B0001143E960F5E700BF3F7E01080F2910B502
:1043C00005D9074B074A762107480FF0FFFAFFF798
:1043D0003BFF4B000321026899401143016010BD6F
:1043E000E37D0108FB7D01083F7E01080F2938B5F8
:1043F0000446154605D97C211B4B1C4A1C480FF06E
:10440000E5FA0F2A03D91B4B184A7D21F6E7FFF77F
:104410001BFF07294FF00F0318D8006A8A0093404A
:1044200020EA03032362236A05FA02F21A43226296
:104430000322236849008A4023EA020323600223FF
:10444000226803FA01F11143216038BDA1F108028D
:10445000406A9200934020EA03036362636A9540D6
:104460001D436562E4E700BFE37D01080E7E01089D
:104470003F7E01082C7E0108012303FA01F189B275
:1044800001837047012303FA01F189B24183704728
:10449000012303FA01F189B20AB101837047418314
:1044A0007047008A084100F0010070470F2938B5B5
:1044B00005460C4603D9A9210548FFF741FA2868AB
:1044C0006400E04000F00300431E5842584138BDEC
:1044D0003F7E0108808A0841C04300F00100704718
:1044E00010B5074C236853B9012005F0C9F92060C5
:1044F00028B9BDE8104036210248FFF721BA10BDA7
:10450000D4060020867E010810B50B4C22681AB92B
:104510003C210A48FFF714FA206842F2107105F0B6
:10452000F7FA01280CBF0124002403D040210348DE
:10453000FFF706FA204610BDD4060020867E01084B
:1045400010B5074C22681AB94D210648FFF7F8F953
:10455000002320681A46BDE81040194605F0ECB863
:10456000D4060020867E010810B50446FFF7B8FF88
:10457000FFF7CAFF21461022034801F07BFC0446E6
:10458000FFF7DEFF204610BD0054004010B5FFF7D6
:10459000A7FFFFF7B9FF01F025FC0446FFF7D0FFA6
:1045A000204610BD08B513460A460146034801F0EF
:1045B00091F8003018BF012008BD00BF0054004032
:1045C00008B513460A460146034801F089F9003050
:1045D00018BF012008BD00BF0054004008B51346B5
:1045E0000A460146034801F00FFA003018BF0120C7
:1045F00008BD00BF0054004008B513460A460146F6
:10460000034801F093FA003018BF012008BD00BF35
:104610000054004008B513460A460146034801F01D
:10462000DFFA003018BF012008BD00BF0054004071
:104630000123064A83405169194205D05361044B56
:1046400053F8203003B11847704700BF0004014001
:10465000D80600200F2838B504460D4603D9262178
:104660000348FFF76DF9034B43F8245038BD00BFF2
:10467000CC7E0108D80600200020FFF7D9BF01201A
:10468000FFF7D6BF0220FFF7D3BF0320FFF7D0BF4D
:104690000420FFF7CDBF08B50920FFF7C9FF0820A8
:1046A000FFF7C6FF0720FFF7C3FF0620FFF7C0FF95
:1046B000BDE808400520FFF7BBBF08B50F20FFF796
:1046C000B7FF0E20FFF7B4FF0D20FFF7B1FF0C205E
:1046D000FFF7AEFF0B20FFF7ABFFBDE808400A2055
:1046E000FFF7A6BFFEE7FEE7FEE7FEE7FEE7FEE711
:1046F000FEE7FEE7FEE7FEE7FEE7FEE7FEE7FEE792
:10470000FEE7FEE7FEE7FEE7FEE7FEE7FEE7FEE781
:10471000FEE7FEE7FEE7FEE7FEE7FEE7FEE7FEE771
:10472000FEE7FEE7FEE7FEE7FEE7FEE7FEE7FEE761
:10473000FEE7FEE70A23B0FBF3F203FB120040EAB8
:104740000210C0B270470000CA22024B5A625322C4
:104750005A62704700280040014B1860704700BF44
:10476000180700204FF400320F4B10B50F4C5A6160
:10477000E368DB0503D430210D48FFF7E1F8FFF7CC
:10478000E3FF4FF40072A36823F48853A360094B3E
:10479000C3F88420FF236362074B1B6813B1BDE895
:1047A0001040184710BD00BF000401400028004021
:1047B000127F010800E100E0180700202DE9FF4703
:1047C0009A46364B80461B7891469DF830709DF88E
:1047D00034602BB9324B334A8C2133480FF0F6F852
:1047E000431E1E2B58D80C2956D8A2F5FA63632B0A
:1047F00052D8BAF1170F4FD83B2F4DD83B2E4BD87C
:1048000002F13000C0B2FFF795FF05460846FFF7FA
:1048100091FF000240EA05454046FFF78BFF054344
:104820005046FFF787FF04463846FFF783FF000234
:1048300040EA04443046FFF77DFF20431B4CFFF75E
:1048400083FFE36845F4005543F08003E360E368C9
:104850005B06FCD565602060E36823F08003E360BD
:10486000124BDA689206FCD5FF2201A85A628DF835
:1048700007808DF80810ADF809908DF806A08DF826
:1048800005708DF8046002F05CFA094BC3E9000181
:10489000012004B0BDE8F0870020FAE71C070020E3
:1048A00045A601086A7F0108127F01080028004020
:1048B0002007002007B5037801934378009383789D
:1048C000B0F805200179C078FFF778FF03B05DF8F4
:1048D00004FB000038B52B4B04461B781BB9E421C0
:1048E0002948FFF72DF8294AD36823F02003D36025
:1048F000D3689B06FCD513685268C2F307410809C8
:1049000000EB800001F00F0101EB4001C9B201F59D
:10491000FA61A4F80510C2F30721C1F30010850065
:10492000284401F00F0101EB4001D2B22171C2F322
:10493000011101EB810102F00F0202EB4102E27072
:10494000C3F30742C2F3011101EB810102F00F0230
:1049500002EB4102A270C3F30722C2F3021101EB82
:10496000810102F00F0202EB4102DBB26270C3F37D
:10497000021202EB820203F00F0303EB42032370E7
:1049800038BD00BF1C070020127F0108002800402E
:104990001FB501A8FFF79EFF01A802F0D2F905B0EC
:1049A0005DF804FB08B5FFF743FA1B4A136843F4AC
:1049B00080731360FFF7C8FE184A536B23F440332B
:1049C00043F482035363164BDA6842F08002DA60E4
:1049D000DA685106FCD5FF221A611A6942F4FE0218
:1049E0001A619A6822F040029A609A6822F44C5246
:1049F0009A60DA6822F08002DA60094BDA6892067F
:104A0000FCD5FF225A620122064B1A70FFF7C0FF45
:104A1000054BC3E9000108BD0070004000380240AA
:104A2000002800401C0700202007002008B5094B83
:104A30001B7823B940F21F110748FEF781FFFFF7EB
:104A400083FE064B9A6822F480729A60FF225A62B3
:104A500008BD00BF1C070020127F0108002800408D
:104A600008B5144B1B7833B9134B144A40F2271185
:104A700013480EF0ABFFFFF767FE124BDA6822F423
:104A80008072DA60104A916841F4003191601168D7
:104A900041F400311160F0210C4A82F829134FF4DF
:104AA000007151609A6842F488529A60FF225A62FB
:104AB00008BD00BF1C07002045A60108767F01083D
:104AC000127F0108002800400004014000E100E0DE
:104AD000F8B51E46194B17461B7833B9184B194ABF
:104AE0004FF4A37118480EF071FF184CFFF72CFE1D
:104AF000A56825F48075A560E56825F48075E560F6
:104B0000FFF718FE05460846FFF714FE000440EACA
:104B100005613846FFF70EFE05463046FFF70AFEF0
:104B2000084340EA0520E368DB07FCD5FF23E0618A
:104B30006362BDE8F840FFF793BF00BF1C07002089
:104B400045A60108587F0108127F0108002800408F
:104B500038B50D46044604F005FB194A136823F0E6
:104B60000103136004F01EFB25B1164A536843F09D
:104B70000603536072B6BFF34F8FBFF36F8F124AB5
:104B80000120136823F0030343F4007343F001038F
:104B9000136000F089FB0D4B1A6942F004021A61A0
:104BA00030BF1A69022022F004021A61FFF708F9E7
:104BB000034A136843F00103136004B162B638BDC1
:104BC00010E000E0002004E00070004000ED00E094
:104BD00062B6704700220E4B10B51A700D4A0E4C8B
:104BE0001388204623F040031B041B0C13800D2167
:104BF0000222FFF7BDFB204602220E21FFF7B8FB81
:104C00002046BDE8104002220F21FFF7B1BB00BFD4
:104C1000280700200038004000040240294A38B527
:104C2000136A054643F480531362052226480C4656
:104C30001146FFF7DBFB052206212348FFF7D6FBD1
:104C4000052207212048FFF7D1FBC5B1022205212B
:104C50001D48FFF72FFB022206211B48FFF72AFB06
:104C6000022207211848FFF725FB012C1BD144F431
:104C700051740122154B1C80154B1A7038BD2A4601
:104C800005211148FFF716FB2A4606210E48FFF7BB
:104C900011FB2A4607210C48FFF70CFB012C09D118
:104CA00044F45974E5E7022CE1D0032C0CBF032433
:104CB0000024DCE7022CF3D0032C14BF00240324CF
:104CC000EEE700BF00380240000002400030014023
:104CD0002907002000220E4B10B51A700D4A0E4C09
:104CE0001388204623F040031B041B0C138005216E
:104CF0000222FFF73DFB204602220621FFF738FB88
:104D00002046BDE8104002220721FFF731BB00BF5B
:104D1000290700200030014000000240064B074AEE
:104D2000988111781A461889C00701D40029FAD150
:104D30009089C0B2704700BF0030014029070020B1
:104D4000054AD36823F4E0631B041B0C43F0BF63E4
:104D500043F40033D360704700ED00E020220021CF
:104D6000114B10B5C3F88420104B114C1A6A204621
:104D700042F480421A625A6942F480425A615A6986
:104D800022F480425A610B4A91811A6A092122F465
:104D900080421A620222FFF7EBFA2046BDE810407B
:104DA00002220A21FFF7E4BA00E100E000380240E5
:104DB000000002400038014010B50B4C40F2255174
:104DC000204600F060FC48B1204600F03AFC074B5A
:104DD0001B683BB1BDE81040C0B21847A388044A25
:104DE000DBB2137010BD00BF003801402C0700205B
:104DF000E44D002010B504468021084800F03DFC39
:104E00000028F9D02146054800F017FC034C40214A
:104E1000204600F032FC0028F9D010BD00380140D7
:104E200010B5441E14F8010F00B910BDFFF7E2FFE2
:104E3000F8E7000008B5024800F003FCC0B208BD66
:104E4000003801402DE9F0410F4601214FF4C066C2
:104E5000804688B0084614461D4600F069FB0121D3
:104E60004FF4804000F072FB3B4B02A93B48CDE978
:104E7000026300F0BFFA07220921384800F0FCFA6B
:104E800007220A21354800F0F7FA452FCDF81080A7
:104E90003AD14FF48063ADF81830072C40D100238D
:104EA000ADF81430052D4CD14FF48053ADF81630C9
:104EB0000023ADF81C300C2304A92948ADF81A30A2
:104EC00000F060FB274B1A6802B1012240F2255125
:104ED000234800F0BAFB0121214800F0A3FBFFF7B3
:104EE000A9FF25238DF804309DF838308DF8053062
:104EF0004FF48073ADF80630FFF722FF01A800F0F1
:104F0000AFF808B0BDE8F0814F2F02D1ADF81860BE
:104F1000C3E70023072CADF818300DD1592107E065
:104F2000082C02D14FF48053BAE7092CBAD154218E
:104F30000D48FEF705FDB5E7082CB0D0092CB1D11E
:104F4000F0E70F2D02D14FF44053AFE7022D0CBF15
:104F50004FF400530023A9E70202000100000240C1
:104F6000003801402C0700208B7F01080E2307B575
:104F7000082200934E210123FFF764FF03B05DF880
:104F800004FB000070B5134C40F22551204600F0A0
:104F90007AFBC0B1104B1D6825B1204600F051FBD3
:104FA000C0B2A84740F226610A4800F06CFB78B115
:104FB00040F22661074800F085FB084B1B683BB1B7
:104FC000BDE870401847A388054ADBB21370E9E7D3
:104FD00070BD00BF004400403007002034070020AF
:104FE000E44D0020BFF34F8F0449054BCA6802F41B
:104FF000E0621343CB60BFF34F8FFEE700ED00E0AC
:105000000400FA0510B5441EE3B2052B03D90E21A6
:105010001148FEF795FCFEF729FF45F255520F4B5C
:105020001A60DA68D207FCD4052C06D8DFE804F051
:10503000030A0C0E101201225A604CF6CC42074BA8
:105040001A6010BD0222F7E70322F5E70422F3E716
:105050000522F1E70622EFE7D27F01080030004089
:1050600030B5012403780A4D03F01F029440C27842
:10507000590952B1074A2B44D26842781201D2B280
:1050800083F8002345F8214030BD2031FAE700BF06
:1050900000E100E000ED00E008B5084B98420BD1BC
:1050A00001214FF4007000F05FFABDE808400021D4
:1050B0004FF4007000F058BA08BD00BF0024014052
:1050C00043680A7923F0407323F4807343EA022390
:1050D0000A6810B513434360D1E9032313438A6878
:1050E00084681343084A224013434A7943EA42033F
:1050F00083600A7D036B013A23F0F873D2B243EA6E
:105100000253036310BD00BFFDF7FFC000234FF043
:105110004072036083808360C0E903230123037529
:105120007047836819B143F001038360704723F02F
:105130000103FAE7044B5A6818B142F400025A60BE
:10514000704722F40002FAE7002701401D2970B5DC
:105150001BD90725A1F11E06C46D06EB4606B54016
:1051600024EA050403FA06F62643C665062A38D85B
:105170001F24013A036C02EB8202944023EA0403E9
:1051800001FA02F21A43026470BD13290DD90726F1
:10519000A1F11405C46805EB4505AE4024EA0604F8
:1051A00003FA05F52543C560E0E709290DD907266F
:1051B000A1F10A04056904EB4404A64025EA0605AA
:1051C00003FA04F42C430461D0E70726446901EB99
:1051D0004105AE4024EA060403FA05F6264346617B
:1051E000C4E70C2A0CD81F24073AC36B02EB8202D7
:1051F000944023EA040301FA02F21A43C263C3E7AC
:10520000122A0CD81F240D3A836B02EB82029440C1
:1052100023EA040301FA02F21A438263B4E7182A6C
:105220000CD81F24133A436B02EB8202944023EA0A
:10523000040301FA02F21A434263A5E71F24193A54
:10524000036B02EB8202944023EA0403914019436A
:10525000016399E7836843F0804383607047806D02
:1052600080B270470368194214BF012000207047C4
:10527000C943016070470000044B1A6818B142F03E
:1052800002021A60704722F00202FAE7003C024074
:10529000044B1A6818B142F004021A60704722F0F9
:1052A0000402FAE7003C0240044B1A6818B142F0CD
:1052B00008021A60704722F00802FAE7003C024038
:1052C000044B5A68D20741BF034ADA60034ADA60E6
:1052D000704700BF003C0240EFCDAB8905040302DC
:1052E000024A536843F0010353607047003C024098
:1052F000014B9861704700BF003C0240084B9A691F
:10530000D10709D49A69D20508D49B6913F4F05FD8
:1053100014BF03200420704701207047022070470B
:10532000003C0240042313B504468DF80730FFF714
:10533000E5FF8DF807009DF80730012B0AD11CB955
:1053400005238DF8073007E0FFF7D8FF013C8DF803
:105350000700F0E7002CF3D09DF8070002B010BD65
:1053600010B504464FF40040FFF7DCFF042804BFEB
:105370000023236010BD000038B504464FF4004000
:105380000D46FFF7CFFF04280BD1064A4FF400402B
:10539000536823F4807353602560BDE83840FFF7FD
:1053A000C1BF38BD003C024038B504464FF4004050
:1053B0000D46FFF7B7FF04281BD135B125704FF418
:1053C0000040BDE83840FFF7ADBFFF2324F00305E0
:1053D00004F003042968E40003FA04F421EA040455
:1053E0002846FFF7BDFF21462846BDE83840FFF7B5
:1053F000C3BF38BD2DE9F0430022012703250E6805
:1054000007FA02F333EA060431D14FEA420C05FAF7
:105410000CF4E44391F804E0D0F800900EFA0CF894
:1054200004EA09090EF1FF3E48EA0908BEF1010F3E
:10543000C0F8008011D8D0F808E004EA0E0E4C79CC
:1054400004FA0CF444EA0E048460848824EA030419
:105450008B7993409BB223438380C36805FA0CF495
:1054600023EA0404CB7903FA0CF32343C36001322B
:10547000102AC5D1BDE8F08310B50F2401F0070351
:10548000C90800EB8100016A9B009C4021EA0401ED
:105490000162016A9A400A43026210BD204B10B5B6
:1054A0009A6802F00C020C2A30D8DFE802F02F2FA5
:1054B0002F2F072F2F2F072F2F2F2000194B184A80
:1054C000036093681849C3F30313CC5C0368E3409B
:1054D00043609468C4F302240C5D23FA04F48460EE
:1054E0009268C2F3C2228A5CD340C36010BD99683F
:1054F0000E4CC1F383419A68615C9B68094BC2F30F
:1055000081524B430132B3FBF2F3D8E74FF4004230
:105510005B68C3F34233013302FA03F3CFE700BF02
:10552000003802400024F4001C0000202C00002061
:10553000054B19B1D9690143D9617047DA6922EA8B
:105540000002DA61704700BF00380240054B19B114
:10555000196A0143196270471A6A22EA00021A6244
:10556000704700BF00380240054B19B1596901432B
:10557000596170475A6922EA00025A61704700BFB8
:105580000038024030B50D460446028AEB8892B2DC
:1055900022F440521A43898902828389288923F49C
:1055A000B052AB8822F00C020343688985B00343F4
:1055B0001343A381A38A68469BB223F440730B4331
:1055C000A382FFF76BFFDDE90213154A944208BF7F
:1055D00019461923A2894B43296810044CBF49007E
:1055E0008900B3FBF1F16425B1FBF5F3A289180141
:1055F000120405FB13130BD5DA003232B2FBF5F2BD
:1056000002F0070242EA00039BB2238105B030BDDD
:105610001B013233B3FBF5F303F00F030343F3E74E
:1056200000380140838919B143F4005383817047E6
:1056300023F400531B041B0CF8E7C1F3080181801D
:1056400070478088C0F30800704701F01F0310B551
:10565000C1F342140121012C01FA03F105D10C30F0
:1056600003683AB11943016010BD022C0CBF103021
:105670001430F5E723EA0101F5E70388194214BF66
:105680000120002070470123C1F3421210B5012A06
:1056900001F01F0403FA04F30DD18289134002883C
:1056A00092B26BB10123090A03FA01F10A4214BF55
:1056B0001846002010BD022A0CBF028A828AEDE73C
:1056C0001846F7E70123090A8B40DB439BB20380AE
:1056D000704700002DE9F3411F46002304460E46A3
:1056E000019315461AB9012002B0BDE8F08140F6D9
:1056F000FF7301934FF40031204600F014FD0028A1
:1057000052D10121204600F0DEFC4FF2FF7120460D
:1057100000F0F2FC0121204600F0BFFC40F6FF73D0
:10572000DFF8B88101934146204600F0F1FC0028E3
:1057300041D039460122204600F0D0FC40F6FF73EC
:10574000614F01933946204600F0EDFC002838D027
:10575000012D42D10021204600F0B5FC03F002FDEE
:1057600029462046238B00F0A3FC03F01BFD40F6E6
:10577000FF73564D01932946204600F0D4FC30B308
:10578000204600F0B6FC307040F6FF73504D019398
:105790002946204600F0C7FC0028A4D0019B5A1ED1
:1057A0000192002BF4D104E0019B5A1E0192002BC0
:1057B000A0D1002098E7019B5A1E0192002BB2D184
:1057C000F7E7019B5A1E0192002BBBD1F1E7019B29
:1057D0005A1E0192002BCED1EBE7022D25D103F00A
:1057E000C1FC4FF40061204600F086FC00212046F9
:1057F00000F069FC238B03F0D5FC40F6FF73354DB8
:1058000001932946204600F08EFC40B1012120463C
:1058100000F04EFC238A3370238A7370B4E7019B37
:105820005A1E0192002BECD1C3E740F6FF77033DEF
:10583000238BDFF8A0803544AE4201972CD1254E52
:105840003146204600F06FFC90B30021204600F066
:105850003AFC03F087FC204600F04BFC0121287045
:10586000204600F025FC03F09DFC204600F041FCA2
:1058700040F6FF73184E687001933146204600F0E1
:1058800047FCD8B1204600F034FCA8707CE7019BAF
:105890005A1E0192002B8CD04146204600F043FC5A
:1058A0000028F4D0204600F024FC06F8010BC3E7E2
:1058B000019B5A1E0192002BC2D17AE7019B5A1E0E
:1058C0000192002BD9D174E70200001040000010B3
:1058D000100000100400001040000300010003004D
:1058E0002DE9F3411D46002304460E460193174659
:1058F0001AB9012002B0BDE8F08140F6FF730193B0
:105900004FF40031204600F00EFC002847D1012161
:10591000204600F0C2FB40F6FF73DFF8E8800193F9
:105920004146204600F0F4FB00283FD029460022E3
:10593000204600F0D3FB40F6FF732E4D019329461D
:10594000204600F0E5FB002836D03546204615F805
:10595000011B3E4400F0CBFB40F6FF77DFF8988058
:10596000B542019733D1244D2946204600F0DBFB98
:10597000002838D02046012100F09AFB40F6FF7342
:105980001E4D1F4C01932946204600F0CCFB0028F9
:10599000AFD0019B5A1E0192002BF4D104E0019B71
:1059A0005A1E0192002BABD10020A3E7019B5A1E87
:1059B0000192002BB4D1F7E7019B5A1E0192002BF4
:1059C000BDD1F1E7019B5A1E0192002BECD041465C
:1059D000204600F0A8FB0028F4D015F8011B204653
:1059E00000F085FBBCE7019B5A1E0192002BBBD146
:1059F000DAE700BF8200070004000010100000106A
:105A000000540040010003002DE9F3411D4600232E
:105A100004460E46019317461AB9012002B0BDE8AC
:105A2000F08140F6FF7301934FF40031204600F0FF
:105A30007AFB002838D10121204600F02EFB40F6E9
:105A4000FF73DFF8E48001934146204600F060FBDD
:105A5000002843D029460022204600F03FFB40F6B4
:105A6000FF732D4D01932946204600F051FB00287D
:105A70003AD03546204615F8011B3E4400F037FB6E
:105A800040F6FF77DFF89480B542019737D1234D78
:105A90002946204600F047FB0028BED1019B5A1E34
:105AA0000192002BF4D104E0019B5A1E0192002BBD
:105AB000BAD12046012100F0FBFA40F6FF73184DE1
:105AC000184C01932946204600F02DFB20B1019B84
:105AD0005A1E0192002BF5D100209FE7019B5A1E10
:105AE0000192002BB0D1E4E7019B5A1E0192002BDA
:105AF000B9D1DEE7019B5A1E0192002BD9D0414655
:105B0000204600F010FB0028F4D015F8011B2046B9
:105B100000F0EDFAB8E700BF8200070004000010B3
:105B200010000010005400400100030000232DE984
:105B3000F3410E464FF4003104461746019300F03E
:105B4000F2FA18B9002002B0BDE8F0810FB90120C7
:105B5000F9E73546204615F8011B3E4400F0C7FA28
:105B600040F6FF77DFF86C80B54201971FD1194DE1
:105B70002946204600F0D7FA28B32046012100F03C
:105B800097FA40F6FF73144D144C019329462046B2
:105B900000F0C9FA0028DAD0019B5A1E0192002BAE
:105BA000F4D1CFE7019B5A1E0192002BCAD0414687
:105BB000204600F0B8FA0028F4D015F8011B204662
:105BC00000F095FAD0E7019B5A1E0192002BCFD12D
:105BD000B8E700BF0400001010000010005400409F
:105BE0002DE9F3411F46002304460E460193154656
:105BF0001AB9012002B0BDE8F0814FF4003100F085
:105C000092FA08B90020F5E70121204600F05BFA7E
:105C10004FF2FF71204600F06FFA0121204600F09C
:105C20003CFA40F6FF73DFF8B88101934146204605
:105C300000F06EFA00283AD039460122204600F0E2
:105C40004DFA40F6FF73614F01933946204600F04C
:105C50006AFA002831D0012D3BD10021204600F006
:105C600032FA03F07FFA29462046238B00F020FA0F
:105C700003F098FA40F6FF73554D019329462046EC
:105C800000F051FAF8B1204600F033FA307040F6D7
:105C9000FF73504D01932946204600F044FA002836
:105CA000A7D0019B5A1E0192002BF4D1AAE7019BB9
:105CB0005A1E0192002BB9D1A4E7019B5A1E0192F2
:105CC000002BC2D19EE7019B5A1E0192002BD5D119
:105CD00098E7022D29D14FF40061204600F00CFA1C
:105CE00003F040FA00212046238B00F0ECF903F08A
:105CF00059FA40F6FF73384D01932946204600F0CB
:105D000012FA60B103F02EFA0121204600F0D0F91A
:105D1000238A3370238A737003F044FAB7E7019B38
:105D20005A1E0192002BE8D16CE740F6FF77033D45
:105D3000238BDFF8A4803544AE4201972DD1264E47
:105D40003146204600F0EFF998B30021204600F0DC
:105D5000BAF903F007FA204600F0CBF901212870C8
:105D6000204600F0A5F903F01DFA204600F0C1F925
:105D700040F6FF73194E687001933146204600F0DB
:105D8000C7F9E0B1204600F0B4F9A8707FE7019BA5
:105D90005A1E0192002B3FF435AF4146204600F0D9
:105DA000C2F90028F3D0204600F0A3F906F8010B51
:105DB000C2E7019B5A1E0192002BC1D122E7019B31
:105DC0005A1E0192002BD8D11CE700BF0200001020
:105DD00040000010100000100400001040000300FC
:105DE0000100030038B5204B08219A691F4842F48E
:105DF00000129A619A6922F400129A615A6A22F496
:105E000000125A62FEF738FB012308211A46174890
:105E1000FEF770FA092115480122FEF7A9FA0921B7
:105E20001248FEF73EFBD8B1012038BD08212846B4
:105E3000FEF722FBFEF76EF808212846FEF722FB4C
:105E4000FEF768F8013CF1D109210848FEF729FB6B
:105E500020B940F263110648FDF772FD2046E4E7E1
:105E60003324024DEEE700BF003802400004024038
:105E70001D8001082DE9FF41444B054698420E461E
:105E800017467CD103F5F2335A6A082142F4001216
:105E90005A629A693E4842F400129A619A6922F461
:105EA00000129A61FEF7E8FA012308211A463848E1
:105EB000FEF720FA092136480122FEF759FA092196
:105EC0003348FEF7EEFA002855D0012308211A4680
:105ED0002F48FEF70FFA042208212D48FEF786FA14
:105EE000012309211A462A48FEF704FA042209214F
:105EF0002748FEF77BFA274B9A6942F400129A6111
:105F00009A6922F400129A61684600F0ADF8224BBB
:105F1000694601934FF48063ADF80A304FF4804333
:105F20002846ADF80C30ADF80870009600F038F84F
:105F30002846012100F0A6F8012019E0082140467A
:105F4000FEF79AFAFDF7E6FF08214046FEF79AFAB7
:105F5000FDF7E0FF013CF1D109210D48FEF7A1FA60
:105F60000028B2D10D4840F28B11FDF7E9FC204624
:105F700004B0BDE8F0813324DFF81480EAE74FF481
:105F8000CD710648FDF7DCFCBEE700BF00540040C1
:105F900000040240003802400000FFBF1D800108DD
:105FA0007FB50446868868460D46FFF777FA029A61
:105FB0002B4926F03F06B2FBF1F13604360C88B2CD
:105FC0000643A6802388274E23F001031B041B0CE5
:105FD00023802B68B3421ED85B00B2FBF3F39BB265
:105FE000042B38BF0423013080B22084A38323888C
:105FF000AA8843F0010323802388698923F48163FD
:106000000A4323F00203134323802A89AB891343F5
:10601000238104B070BD4BF6FF70EE8886421BBF33
:106020001920434303EB4303B2FBF3F30BBFB2FB73
:10603000F3F39BB29BB243F48043C3F30B020AB960
:1060400043F001034FF496724A434FF47A71B2FB66
:10605000F1F2013292B243F400432284C6E700BF5A
:1060600040420F00A086010041F28832044BC0E993
:106070000023002383604FF480438381704700BF77
:106080000000FFBF038819B143F00103038070478C
:1060900023F001031B041B0CF8E7038819B143F438
:1060A00080730380704723F480731B041B0CF8E794
:1060B000038819B143F400730380704723F400731D
:1060C0001B041B0CF8E7038819B143F480630380B9
:1060D000704723F480631B041B0CF8E722B141F0E6
:1060E000010189B20182704701F0FE01F9E70182E6
:1060F0007047008AC0B270470388B1F5006F1BBFBC
:1061000023F400631B0443F400631B0C03807047FB
:10611000838A008B43EA00430B4023F07F435B1AE2
:10612000584258417047002382B0009301930B0FEF
:1061300001900093009B21F07F4153B1019B1433E8
:106140000193019B1B680B4214BF0120002002B089
:106150007047019B090C1833F2E7F8B50E46054667
:1061600080B14F1C384600F03BFF044640B13A4630
:1061700000210DF073FD3246294620460DF046FD04
:106180002046F8BD0446FBE738B50D46044628B165
:106190000EF04EFC23462044834201D1002038BD3E
:1061A00013F8012BAA42F7D10120F8E773B5054691
:1061B0000E4600240DF036FC2246046001A9284654
:1061C0000EF04AFD05460DF02DFC0368222B0BD086
:1061D000019B1B7843B9A542ADBF28462046012349
:1061E0002346336002B070BD01232046F9E700006A
:1061F0002DE9F04F05464FF0010B002687B0CDE9A1
:10620000031206F10903122B8CBF0320022000F0B9
:10621000E7FE0090E8B1324636490EF0D7FB039B0B
:1062200053F82690EDB90024009800F0C3FEBBF1AE
:10623000000F02D1284600F0BDFE84B1049B013658
:10624000B34225464FF0000BDBD1204607B0BDE836
:10625000F08FBBF1000F02D1284600F0ABFE002406
:10626000F3E7254B4FF00008B9F1000F08BF99463E
:1062700048460EF0DDFB019000980EF0D9FB02902D
:10628000284649460EF001FCB8B928460EF0D0FB6E
:10629000DDE9012301309B1A08FB030000F0A0FE9A
:1062A00004460028BFD003462F4618F1FF3809D214
:1062B000394618460EF0B4FBB6E7019B08F1010819
:1062C0001844DEE74946384605930EF0DEFB059B91
:1062D000A0EB070A5246394618460EF0C3FB009958
:1062E00050440EF09DFB019A029B9244C318574400
:1062F000DBE700BF85810108BE6F010830B580B1C2
:106300000346021F00F1180452F8045F8D4208D0C2
:10631000A242F9D11C301A4614680433013401D169
:10632000116030BD8342F6D1FBE7000068B1084937
:10633000431E13F8010F00B970470A5C02F0030214
:10634000022A08BF20381870F3E70120704700BF09
:1063500091BA010870B5044680B1064600EB81058C
:10636000AE4204D12046BDE8704000F023BE56F88E
:10637000040B0028F4D000F01DFEF1E770BD000012
:106380002DE9F74F8B460092002839D00027C35DD6
:1063900093BB1D46064600EB070A024638485245A5
:1063A00038D103B10135002D63D00137384600F0F4
:1063B00017FE804600285AD03A4600210DF04EFCC8
:1063C000A80000F00DFE0446002854D04FF000094C
:1063D0000021B2452CD131B14046FFF7BEFE002866
:1063E00049D044F82900404600F0E4FD009B1D60C0
:1063F000204603B0BDE8F08F0137B7F5807FC6D1E6
:1064000000242546204600242946FFF7A3FF009BD1
:106410001C60EDE712F8011B594504D1002BBED0DA
:1064200001350023BBE7095C090758BF0133B6E714
:1064300016F8013B5B4512D10029CAD04046FFF750
:106440008CFEC0B109F1010344F829003A4600214D
:10645000404601930DF002FC019B9946B8E7084ABB
:10646000985C02075CBF08F801300131B1E70446CF
:10647000C8E72C46BCE7404600F09CFDC2E700BFE1
:1064800091BA01082DE9F743002506460820884601
:1064900091461F46009500F0A3FD0446002865D0F4
:1064A000C0E9005530460EF0C3FA01280FD1337809
:1064B0002A2B0CD109F1FF33C4F8008063602268F5
:1064C0004A4502D263684B4540D3294B0DE02D214C
:1064D0003046FFF759FE0546B8B9019001A930468C
:1064E000FFF764FE019B63B1224B3B600099284695
:1064F000FFF730FF002C35D0204600F05BFD002474
:1065000030E0C4E900001D46D9E76A462D21304637
:10651000FFF736FF009B0546013B012B01D9164BC7
:10652000E3E7002301A900680193FFF73FFE206025
:10653000019B0BB1114BD8E701A96868FFF736FE44
:106540006060019B002BBAD00D4BCEE7424501D3D2
:10655000434501D20B4BC8E700992846FFF7FAFEE6
:1065600000233B60204603B0BDE8F0830546BDE74D
:1065700040810108BA800108D98001080281010820
:10658000218101086081010808B520B34A1C22D08E
:10659000062920D8DFE801F0040D101316191C009D
:1065A000002303600DF03CFC0840431C5842584156
:1065B00008BD00234360F5E700238360F2E7002372
:1065C0008361EFE70123C360ECE700230361E9E7A0
:1065D00000234361E6E70120EAE770B506460D1F98
:1065E00001F1180455F8041F4B1C03D1A542F9D141
:1065F000002070BD3046FFF7C7FF0028F6D0F8E74F
:1066000000290B46B8BFCB1D4A4202F0070201F039
:10661000070158BF51420122C3F3C703C9B202FAAE
:1066200001F1C25C1143C154704700290B46B8BF49
:10663000CB1D4A4202F0070201F0070158BF514248
:106640000122C3F3C703C9B28A40C15C21EA020137
:10665000C15470470B460029B8BFCB1DC3F3C70315
:10666000C05C4B4203F0070301F0070158BF5942D9
:10667000C9B2084100F0010070472DE9F047089EBB
:106680008A4690461D46DDF82890074610B114460C
:10669000A24507D875B9012200240B9B1A60204639
:1066A000BDE8F08721463846FFF7D4FF00285ED1C9
:1066B0000134EDE7099B023B042B04D8DFE803F02B
:1066C000282C2C3034006B6801336B6028460DF0A9
:1066D000A7FB013108BFB0F1FF3FDCD031462846AF
:1066E000FFF752FF0028D6D117B30446214638469B
:1066F000FFF7B0FF00283FD10134A245F6D1044690
:10670000013E042E16D8DFE806F0282A2C2E300091
:10671000AB680133AB60D9E7EB680133EB60D5E7D9
:106720002B6901332B61D1E76B6901336B61CDE7D5
:106730003C46E5E72C6028460DF072FB013108BFAE
:10674000B0F1FF3FA7D0B9F1000FA4D049462846C9
:10675000FFF743FF0028A2D09DE76C60EBE7AC6039
:10676000E9E7AC61E7E7EC60E5E72C61E3E7A0452A
:1067700095D0002DC4D18EE7A045C1D18FE72DE97A
:10678000F04F4FF000098BB006461C200C46904697
:10679000CDF8249000F024FC0546002800F0E080AD
:1067A0001C2000F01DFC0746002800F0D9804B4655
:1067B0004FF0FF3245F8232047F823200133072B01
:1067C000F8D100230121D4F800A00DF12409CDE96E
:1067D0000031CDE902793C21234652463046FFF78D
:1067E0004CFF0999002940F08E80824502D128464D
:1067F000FFF784FD02234FF0010AD4F804B0CDE97D
:1068000000A3CDE9025923465A463C2106F108006F
:10681000FFF733FF099B002B75D183456BD15146A0
:106820002846FFF76BFD03234FF0020AD4F808B0A7
:10683000CDE900A3CDE9025923465A46182106F1B5
:106840001000FFF71AFF099B002B5CD1834565D12F
:1068500051462846FFF752FD40F26F1BA36905938E
:10686000E368049306F114030693DDF810A006F123
:106870001303079351460698FFF7ECFE20B10599E4
:106880000798FFF7E7FE88B9BBF1010B0ED0E3686C
:1068900020460133E3600DF0C3FA013108BFB0F1C7
:1068A000FF3F44D101234FF0000A0993099B53BBDA
:1068B000049B534544D104212846FFF71FFD0523BF
:1068C0000622D4F810A0CDE90032CDE902592346C2
:1068D00052460C2106F11800FFF7CFFE099B93B931
:1068E000824510D06369A3EB0803042B31D94FF024
:1068F000FF33099307E0424621463046FFF73FFF4A
:10690000099000288FD0284600F054FB17B1384674
:1069100000F050FB09980BB0BDE8F08F42462146CD
:106920003046FFF72CFF0990002895D0EBE7A369CC
:1069300029462046D4F80CA00593FFF74EFE99E7B0
:10694000424621463046FFF71AFF09900028B6D08C
:10695000D9E7424621463046FFF711FF0990D2E7BA
:106960004FF0FF330993002DD4D00027CBE7000070
:106970002DE9F04F002487B0894692462C2103AAC6
:106980009846109D0394FFF7FBFC074688B93E4BE1
:106990002B6003993846FFF7DDFC07B0BDE8F08FA8
:1069A000D0F800B072685A451CD2304600F002FBA5
:1069B0000134039BA342ECD957F824602F213046C1
:1069C000FFF7E2FBA8B92B46304642465146FFF797
:1069D00059FD2B680646002BE2D00028D9D000F0E4
:1069E000E9FAD6E759464846FFF70AFE0BF1010BD4
:1069F000D8E700232F21304604AA0493FFF7C0FCF8
:106A0000049906464B1E012B04D9204B2B60FFF73F
:106A1000A1FCBEE742462B4651460068FFF732FD17
:106A20002A6883462AB108B100F0C4FA04993046B6
:106A3000EDE72D213068FFF7A7FB18B908F1FF3209
:106A4000CBF80420002305A970680593FFF7AEFB7F
:106A5000059A00901AB10E4A58462A60E4E7DBF81E
:106A60000020DBF80410914205D230460499FFF76C
:106A700071FC58469AE7114648460192FFF7C0FD5F
:106A8000DDE900321A44ECE7888101089A810108A7
:106A9000BF8101082DE9FF4100230E4603931446F0
:106AA00002B902AC236048B90546564B23600399EE
:106AB0002846FFF74FFC04B0BDE8F08103AA20216F
:106AC000FFF75EFC039B0546062B02D04E4B23606E
:106AD000EDE71A22002130460DF0C0F800940022A4
:106AE0003C2331462868FFF743FF2268002ADED1A5
:106AF00000943C2306F108016868FFF739FF22681B
:106B0000002AD4D10094182306F11001A868FFF7D9
:106B10002FFF2368002BCAD16869FFF707FC072203
:106B20003A496869FFF764FB80460DF081FF012850
:106B300006F1130706D198F800303F2B04BF2A2333
:106B400088F8003000220823394640460094FFF7B9
:106B50000FFF404600F02EFA2268002AA7D1072135
:106B60003846FFF777FD30B111463846FFF748FD4C
:106B70000721FFF75AFDEF6806F1140838460DF0BB
:106B800057FF012804D13B783F2B04BF2A233B70D9
:106B900020230022414638460094FFF7E9FE0021F9
:106BA0004046FFF742FD2368002B80D12F6938460D
:106BB000FFF7BCFB00287FF47AAF38460D2214495A
:106BC000FFF716FB074600283FF471AF1836009414
:106BD0000D2301223146FFF7CBFE384600F0EAF9DB
:106BE000012421463046FFF735FD30B1611E3046A5
:106BF000FFF706FD2146FFF718FD01340D2CF0D1FB
:106C000055E700BF648001087C800108380000203F
:106C100054000020F0B58DB0CDE90023054628B919
:106C20004FF0FF304FF0FF310DB0F0BD24220021B6
:106C300003A80DF013F803A968460CF01DFF0446E5
:106C40000028EDD00DF0ECF84A1C08BFB0F1FF3F72
:106C500006460F46E4D0626921462846FFF78FFDBD
:106C60000028DDD120460DF0DBF84B1C08BFB0F149
:106C7000FF3FD5D08F4208BF864203D020460DF09B
:106C8000CFF8D1E723682046013323600DF0C8F820
:106C9000013108BFB0F1FF3FC2D0626921462846EA
:106CA000FFF76DFD0028E9D0BAE770B53C258AB042
:106CB000DDE90E64019496FBF5F405FB146402947F
:106CC000182493FBF4F505FB1433CDE903300C20B5
:106CD000013991FBF0F300FB131305930023CDE979
:106CE00007339DF84030A2F26C7201A80692099316
:106CF0000DF096F80AB070BDF7B504466846CDE9C8
:106D000000230CF0A7FE0269037A551C426990F833
:106D100004C0077B02F26C71067EC2690068A37032
:106D20000033207018BF01232046013284F801C0CF
:106D3000E7702571A4F80510E6712272637203B042
:106D4000F0BD1FB5437A0293037801934378009313
:106D50008378B0F805200179C078FFF7A6FF05B069
:106D60005DF804FB904271EB0303B4BF01200020E7
:106D700070470000032210B5104986B00B7801332C
:106D8000B3FBF2F202EB42029B1A0D4A0B7052F86F
:106D9000234003780B4A049343781A2103938378A2
:106DA0000293C378019303790093B0F8053020462D
:106DB0000DF0D8FD204606B010BD00BF86070020AC
:106DC000688201082E820108B1F1004F08BF002837
:106DD0001FB502460B4608D001A8FFF78DFF01A89A
:106DE000FFF7C8FF05B05DF804FB0148FAE700BFF4
:106DF000608201082DE9FF4703220D462B49002838
:106E00000B78044603F10103B3FBF2F202EB4202FA
:106E1000A3EB0203264A0B7052F8236075F10003BE
:106E20003EDA4FF0010A444265EB4505214A002352
:106E3000204629460CF010FC1E4A07460023204637
:106E400029460CF009FC104619464FF461620023F4
:106E50000CF002FC4FF46162804600232046294674
:106E60000CF0FAFB104619463C2200230CF0F4FB10
:106E70003C2281460023204629460CF0EDFBCDF84C
:106E80000080CDE901923B46BAF1000F0BD00A4ACF
:106E90001A2130460DF066FD304604B0BDE8F0879B
:106EA0004FF0000AC2E7054AF2E700BF860700205C
:106EB00068820108805101004C8201084D8201085E
:106EC0000FB404B0704700000FB437B51B4C2568F1
:106ED00055B903222946012002F00AFC2B462A4616
:106EE0002946206002F028FC154D2A68013A033239
:106EF0001ED86421206802F00BFE80220021114878
:106F00000CF0ACFE07AB069A80210E4801930EF000
:106F100011F97F2803DD0C490C480DF081FD2B6829
:106F200008489847002320681A46194602F004FCD6
:106F300003B0BDE8304004B0704700BF1008002027
:106F40008807002090070020E2B701080B08002006
:106F50000FB410B50D4CA2B02268013A033210D81C
:106F600025AB249A802102A801930EF0E3F87F2834
:106F700004DD07490DF183000DF052FD236802A8DE
:106F8000984722B0BDE8104004B070478C0700203D
:106F9000E2B7010870B50446054E4518AC4200D171
:106FA00070BD14F8011B3046FFF78EFFF6E700BFF7
:106FB000D79B010810B5044670B102F0F9F92046DC
:106FC00002F094FA02F0CEF8BDE81040034A93882C
:106FD0000133938002F0E6B810BD00BFE64D0020FB
:106FE00070B5214C8AB0226806460132632A2260BD
:106FF0001E4D0BDD03F0B0FD0523002201A903F0B7
:107000005DFD03F065FA00232860236003F060FA59
:107010002B6803F57A73984204D903F059FA0023D8
:1070200028602360124A134C13781BB923606360F5
:107030000123137002F0BCF9304602F0CBF905468B
:1070400068B1324600210CF009FE02F08BF823886B
:107050000133238002F0A6F828460AB070BD638889
:1070600001336380F8E700BF180800201C080020E7
:1070700014080020E64D002038B505460C460DF0FA
:107080002DFC611B013190FBF1F303FB110028443F
:1070900038BD0078013070470FB404B0704700006D
:1070A0002DE9FF470F460021254D03AE804692464D
:1070B000286832469946039102F06CFE0128039B32
:1070C00031D13BB14FF080521E4B1A60BFF34F8F4E
:1070D000BFF36F8FB7F5C87F88BF4FF4C8774146BD
:1070E0003A4619480CF092FD184C174B3146286867
:1070F000A7802360A4F806A084F8089002F02CFC76
:10710000039B3BB14FF080520E4B1A60BFF34F8F81
:10711000BFF36F8F0E480096002301220421006800
:1071200003F0DCFE039B3BB14FF08052054B1A602D
:10713000BFF34F8FBFF36F8F04B0BDE8F08700BF80
:10714000200A002004ED00E08408002078080020D8
:10715000280A00200348002301220221006803F0CE
:1071600053BE00BF280A00201FB500230B4A402150
:10717000107003AA0A48009200680122039303F0EA
:10718000ADFE039B3BB14FF08052064B1A60BFF33C
:107190004F8FBFF36F8F05B05DF804FB6C080020C4
:1071A000280A002004ED00E01FB5002303AA0A48C6
:1071B0000092802101220068039303F08FFE039B5D
:1071C0003BB14FF08052054B1A60BFF34F8FBFF3B6
:1071D0006F8F05B05DF804FB280A002004ED00E085
:1071E0001FB50F4B1C680346A0B1002303AA0092F1
:1071F000082101222046039303F070FE039B3BB15C
:107200004FF08052074B1A60BFF34F8FBFF36F8F61
:1072100004B010BD01220821204603F0F5FDF7E778
:10722000280A002004ED00E01FB503AA0092012205
:107230000023094811460068039303F04FFE039BA7
:107240003BB14FF08052054B1A60BFF34F8FBFF335
:107250006F8F05B05DF804FB280A002004ED00E004
:107260001FB5002303AA0A480092102101220068DA
:10727000039303F033FE039B3BB14FF08052054B69
:107280001A60BFF34F8FBFF36F8F05B05DF804FB3B
:10729000280A002004ED00E0004870476408002040
:1072A000114810B5002303224FF48071006803F0E9
:1072B000ABFD4FF080520D4B1A60BFF34F8FBFF301
:1072C0006F8F0B4C206802F0B1FD40B1BDE810405B
:1072D000002308481A461946006802F02DBA01201A
:1072E00003F048FAEEE700BF280A002004ED00E0B2
:1072F000240A00201C0A0020F8B5104B014618682B
:1073000002F006FC0446B8B14FF080560C4F0D4D0C
:10731000002303224FF40071386803F075FD2E60DE
:10732000BFF34F8FBFF36F8F386803F047F82E60BD
:10733000BFF34F8FBFF36F8F2046F8BD1C0A0020AC
:10734000280A002004ED00E0014B1860704700BFE0
:10735000140A002070B5044678B10378032B0CD1D1
:10736000436853B10025054E1868F269904760687C
:10737000F369056098476560257070BD400800207E
:1073800010B50D480D4C002305222146006802F07F
:10739000D3F9012805D10A4B1B6863B1BDE8104041
:1073A0001847084B217808485B6998472046BDE894
:1073B0001040FFF7CFBF10BD180A00207008002052
:1073C000140A0020400800209082010873B50024B0
:1073D000094E00226946306802F008FB651C30B98E
:1073E000064BE1B25B690648984702B070BD68463B
:1073F000FFF7B0FF2C46ECE7180A002040080020F9
:10740000B7820108014B1868704700BF180A0020B6
:1074100010B50446064B010AA3F84A00202000F0EC
:1074200057FCE1B22120BDE8104000F051BC00BF84
:10743000F04D002008B5FFF7EBFF0122014B83F868
:10744000522008BDF04D0020002238B50B4B0546F8
:107450001D2083F84E100C4683F84C2000F090FC61
:1074600020F0060040EA4401C9B21D2000F030FCC3
:107470002946BDE83840232000F02ABCF04D00200A
:107480002DE9F74F5E4C1546226C8246022A0F46C4
:107490001E4600F2A3805B4B03EBC203D3E90089D5
:1074A0000120636C98400BF039FA02460B464046C7
:1074B00049460BF0D7FB02460B46002052490BF021
:1074C000D1FB804689463FB149A3D3E900230BF0A5
:1074D0009FFA0BF037FD3860B4F84A000BF02EFA33
:1074E00000224A4B0BF0DEF842464B460BF090FA76
:1074F000CDE900013EB13EA3D3E900230BF088FAA9
:107500000BF020FD3060636C94F84C104FEA830B55
:1075100094F84E000029CBF11C0202EB001214BFBC
:107520001420002002EBCA0AAAEB00000BF0F6F9C7
:1075300094F848200646002A14BF02200020ABEB36
:1075400000000F460BF0EAF902460B46304639467A
:107550000BF088FB0AF050FF06460F4694F84900EE
:1075600004300BF0EBF932463B460BF051FA0022A7
:10757000002306460F460BF0DBFCA0B30022244B91
:10758000304639460BF08EF84B4642460BF040FA37
:107590000C9B06460F4643B115A3D3E900230BF01D
:1075A00037FA0BF0CFFC0C9B1860A5B1DDE90001A8
:1075B00032463B460BF076F80DA3D3E900230BF0DF
:1075C00027FA0DA3D3E900230BF06CF80AF098FF1B
:1075D0000BF0B8FC286003B0BDE8F08F4FF0000856
:1075E0004FF000095CE700200949CDE7AFF30080C8
:1075F0000000000080842E412B8716D9CEF7EF3F84
:10760000F04D0020788201080000F03F000011409A
:107610000000204013B5164C0120A36898470023B2
:1076200041F6FE720093009B934218DDA36802208E
:107630009847002341F6FE720193019B934212DDAD
:107640000C4BB5211C6C4020A047A0214120A04735
:1076500000210120234602B0BDE810401847009BDE
:1076600001330093DFE7019B01330193E5E700BF9E
:1076700040080020EC850108094B07B51B6CC221AE
:107680003B209847002341F6FE720193019B9342F1
:1076900002DD03B05DF804FB019B01330193F5E7C4
:1076A000EC8501088E488F4B2DE9F04F03608E4B1F
:1076B0008E4F83608E4B8F4C43608F4B85B0C36081
:1076C0008E4B8F4D03618F4BDFF86CA283618E4B25
:1076D000DFF86892C3613B68984763698B489847B5
:1076E000002328681A46194602F026F8DFF850B23F
:1076F0009AF8040068B94FF0FF33194603AA03F063
:107700003FFB68B9666903F017FA01468048B04745
:10771000EEE741F2883303AA4FF0FF310020EEE795
:10772000039BDA0516D500F093FA002000F034FE32
:10773000FB6A9847FFF74AFE63697648984700233B
:10774000D9F800001A46194601F0F6FF002003F0B0
:1077500089F8CDE79B0510D500F07AFAFFF78CFF8A
:10776000FB6A9847FFF732FE63696B4898476421CC
:10777000D9F8000002F0CCF9BAE7D9F8000002F01D
:1077800055FB012803D1636964489847B0E7DBF8EB
:10779000003023B940F23B116148FCF7D1F8039B5C
:1077A0001E0604D507225F4B1A70FFF7E9FD039B05
:1077B000580752D50021286802F0AAF901284CD1B7
:1077C000A3690C209847064688B963690C2156487E
:1077D0009847334632463146286801F0ADFF00280D
:1077E00086D14FF4A7714E48FCF7AAF880E7DFF87E
:1077F0005481A369B8F8040098470346A0B9B8F8C3
:1078000004100190626949489047E2693046904708
:10781000019B28681A46194601F08EFF00287FF464
:1078200067AF4FF4AB71DEE708F1040203CA3360BF
:107830007060B1601846D8F80010B8F804200CF059
:10784000E5F90322374B1A705E60FFF799FD0023BC
:1078500028681A46194601F06FFF039BD90706D521
:107860000122304B1A7000225A60FFF789FD039BFA
:10787000DB0606D505222B4B1A7000225A60FFF753
:107880007FFD039B1E0706D50422264B1A7000229B
:107890005A60FFF775FD039B980706D50222214B1E
:1078A0001A7000225A60FFF76BFD039B990606D5FC
:1078B00006221C4B1A701E4A5A60FFF761FD039B9B
:1078C0005B067FF515AF1B4B1B78002B14BF0822FE
:1078D0000922144B1A7000225A60FFF751FD07E786
:1078E0002008002029720008A1700008EC8501081A
:1078F0005571000840080020E1710008617200081D
:10790000200A002069710008A9710008B1840108EB
:10791000C7840108E58401080D8501082485010854
:107920003A850108700800207E850108B4850108A9
:107930006D0800206C08002064080020240A002044
:10794000180A002078080020044B10B55B6998479E
:107950000446FFF75FFE204610BD00BFEC8501081E
:10796000F0B56B4C064625460F460FCE0FC596E880
:107970000F0085E80F0097E803006369654E013B3F
:10798000033388BF644B85B088BF6361636886E852
:107990000300013B033307D960486369984740F20D
:1079A00087215F48FBF7CCFF2368013B033307D9EE
:1079B0005C486369984740F28B215948FBF7C0FF48
:1079C000A368013B033307D957486369984740F2DE
:1079D0008F215348FBF7B4FFE368013B033307D91A
:1079E00052486369984740F293214D48FBF7A8FF3E
:1079F0002369013B033307D94D486369984740F237
:107A000097214748FBF79CFFE369013B033304D907
:107A100040F29B214248FBF793FFA369013B0333EC
:107A200004D940F29F213E48FBF78AFF414B0FCB20
:107A30008DE80F0094E80F0000F0E0F82368984705
:107A4000FFF7E8FD3C4B42205B6C9847222801463B
:107A5000636931D13948984703220021012001F0A0
:107A600047FE374B1860012001F00AFF354B1860C4
:107A700020B940F2BA212A48FBF762FF012001F049
:107A8000FFFE314D286020B940F2BE212448FBF7AB
:107A900057FF4FF0FF31286802F03AF80022082122
:107AA000032001F025FE294B186078B96369284846
:107AB00098474FF4317103E02648984740F2B121CE
:107AC0001748FBF73DFF002005B0F0BD224B234ACD
:107AD0001A6033680BB904233360214B1D680DB164
:107AE0000120F1E701933368FA2200931D49012335
:107AF0001D4802F0CBFA0128F2D063691B48984771
:107B0000074840F2D621FBF71BFF2846DCE700BF01
:107B1000400800206408002099700008E8820108ED
:107B20003A850108298301086083010898830108C8
:107B3000D183010850080020EC8501080D8401085C
:107B4000200A00201C0A0020240A0020180A002015
:107B50003F84010824840108600800209370000815
:107B6000280A002073840108A57600087B84010898
:107B700070B5084C054622680E4622B940F2E6214F
:107B80000548FBF7DDFE236831462846BDE8704016
:107B9000184700BF600800203A85010800F048B887
:107BA000034B0344034883428CBF002001207047ED
:107BB0000071BDCCFF6789090120704708B5FFF748
:107BC0006BFB4379002B0CBF8020002008BD000018
:107BD000094B0022194610B51C68844202D89C68E3
:107BE000844205D80132152A03F10803F4D1FEE7D7
:107BF00001EBC202107910BD5886010884B030B57F
:107C000003AC84E80F00064C03AD0FCD0FC495E81C
:107C10000F0084E80F00BDE8304004B0704700BF9B
:107C2000CC0B0020014B1878704700BFF04D0020AE
:107C3000642307B50093002304481A460321006813
:107C400003F078FA03B05DF804FB00BF340A0020AB
:107C500013B5104C0120A368984700230093009BA4
:107C6000B3F5CC7F0FDDA36800209847002342F6D0
:107C7000FE720193019B934208DD0220A36802B0CB
:107C8000BDE810401847009B0133E7E7019B013333
:107C90000193EFE7CC0B00202DE9F04107460B4C98
:107CA0000020E3680D4616469847236947F0800098
:107CB00098472E44B54204D1E3680120BDE8F04165
:107CC0001847236915F8010B9847F3E7CC0B002000
:107CD00007B501228DF807100DF10701FFF7DCFF52
:107CE00003B05DF804FB0000134A10B55060134A5E
:107CF000904219D00AF012FE0DA3D3E900230AF036
:107D0000B1FF0BF01FF90446C4F307410620FFF74B
:107D1000DFFFC4F307210720FFF7DAFFE1B20820F5
:107D2000BDE81040FFF7D4BF054CEDE7AFF300808E
:107D30000000000080844E40F04D0020F01FCB3347
:107D4000CD3CD9002DE9F04107460C4C0020E368FA
:107D50000D4616469847236907F07F0098472E4442
:107D6000B54204D1E3680120BDE8F041184723691A
:107D70000020984705F8010BF2E700BFCC0B00206C
:107D800007B501220DF10701FFF7DCFF9DF80700A1
:107D900003B05DF804FB000001282DE9F84F884688
:107DA00004D0022852D00020BDE8F88F6A4C27206A
:107DB000A58BFFF7E5FF013520F0F80028440AF015
:107DC000ADFDA37F0022002B3BD1644B0AF06AFC7F
:107DD000064630200F46FFF7D3FF30F0F9030CBF03
:107DE00000235E4B0022304639460AF05BFC064613
:107DF00040460F460AF0A2FD02460B463046394681
:107E00000AF050FC94F820300022E3B900230AF075
:107E100049FC0022524B0AF0FBFD0646A0690F46C2
:107E20000AF07CFD02460B46304639460AF01AFF3E
:107E300000224C4B0AF0ECFD0AF0E6FB0BF082F856
:107E4000B2E70023C2E74FF08043E0E7424C226CE8
:107E5000022A76D8444B03EBC203D3E90067012022
:107E6000656CA8400AF06AFD02460B46304639466A
:107E70000AF0F8FE02460B46002038490AF0F2FEEE
:107E800006460F46B4F84A000AF058FD0022374B68
:107E90000AF008FC32463B460AF0BAFD94F84C3032
:107EA000AD00824694F84E00002B8B46C5F11C01B4
:107EB00001EB001114BF1420002001EBC801081AC7
:107EC0000AF02CFD94F848308046002B14BF0220A5
:107ED0000020281A89460AF021FD02460B4640463A
:107EE00049460AF0BFFE0AF087FA8046894694F8B0
:107EF000490004300AF022FD42464B460AF088FD54
:107F00000022002304460D460BF012F8E0B10022D7
:107F1000134B204629460AF0C5FB32463B460AF081
:107F200077FD52465B460AF0BDFB00220D4B0AF07E
:107F30006FFD07A3D3E900230AF0B4FB0AF0E0FACF
:107F40007CE7002600278AE700200549E5E700BF17
:107F50002B8716D9CEF7EF3FF04D00200000F03F01
:107F60000000204000408F40408601080000114082
:107F7000012808B504D002280AD04FF0FF3008BD10
:107F80001120FFF7FDFEC0F34700404200B2F6E7C4
:107F90001B20FFF7F5FE8B38F8E700000B4B10B500
:107FA0005B68044660B9022098470120FFF7E8FEAD
:107FB00000F0F80121430120BDE81040FFF788BE22
:107FC00003280CBF01200020EEE700BFCC0B0020EF
:107FD00013B5642400230F4800941A460321006857
:107FE00003F0A8F800230C4800941A460321006807
:107FF00003F0A0F80023094800941A460321006802
:1080000003F098F80020FFF7C9FF0022044B1A7014
:1080100002B010BD340A0020C80B0020300A002036
:10802000F04D002013B5642400230F4800941A4635
:108030000321006803F07EF800230C4800941A46E0
:108040000321006803F076F80023094800941A46DB
:108050000321006803F06EF80120FFF79FFF002264
:10806000044B1A7002B010BD340A0020C80B002067
:10807000300A0020F04D002007B50022144B8DF887
:1080800007201A87DA869A8583F82E2093F8223003
:1080900023B903B05DF804EBFFF79ABF3F20FFF769
:1080A0006FFE8DF807009DF80730DB0603D5102121
:1080B0003F20FFF70DFE0D20FFF762FE40F040016C
:1080C0000D20C9B203B05DF804EBFFF701BE00BF9D
:1080D000F04D0020044B1A8840F201139A4201D15E
:1080E000FFF7CABF704700BFF04D0020F7B5614CE5
:1080F00006466378012B3CD0022B6CD00027002170
:108100004FF4C8725C480BF0A9FD012323705B4B50
:108110004FF0FF311868002E00F09E804FF47A7502
:1081200005FB06F200910023B2FBF5F2042103F0F7
:1081300001F86478012C40F094800520FFF72EFFB1
:108140000D20FFF71DFE40F02001C9B20D20FFF702
:10815000BFFD67B14A4B1D6802F0BAF94FF0FF331B
:108160000246009321460023284602F0E3FF03B0B5
:10817000F0BD402094F82270FFF702FE0C21402051
:10818000FFF7A6FD4120FFF7FBFD60F00E01C9B22D
:108190004120FFF79DFD3520FFF7F2FD00F0C00103
:1081A00041F01F013520FFF793FD3520FFF7E8FD73
:1081B00000F03F0084F83A000D20FFF7E1FD00F0E9
:1081C000400141F0B9010D20FFF782FD0023A38596
:1081D0002387E38693E794F8513033202BB3FFF7DE
:1081E000CFFD40F04101C9B23320FFF771FD1921E5
:1081F0003B20FFF76DFD94F84F3094F85270FBB1BF
:108200001D211120FFF764FD4020FFF7B9FD00F0AC
:1082100033014020FFF75CFD00210F20FFF758FDE0
:1082200000210D20FFF754FD69E7FFF7A9FD00F0DD
:10823000BE0141F001013320FFF74AFD1D21D7E7C0
:108240000F211120FFF744FD4020FFF799FD00F0BA
:108250003C0141F00101DCE7009133463246032145
:1082600065E72FB1052003B0BDE8F040FFF796BEEB
:108270000620F8E7F04D0020380A0020340A0020DC
:10828000300A002037B54FF47A72642350432C4DE6
:108290002C4C0093B0FBF2F200230421286802F07A
:1082A00049FF6378012B14D0022B2CD002232370BA
:1082B0002C6802F00DF905230246009301210023EA
:1082C000204602F037FF032003B0BDE83040FFF73F
:1082D00065BE4020FFF754FD00F0030141F010019E
:1082E0004020FFF7F5FC4120FFF74AFD00F03E017A
:1082F0004120FFF7EDFC3520FFF742FD00F03F0085
:1083000084F83A00D2E794F84F3073B1F521112088
:10831000FFF7DEFC4020FFF733FD00F0330141F0B2
:1083200040014020FFF7D4FCC0E7F7211120FFF700
:10833000CFFC4020FFF724FD00F03F01EFE700BF36
:10834000C80B0020F04D002010B5114C6378012BB4
:1083500004D0022B09D040F2E53101E040F2CE31E9
:10836000BDE810400B48FBF7EBBAFA211120FFF7EC
:10837000AFFC4020FFF704FD00F0FC014020FFF7B8
:10838000A7FC032307202370BDE81040FFF706BEBB
:10839000F04D00201187010808B51A4B5A78824227
:1083A0002ED0022858704FF0000013D0FFF7F6FDD2
:1083B0000120FFF7E5FC00F07F010120FFF788FCBA
:1083C00000214020FFF784FC30214120BDE8084017
:1083D000FFF77EBCFFF7E2FD0120FFF7D1FC60F064
:1083E0007F01C9B20120FFF773FC00214020FFF795
:1083F0006FFC00214120FFF76BFC43213120E5E7B2
:1084000008BD00BFF04D0020244B13B518600023B9
:10841000234C1A4600944FF47A71224802F068FE09
:10842000214B186018B9FF212048FBF789FA002377
:1084300000941A464FF47A711D4802F059FE1D4B04
:10844000186020B940F201111848FBF779FA1A4B6D
:10845000012200934FF4FA610023184802F048FE0D
:10846000174B186020B940F203111048FBF768FA67
:10847000FFF7EEFB0020FFF78FFF0020FFF78EFDD8
:108480004FF4C87200210F480BF0E8FB4FF48072E4
:108490000D4B1A8500221A7002B010BD2C0A002064
:1084A000858A000808870108C80B00201187010889
:1084B0000B870108340A0020D58000080E870108C8
:1084C000300A0020380A0020F04D002073B50E4617
:1084D00014460546FFF760FF3046FFF705FC052010
:1084E000FFF75CFD00230193019BB3F5CC7F0BDD0F
:1084F0002846FFF73DFD0546FFF76AFDA542CCBFC4
:108500000020012002B070BD019B0133EBE773B581
:1085100000240220FFF740FFFF211120FFF7D8FBC6
:108520000520FFF73BFD254626460196019BB3F546
:10853000CC7F0DDD2C20FFF723FC00F00100A040D4
:108540000134202C45EA0005EFD1284602B070BD69
:10855000019B01330193E9E72DE9F04F824687B093
:108560000093109B9DF858C001939DF85C30934692
:1085700002939DF860209DF86430049203930C46AA
:10858000BDF84450BDF848909DF84C609DF850707F
:108590009DF85480CDF814C0FFF7FEFEDDE90332EC
:1085A000BAF1010F07D0BAF1020FDDF814C06CD098
:1085B00007B0BDE8F08FDFF824920199C9F818B030
:1085C00089F8212089F822305846C9F81040C9F8A6
:1085D000141089F81E6089F81F7089F82080A9F8A6
:1085E0001C500AF09BF90B46024679A1D1E9000123
:1085F0000AF038FB0AF0A6FC1FFA80FB4FEA1B21A9
:108600000220FFF765FB5FFA8BF10320FFF760FBA9
:108610002046FFF7DDFA01461220FFF759FB0198CB
:10862000FFF7D6FA01461320FFF752FB290A25204F
:10863000FFF74EFBE9B22620FFF74AFBB9F81E30E0
:10864000012B1FD0002340F29711634889F829308D
:10865000FBF776F939463220FFF73AFB3020FFF777
:108660008FFB002E14BF0021802100F06F0040EA34
:108670000818302041EA0801C9B207B0BDE8F04F40
:10868000FFF726BB89F82930E4E754480099BBF18D
:108690000C0F80F849100299C0E9104BA0F84A501D
:1086A00080F84C6080F84D7080F84E8080F84FC0A4
:1086B00080F8501080F8512080F85230824675D8EA
:1086C000BBF1050F7DD9002C74D1ABF10B03012B4D
:1086D0008CBF002301231D208AF84830FFF750FB90
:1086E000009B9AF848101D2041EAC30141EA480165
:1086F00041EA860141EA8411C9B2FFF7E9FA1E2076
:10870000FFF73EFBC9F3012100F00C00014341EAF1
:108710000B11C9B21E20FFF7DBFA5FFA89F11F20A7
:10872000FFF7D6FA290A2020FFF7D2FAE9B2212072
:10873000FFF7CEFA1EB139462220FFF7C9FA9AF8A0
:108740004F306BB14B20FFF71BFB60F07F01C9B2CC
:108750004B20FFF7BDFA9AF850102420FFF7B8FA23
:10876000BBF1060F4FF0310015D1FFF709FB00F008
:10877000F80141F005013120FFF7AAFA0C2137205A
:108780007BE70023A7E701234FF00C0BA3E7234669
:108790004FF0060B9FE7FFF7F3FA00F0F80141F006
:1087A00003013120FFF794FA0A21E8E7002CEAD010
:1087B0004FF00C0B012CE4D1ABF10C0253425341AE
:1087C00089E7002CE3D04FF0060BF3E7AFF300800E
:1087D0000000000080847E4111870108F04D0020D8
:1087E0002DE9F04F89B09A469DF84C3001920293E2
:1087F0009DF85C300D4603939DF860300090069321
:108800009DF86430129E04931A9BBDF85070059336
:108810009DF854809DF85890FFF7BEFD0920FFF7A2
:10882000AFFA04465A20FFF7ABFA04F07F03944CEA
:10883000834660680793FFF7C1F9079B1843C0B2EE
:10884000020600F0F00C25D5112D1ADD142DA8BF5D
:1088500014254BF007025FFA82FB691F4CEA010CFA
:108860005FFA8CF10920FFF733FA59465A20FFF7D7
:108870002FFA009B012B14D0022B66D009B0BDE863
:10888000F08F022DB8BF02250BF0F80242F0040B66
:10889000A91EE3E70E2DA8BF0E2545EAE575691C64
:1088A000DCE7019B84F82090C4E9033A049B25721D
:1088B00084F82130059BA6616362A78384F81E803B
:1088C00001980AF02BF86AA3D3E900230AF0CAF949
:1088D0000AF038FB84B2210A0420FFF7F9F9E1B26B
:1088E0000520FFF7F5F930460AF018F802460B4666
:1088F00061A1D1E900010AF0B5F90AF023FB84B2C5
:10890000210A0220FFF7E4F9E1B20320FFF7E0F9C2
:10891000390A2520FFF7DCF9F9B22620FFF7D8F94C
:108920003020FFF72DFAB8F1000F14BF002180218D
:1089300000F06F0040EA0919302041EA0901C9B28C
:1089400009B0BDE8F04FFFF7C3B9029B0C2E84F8C5
:108950004930039B84F83C5084F84F30069BC4E9AF
:1089600010A684F85030049BA4F84A7084F8513063
:10897000059B84F84C8084F84E90636566D8052E7C
:1089800070D9BAF1000F65D1A6F10B02012A8CBF94
:10899000002201223A4D039B85F848206BB14B2001
:1089A000FFF7EEF960F07F01C9B24B20FFF790F9B5
:1089B00095F850102420FFF78BF91D20FFF7E0F900
:1089C000029B94F848101D2041EAC30141EA49097D
:1089D00049EA880848EA8A185FFA88F1FFF778F9C7
:1089E0001E20FFF7CDF900F00F0141EA0611C9B2D0
:1089F0001E20FFF76DF9390A2020FFF769F92120C1
:108A0000F9B2FFF765F9062E4FF0310013D1FFF7E9
:108A1000B7F900F0F80141F005013120FFF758F9EE
:108A20000C2137208CE70022B4E701220C26B1E7A5
:108A300052460626AEE7FFF7A3F900F0F80141F031
:108A400003013120FFF744F90A21EAE7BAF1000FE8
:108A5000EBD00C26BAF1010FE5D1A6F10C035A4276
:108A60005A4197E7BAF1000FE2D00626F2E700BFBD
:108A70000000000080844E400000000080847E41A1
:108A8000F04D002010B5214C2378012B02D0022B91
:108A90002FD010BD6378012B24D100230B213E2061
:108AA000A3852387E386FFF713F910213F20FFF703
:108AB0000FF994F822309BB10D20FFF761F940F0D7
:108AC0002001C9B20D20FFF703F9114B1B68002BE1
:108AD000DFD0DB68002BDCD0BDE810400020184759
:108AE0002370F2E794F85230002BEED0FFF79AFA99
:108AF000EBE700232370064B1B68002BC9D05B6893
:108B0000002BC6D0BDE81040184700BFF04D002034
:108B10002C0A00202DE9F04107460C4C0020E368A8
:108B20000D4616469847236907F07F0098472E4464
:108B3000B54204D1E3680120BDE8F041184723693C
:108B400000209847C04305F8010BF1E7CC0B00204B
:108B50000A4601460020FFF79FB80000F7B5374CE2
:108B6000064663780D46012B07D0022B27D0002044
:108B700003B0BDE8F040FFF785BB00232387A37F48
:108B8000E18613B13220FFF7A3F86B1E3F2B0DD8FF
:108B900084F83B50304694F83B10FFF7D9FF228F02
:108BA00094F83B30606A13442387E1E72A46314654
:108BB00023480BF02BF8202384F83B30EAE794F8A5
:108BC0005130332023B3FFF7DBF800F0BE01332030
:108BD000FFF77EF819213B20FFF77AF8294622207B
:108BE00084F85C50FFF774F800210E20FFF770F84E
:108BF00000210D20FFF76CF80120FFF7C1F830F0DD
:108C0000F80710D030462946FFF7A2FF606DAFE7A6
:108C1000FFF7B6F800F0BE0141F001013320FFF785
:108C200057F81D21D7E7FFF7FDF90197019BB3F531
:108C3000CC7FE7DC019B01330193F7E7F04D002087
:108C4000380A00200A4601460020FFF77BB80A4692
:108C500001460020FFF75EBF38B505460C46FFF71A
:108C60009BFB012D02D0022D0AD038BD064B9B7F05
:108C7000002BFAD121463220BDE83840FFF728B852
:108C800021462320F8E700BFF04D00207FB50022E9
:108C90005E4C8DF80B2023780392012B254604D0DF
:108CA000022B00F0918004B070BD6378012B32D0AC
:108CB000022BF8D140211220FFF70AF81220FFF70B
:108CC0005FF88DF80B009DF80B30514E13F0200F1C
:108CD00027D020211220FEF7FBFF94F8523003B971
:108CE000237000224B48009203AB0821006802F079
:108CF00021FA039B3BB14FF08052474B1A60BFF300
:108D00004F8FBFF36F8F3368002BCCD01B69002BC4
:108D1000C9D09847C7E740F2EE414048FAF710FE45
:108D2000C1E71920FFF72CF840B2002884F858005A
:108D3000BFBF40428010404244B2A8BF84101A20F6
:108D4000FFF71EF8002C40F30B13B8BF00198B3847
:108D50009BB203441BB21320A5F85A30FFF710F85A
:108D600085F85C001020FFF70BF801460D20FEF798
:108D7000AFFF95F85C102A48FFF764FF95F8522082
:108D80008AB924482A70009203AB0821006802F0D7
:108D9000D1F9039B3BB14FF080521F4B1A60BFF3D8
:108DA0004F8FBFF36F8F3368002B3FF47CAF9C680D
:108DB000002C3FF478AF95F95830B5F95A2095F862
:108DC0005C101748A0476EE71648009203AB0821D5
:108DD000006802F0AFF9039B3BB14FF080520E4B9D
:108DE0001A60BFF34F8FBFF36F8F6B78022B03D1E5
:108DF00008211220FEF76CFF00232B70044B1B6828
:108E0000002B3FF450AF1B6881E700BFF04D0020FE
:108E10002C0A0020340A002004ED00E0118701082C
:108E2000380A0020C80B0020002230B5544D85B010
:108E30002B780392012B8DF80B202C4604D0022BAB
:108E400000F0848005B030BD6B78012B22D0022B5E
:108E5000F8D14C48009203AB0821006802F06AF98F
:108E6000039B3BB14FF08052474B1A60BFF34F8FCB
:108E7000BFF36F8F80211220FEF72AFF002323709B
:108E8000424B1B68002BDDD0DB68002BDAD00120C1
:108E90009847D7E73F20FEF773FF8DF80B009DF84A
:108EA0000B309B06CED595F8293023B940F28E5170
:108EB0003748FAF745FD238F364894F83A1018449E
:108EC00094F82830022B17D1FFF7C1FE238FB3B1DE
:108ED000228F94F83A30E18E13449BB28B42238761
:108EE000B0D32A4B1B68BBB19D68ADB1002394F988
:108EF0002E202848A8470FE0FFF7A4FEE6E794F8E5
:108F00002D304BB194F83A102248FEF731FEE0863E
:108F10000138B0F5C77FDBD9FFF7AEF81E4B1C68F0
:108F200001F0DCFA002302460093072103AB204640
:108F300002F000F9039B002B84D04FF08052124BBB
:108F40001A60BFF34F8FBFF36F8F7BE76B78012BF6
:108F50007FF478AF2A8FEB8E95F83B100D489B1A63
:108F60008B42104407DDFFF7F3FD95F83B302A8F65
:108F700013442B8766E7D9B2FFF7EAFDEB8EF8E7DB
:108F8000F04D0020340A002004ED00E02C0A0020FF
:108F900011870108380A0020300A002010B5184C4B
:108FA0002378012B02D0022B28D010BD6178012933
:108FB00018D00229F9D194F84F30002BF5D01220A7
:108FC000FEF786FE0F4B1B68002BEED05C69002C71
:108FD000EBD01C20FEF7D4FE2346BDE8104000F085
:108FE0003F00184700231120238784F82D10FEF737
:108FF000C7FE4008404284F82E00D6E76178D8E7E3
:10900000F04D00202C0A00201F4B70B55A78022A20
:1090100004D11B78012B02D0032B13D070BD12207A
:10902000FEF7AEFEC306F9D510211220FEF750FE62
:10903000164B1B68002BF1D0DB69002BEED0BDE88E
:10904000704018471220FEF79BFE10F001050F4CF0
:109050000DD005211220FEF73BFE2368002BDDD04A
:109060009B69002BDAD00120BDE87040184704212D
:109070001220FEF72DFE2368002BCFD09B69002B1A
:10908000CCD02846F0E700BFF04D00202C0A00208D
:10909000074B5A78012A0AD11A78012A07D183F896
:1090A0002C20002202213E201A87FEF711BE7047B5
:1090B000F04D00207047000006480068006880F30B
:1090C000088862B661B6BFF34F8FBFF36F8F00DFC2
:1090D00000BF000008ED00E0002307B501930B4B33
:1090E0001B68013303D0CA210948FAF729FC4FF065
:1090F000500383F31188BFF36F8FBFF34F8F019B32
:10910000002BFCD003B05DF804FB00BF88000020FA
:109110005E8701084FF0807340F8043C054B21F056
:10912000010140F8081C40F80C3C40F8202C403865
:10913000704700BFD9900008000000000000000048
:10914000074B19680868B0E8F00F80F30988BFF38F
:109150006F8F4FF0000080F311884EF00D0E7047B6
:109160000C4800204FF0500383F31188BFF36F8F3A
:10917000BFF34F8F084A13680133012B136009D1E5
:10918000064B1B6813F0FF0F04D040F27511044822
:10919000FAF7D6BB704700BF8800002004ED00E05E
:1091A0005E87010810B5074C236823B94FF4BE71E0
:1091B0000548FAF7C5FB2368013B23600BB983F32D
:1091C000118810BD880000205E87010800000000A3
:1091D000EFF30980BFF36F8F0D4B1A6820E9F00F92
:1091E00010602DE908404FF0500080F3118801F025
:1091F000E7FA4FF0000080F31188BDE808401968D5
:109200000868B0E8F00F80F30988BFF36F8F7047EC
:109210000C48002008B54FF0500383F31188BFF3CA
:109220006F8FBFF34F8F01F061F918B14FF080528B
:10923000024B1A60002383F3118808BD04ED00E09F
:109240000022054B05491A600A6041F26701044A91
:10925000116007221A60704710E000E018E000E09B
:1092600014E000E013B5254B254C1A78D2B20192D8
:10927000FF221A701B78234ADBB28DF803309DF869
:10928000033003F0500313700723002223609DF87E
:109290000310581E090628D412B1032B236004D0F2
:1092A0004FF49B711848FAF74BFB2368134A1B02D3
:1092B00003F4E06323600024019BDBB21370134BC3
:1092C0001A6842F470021A601A6842F070421A601A
:1092D000FFF7B6FF0E4B1C60FFF7EEFE01F070FAD1
:1092E000FFF7FAFE204602B010BD9DF803300122C0
:1092F0005B00DBB28DF803300346C8E700E400E012
:10930000F00B0020EC0B00205E87010820ED00E050
:109310008800002008B5EFF305830F2B0AD90D4A0A
:109320009B5C0D4A12789A4204D940F2A5210B4861
:10933000FAF706FB0A4B0B4A1B68126803F4E0635A
:10934000934206D9BDE8084040F2B5210348FAF738
:10935000F7BA08BDF0E300E0EC0B00205E870108DF
:109360000CED00E0F00B002010B50F4B1A688242A4
:1093700018D35C681919884201BF41681846091959
:109380005960446801198A4207D1084909688A422C
:109390001FBF51681268091941609842026018BFE6
:1093A000186010BD1346E1E704480020F40B0020CC
:1093B00038B5064B064D1C68246804B938BD6307F0
:1093C000FAD077212846FAF7BBFAF5E704480020DF
:1093D000B68701082DE9F843074601F071F83B49CB
:1093E0003B4D0B68D3B93B4B3B4A58074FF000004D
:1093F0001CBF073323F0070313605060374A22F085
:109400000702C2E90000D01AC3E90020344B0A6009
:109410001860344B18604FF000432B602B681F42DC
:1094200052D1002F41D007F1080462071CBF24F07D
:1094300007040834002C47D02A4B1A689846A242E9
:1094400042D3254B1E687268A24202D230680028BF
:1094500037D10968B14237D01F683168121B102A12
:1094600007F10807196010D906EB040919F0070F76
:1094700003D0D5211C48FAF763FA736848461B1BD2
:10948000C9F804307460FFF76FFF15497268D8F8A7
:10949000003008689B1A8342C8F8003038BF0B6060
:1094A0002B68134373600023336001F0AFF87B0730
:1094B00004D040F215110C48FAF742FA3846BDE8DC
:1094C000F88333460646BEE70027EEE7F40B00209C
:1094D000F8470020F80B002004480020F047002047
:1094E00000480020FC470020B687010838B5044634
:1094F00070B3184D50F8041C2A68114204D140F290
:1095000029111548FAF71CFA54F8083C23B14FF416
:1095100095711148FAF714FA54F8043C2A6813427A
:1095200016D054F8081C99B923EA020344F8043C05
:1095300000F0C6FF094A54F8043C1168A4F1080081
:109540000B441360FFF710FFBDE8384001F05EB830
:1095500038BD00BFF8470020B6870108FC4700204F
:1095600010B50446FFF7FEFDA46BFFF71BFEB4FA2F
:1095700084F0400910BD70B51546026C0446866B38
:1095800042B905689DB9806801F04EFBA5600136BF
:10959000A66370BD6DB940680AF038FB6368226C41
:1095A0001344A2686360934201D323686360002080
:1095B000EDE7C0680AF02AFB236CE2685B42216891
:1095C0001A448A42E2603EBFA2689B18E360022D03
:1095D000EDD10EB1013EEAE73046D8E703461A6CFA
:1095E00010B4084662B1D9689C681144A142D960A0
:1095F00028BF196810BC28BFD960D9680AF006BB1B
:1096000010BC704770B50446FFF7ACFD94F84550A8
:1096100004F124066DB2002D14DCFF2384F84530DC
:10962000FFF7C0FDFFF79EFD94F8445004F11006CB
:109630006DB2002D12DCFF2384F84430BDE8704089
:10964000FFF7B0BD636A002BE7D0304601F0AEF9FA
:1096500008B101F02DFA013D6DB2DCE72369002B62
:10966000E9D0304601F0A2F908B101F021FA013D3C
:109670006DB2DEE738B50D46044620B940F203115D
:109680001948FAF75DF9FFF76DFDD4E90F314B4347
:109690002268D0185B1A1344A060E3600020FF2307
:1096A000A063626084F8443084F8453095B923693A
:1096B00063B104F1100001F079F938B14FF0805234
:1096C0000A4B1A60BFF34F8FBFF36F8FFFF76AFD2E
:1096D000012038BD04F1100001F06CFE04F12400FB
:1096E00001F068FEF2E700BF0C88010804ED00E01D
:1096F000F8B50D461746064620B94FF4BB710D4824
:10970000FAF71EF905FB06F05030FFF763FE04463A
:1097100058B165B100F150032360C4E90F65012120
:109720002046FFF7A7FF84F84C702046F8BD03469B
:10973000F2E700BF0C8801082DE9FF478846019237
:109740001E46044620B940F2F1214B48FAF7F8F8DA
:10975000B8F1000F06D1236C23B140F2F221464844
:10976000FAF7EEF8022E07D1E36B012B04D040F29A
:10977000F3214148FAF7E4F801F0F4F930B9019B1C
:1097800023B140F2F6213C48FAF7DAF80027B9464F
:10979000DFF8E8A0FFF7E6FCA26BE36B9A4201D387
:1097A000022E19D1324641462046FFF7E4FE636A95
:1097B0001BB104F1240001F0F9F838B14FF08052E8
:1097C0002E4B1A60BFF34F8FBFF36F8FFFF7EAFC8A
:1097D000012004B0BDE8F087019D1DB9FFF7E2FC50
:1097E0000020F6E717B902A801F020F9FFF7DAFC2C
:1097F00000F066FEFFF7B6FC94F84430FF2B08BF7C
:1098000084F8449094F84530FF2B08BF84F84590C5
:10981000FFF7C8FC01A902A801F014F928BBFFF763
:10982000A1FCA26BE36B9A420ED1FFF7BBFC01993E
:1098300004F1100001F080F82046FFF7E3FE00F08D
:10984000E5FE48B10127A5E7FFF7ACFC2046FFF78E
:10985000D9FE00F0DBFEF5E74FF08053CAF8003088
:10986000BFF34F8FBFF36F8FECE72046FFF7CAFEC1
:1098700000F0CCFEB4E700BF0C88010804ED00E066
:1098800010B5024600210120FFF732FF044638B12F
:10989000002383600360C3601A461946FFF74CFF3C
:1098A000204610BD2DE9F843894690461F460446E0
:1098B00020B940F2C3312748FAF742F8B9F1000F56
:1098C00006D1236C23B14FF471712248FAF738F8AE
:1098D000022F07D1E36B012B04D040F2C5311D48A4
:1098E000FAF72EF8FFF716FDEFF311864FF050034D
:1098F00083F31188BFF36F8FBFF34F8FA26BE36BBE
:109900009A4201D3022F22D194F845503A466DB2C3
:1099100049462046FFF72FFE6B1C13D1636A0BB933
:1099200001200BE004F1240001F040F80028F7D0FA
:10993000B8F1000FF4D00120C8F8000086F31188B8
:10994000BDE8F88301356DB284F84550E8E70020A2
:10995000F4E700BF0C88010870B50D46044620B935
:109960004FF48C612048F9F7EBFF236C23B140F2F0
:1099700064411D48F9F7E4FF236833B9A36823B1B4
:1099800040F269411848F9F7DBFFFFF7C3FCEFF33A
:1099900011864FF0500383F31188BFF36F8FBFF32D
:1099A0004F8FA26BE36B93421CD994F84530013280
:1099B0005BB2A2635A1C10D1636A0BB9012009E0A3
:1099C00004F1240000F0F2FF0028F7D0002DF5D0BC
:1099D0000120286086F3118870BD01335BB284F8E2
:1099E0004530EBE70020F5E70C8801082DE9F0434E
:1099F00085B00F460192044620B94FF4A061424859
:109A0000F9F79EFF37B9236C23B140F204513E4869
:109A1000F9F796FF01F0A6F830B9019B23B140F2A7
:109A200009513948F9F78CFF0026B046DFF8DC9081
:109A3000FFF798FBA56BD5B139462046013DFFF7EE
:109A4000CDFDA563236963B104F1100000F0AEFF02
:109A500038B14FF080522D4B1A60BFF34F8FBFF3D8
:109A60006F8FFFF79FFB012005B0BDE8F083019DDC
:109A70001DB9FFF797FB0020F6E716B902A800F022
:109A8000D5FFFFF78FFB00F01BFDFFF76BFB94F892
:109A90004430FF2B08BF84F8448094F84530FF2BF6
:109AA00008BF84F84580FFF77DFB01A902A800F0FC
:109AB000C9FFF0B92046FFF753FDA0B1019904F1A9
:109AC000240000F039FF2046FFF79CFD00F09EFDCA
:109AD00038B94FF08053C9F80030BFF34F8FBFF350
:109AE0006F8F0126A4E72046FFF78CFD00F08EFD66
:109AF000F7E72046FFF786FD00F088FD2046FFF7D8
:109B00002FFD0028EDD0B6E70C88010804ED00E039
:109B10002DE9FF410446019120B940F2915152488C
:109B2000F9F70EFF236C23B140F295514E48F9F737
:109B300007FF01F017F830B9019B23B140F29A51A9
:109B40004948F9F7FDFE00252F462E46DFF81C8117
:109B5000FFF708FBA36BE3B1013BA363236813B9D1
:109B600001F002F9A060236963B104F1100000F074
:109B70001DFF38B14FF080523C4B1A60BFF34F8F3E
:109B8000BFF36F8FFFF70EFB0125284604B0BDE839
:109B9000F081019B4BB925B140F2E1513248F9F710
:109BA000CFFEFFF7FFFA0025EFE717B902A800F094
:109BB0003DFFFFF7F7FA00F083FCFFF7D3FA94F8C4
:109BC0004430FF2B08BF84F8446094F84530FF2BE5
:109BD00008BF84F84560FFF7E5FA01A902A800F084
:109BE00031FF40BB2046FFF7BBFCF0B123683BB917
:109BF000FFF7B8FAA06800F0C5FF0546FFF7D2FAF4
:109C0000019904F1240000F097FE2046FFF7FAFCCA
:109C100000F0FCFC38B94FF08053C8F80030BFF3B7
:109C20004F8FBFF36F8F012792E72046FFF7EAFCC3
:109C300000F0ECFCF7E72046FFF7E4FC00F0E6FC60
:109C40002046FFF78DFC0028EDD0002D9DD0FFF7BA
:109C500089FA616A19B1236B1968C1F10501A0681D
:109C600001F02EF89DE700BF0C88010804ED00E02C
:109C70002DE9F04385B00F460192044620B94FF418
:109C8000CD614248F9F75CFE37B9236C23B140F24D
:109C90006C613E48F9F754FE00F064FF30B9019B57
:109CA00023B140F271613948F9F74AFE0026B04607
:109CB000DFF8DC90FFF756FAA36BD3B139462046A4
:109CC000E568FFF78BFC636AE56063B104F124008B
:109CD00000F06CFE38B14FF080522D4B1A60BFF38C
:109CE0004F8FBFF36F8FFFF75DFA012005B0BDE81E
:109CF000F083019D1DB9FFF755FA0020F6E716B96C
:109D000002A800F093FEFFF74DFA00F0D9FBFFF731
:109D100029FA94F84430FF2B08BF84F8448094F863
:109D20004530FF2B08BF84F84580FFF73BFA01A9B7
:109D300002A800F087FEF0B92046FFF711FCA0B1A1
:109D4000019904F1240000F0F7FD2046FFF75AFCCA
:109D500000F05CFC38B94FF08053C9F80030BFF315
:109D60004F8FBFF36F8F0126A4E72046FFF74AFC11
:109D700000F04CFCF7E72046FFF744FC00F046FCFF
:109D80002046FFF7EDFB0028EDD0B6E70C88010870
:109D900004ED00E02DE9F84389469046054620B9D8
:109DA00040F2FB612048F9F7CBFDB9F1000F06D175
:109DB0002B6C23B140F2FC611B48F9F7C1FDFFF7A2
:109DC000A9FAEFF311874FF0500383F31188BFF323
:109DD0006F8FBFF34F8FAC6B1CB395F8446049464F
:109DE00076B22846FFF7FAFB013C731CAC6313D133
:109DF0002B690BB901200BE005F1100000F0D6FD36
:109E00000028F7D0B8F1000FF4D00120C8F8000006
:109E100087F31188BDE8F883013676B285F844608F
:109E2000E8E72046F4E700BF0C88010810B50446B7
:109E300020B940F28A710548F9F782FDFFF792F9DF
:109E4000A46BFFF7AFF9204610BD00BF0C880108D6
:109E500038B5054620B940F2A4710648F9F770FDFF
:109E6000FFF780F9A86BEC6B241AFFF79BF92046EB
:109E700038BD00BF0C880108002330B5064A52F8EF
:109E8000335002EBC3041DB942F83310606030BD9B
:109E90000133052BF3D1FAE7504E0020002310B513
:109EA000084951F83320DC00824206D10021064ADD
:109EB00042F833102244516010BD0133052BF0D11C
:109EC000FAE700BF544E0020504E002010B5044663
:109ED00020B94FF4F8610548F9F732FD2046FFF745
:109EE000DDFFBDE81040FFF701BB00BF0C88010893
:109EF00070B504460D461646FFF734F994F8443021
:109F0000FF2B04BF002384F8443094F84530FF2B26
:109F100004BF002384F84530FFF744F9A36B2BB945
:109F20003246294604F1240000F020FD2046BDE819
:109F30007040FFF767BB0000064A13681968064BBC
:109F400019B94FF0FF321A6070471268D268D268B0
:109F50005268F8E710480020C048002010B50446B9
:109F600020B940F2F2610848F9F7EAFC6269074B50
:109F70009A4207D1A06A064B984203D0B0FA80F00B
:109F8000400910BD0020FCE750880108E04800208F
:109F9000C8480020F8B51B4B1B4E1C6805463068AE
:109FA0000F46043001F037FA334640B901203168DA
:109FB000164EC96A3268884022EA000232606A1C82
:109FC00007D137B1196812480431BDE8F84001F0F3
:109FD000FFB91A686419546007D30E4A10681968EB
:109FE000BDE8F840043101F0FFB90B4A1068196868
:109FF000043101F0F9F9094B1A68A24288BF1C60CC
:10A00000F8BD00BF084900200C48002090480020FF
:10A01000E04800201448002010480020C0480020DC
:10A0200080B5DFF86480144F144C154E236863B973
:10A03000144B1B68012BF8D94FF08053C8F800303F
:10A04000BFF34F8FBFF36F8FEEE7FFF78BF8FB681F
:10A05000DD68281D01F0DFF93368013B33602368B8
:10A06000013B2360FFF79EF8286BFFF73FFA284675
:10A07000FFF73CFADAE700BFF448002080480020F0
:10A080007C4800201848002004ED00E02DE9F84F3E
:10A090004FEA820A804650460D4699460B9EFFF7CE
:10A0A00099F90746002800F0AA805C20FFF792F992
:10A0B0000446002800F0A080076325B94FF45871CA
:10A0C0005648F9F73DFC5246A521206B09F0C6FD24
:10A0D000236BAAF1040A9A442AF0070A6B1E04F1C2
:10A0E00034020F3513F8011F02F8011B09B19D421C
:10A0F000F8D10A9D4FF0000B042D28BF0425271D21
:10A10000E562C4E9135B384684F843B001F05DF9B9
:10A11000C5F1050504F1180001F057F9C4F854B071
:10A120002461A561646284F858B04A4641465046AD
:10A13000FEF7F0FF206006B13460FFF713F8384BEC
:10A14000384E1A68DFF8188101321A603268002A26
:10A1500058D134601B68012B25D1334801F02AF90E
:10A16000324801F027F9324801F024F9DFF8F49081
:10A17000304801F01FF9304D304801F01BF94846D6
:10A1800001F018F9284601F015F92D4801F012F9EF
:10A190002C4801F00FF92C4801F00CF92B4BC3F8B7
:10A1A00000902B4B1D6001252A4A2B491368086833
:10A1B00001331360E26A636405FA02F30343142077
:10A1C0000B60194B394600FB023001F001F9FEF734
:10A1D000E9FFD8F8003063B13368DA6AE36A9A427B
:10A1E00007D24FF080521D4B1A60BFF34F8FBFF361
:10A1F0006F8F2846BDE8F88F3846FFF777F94FF0A4
:10A20000FF35F6E7D8F80030002BCCD13368DA6A96
:10A21000E36A9A4298BF3460C5E700BF50880108DE
:10A220007C4800200C480020184800202C480020C2
:10A230004048002054480020A848002068480020DA
:10A24000C8480020F4480020E048002010480020C2
:10A25000144800208C4800209048002004ED00E0C5
:10A26000DC4800209448002070B50446284DFEF7D5
:10A2700079FF04B92C68261D304601F0CCF860B98E
:10A280001421E06A234B41435B5833B90122224930
:10A2900082400B6823EA02030B60A36A1BB104F13E
:10A2A000180001F0B8F81D4A1368013313602B68D9
:10A2B000A34220D131461A4801F08AF8194A13689E
:10A2C00001331360FEF76EFF174B1B6893B12B68C9
:10A2D000A3420FD1154B1B6823B140F2B64114487D
:10A2E000F9F72EFB4FF08052124B1A60BFF34F8FDD
:10A2F000BFF36F8F70BD104A206B1368013B136072
:10A30000FFF7F4F82046FFF7F1F8FFF715FED9E75D
:10A310000C48002018480020904800208C4800205D
:10A32000F448002080480020DC48002088480020B5
:10A330005088010804ED00E07C480020F8B505468F
:10A3400020B940F24C511748F9F7FAFA164B1B683E
:10A35000AB4220D0FEF706FF144B6C691F68144B0C
:10A360001E68FEF71FFFBC4217D0B44215D0114B38
:10A370009C4208D1AB6A83B995F85830012B0CBFC9
:10A3800002200320F8BD0C4B9C4208D0002C0CBFCF
:10A3900004200120F6E70020F4E70220F2E7042081
:10A3A000F0E700BF508801080C480020104800204A
:10A3B00014480020E0480020F448002070B504460E
:10A3C00020B940F21C711948F9F7BAFA184D2B68F8
:10A3D000A34229D044B3FEF7C5FE2046FFF7BEFDD9
:10A3E000F0B1261D304601F016F801231149E26A4A
:10A3F00008689340034314200B600F4B314600FB69
:10A40000023000F0E5FF2B68E26ADB6A9A4207D36C
:10A410004FF08052094B1A60BFF34F8FBFF36F8F1D
:10A42000BDE87040FEF7BEBE70BD00BF5088010899
:10A430000C480020904800201848002004ED00E05F
:10A4400013B50024174B009401935022234616495C
:10A450001648FFF71BFE012818D100F023FE012843
:10A4600014D14FF0500383F31188BFF36F8FBFF304
:10A470004F8F4FF0FF320E4B1A600E4B18600E4B91
:10A480001C6002B0BDE81040FEF7ECBE013007D101
:10A4900040F60401094802B0BDE81040F9F750BA8F
:10A4A00002B010BDBC4800209488010821A000081B
:10A4B000C0480020DC4800200849002050880108DE
:10A4C000024A136801331360704700BF88480020B8
:10A4D000014B1868704700BF0849002008B5FEF717
:10A4E00019FF014B186808BD084900202DE9F84FF5
:10A4F0003A4B1B68002B6AD1394B1C6801341C6035
:10A500009CB9384D2B681B6823B140F66221364850
:10A51000F9F716FA354B2A68196829601A60344A27
:10A52000136801331360FFF707FD324D4FF0000B46
:10A530002B68314FA34211D93A68304BD16A1422AB
:10A540004A439A58022A28BF4FF0010B2C4A12683E
:10A55000002A0CBF58460120BDE8F88FDFF884A020
:10A56000DFF8A490DAF8002012681AB94FF0FF3231
:10A570002A60E1E7DAF80020D268D66871688C4278
:10A5800001D22960D8E706F10408404600F043FFF5
:10A59000B16A19B106F1180000F03DFF01224FF039
:10A5A000140CF06AD9F8003002FA00F11943134B89
:10A5B000C9F800100CFB0030414600F009FF386874
:10A5C000F16AC26A914228BF4FF0010BCAE70D4AF7
:10A5D0004FF0000B136801331360B7E78848002081
:10A5E0000849002010480020508801081448002025
:10A5F000C4480020C04800200C4800201848002013
:10A600000C49002084480020904800202DE9F843A0
:10A610002E4C236823B940F668012D48F9F790F9CC
:10A62000FEF7A0FD2368013B236024682CB10024C1
:10A63000FEF7B8FD2046BDE8F883264B1B68002BCB
:10A64000F5D0254D254EDFF8A8801FE0EB680127E7
:10A65000DC6804F1040904F1180000F0DCFE48464F
:10A6600000F0D9FE1420E26A316807FA02F30B43C6
:10A6700000FB02804946336000F0AAFE184BE26AF4
:10A680001B68DB6A9A4201D3164B1F602B68002BB4
:10A69000DCD10CB1FFF750FC134D2C6844B10127FD
:10A6A000104EFFF723FF00B13760013CF9D12C6059
:10A6B0000C4B1B68002BBAD04FF080520B4B1A602A
:10A6C000BFF34F8FBFF36F8F0124B1E7884800209D
:10A6D000508801087C480020C8480020904800208D
:10A6E0000C4800200C4900208448002004ED00E0C4
:10A6F0001848002038B50C46054620B940F2CA413A
:10A700001848F9F71DF924B940F2CB411548F9F77B
:10A7100017F9154B1B6823B140F2CC411148F9F7EA
:10A720000FF9FFF7CDFE114B2A68186814192CBFDA
:10A730000121002182422C600CD961B9FFF766FF2C
:10A7400038B94FF080520A4B1A60BFF34F8FBFF3F6
:10A750006F8F38BD09B9A042F0D20021201AFFF74F
:10A7600019FCEBE7508801088848002008490020C0
:10A7700004ED00E010B5044640B94FF080520D4B97
:10A780001A60BFF34F8FBFF36F8F10BD0A4B1B686A
:10A7900023B14FF4A4610948F9F7D2F8FFF790FE0E
:10A7A00000212046FFF7F6FBFFF730FF0028E4D03A
:10A7B000EBE700BF04ED00E0884800205088010866
:10A7C000224B70B51A68224B12B101221A6070BD7B
:10A7D000204E1A6033681B6B1A68B2F1A53F0BD18B
:10A7E0005A68B2F1A53F07D19A68B2F1A53F03D1EB
:10A7F000DB68B3F1A53F04D0306831683431F9F734
:10A800006BF8154B1C68B4FA84F41423E4B2C4F159
:10A810001F046343114DEB5823B940F688311048AB
:10A82000F9F78EF8142202FB04F3E918486808339C
:10A8300040682B44984202FB045408BF43684860B8
:10A8400008BF4B606368DB683360C0E7884800205E
:10A850000C4900200C480020904800201848002097
:10A860005088010870B504462A4EFEF77BFC04B9F7
:10A870003468251D284600F0CEFD60B91421E06A39
:10A88000254B41435B5833B90122244982400B6870
:10A8900023EA02030B60A36A1BB104F1180000F065
:10A8A000BAFD29461E4800F093FD94F858301D4D1E
:10A8B000012B04BF002384F85830FEF773FC2A688C
:10A8C0002AB1FEF74FFCFFF737FBFEF76BFC33684E
:10A8D000A34211D12B6883B1134B1B6823B14FF4F2
:10A8E000D9611248F9F72CF84FF08052104B1A60DA
:10A8F000BFF34F8FBFF36F8F70BD094A11680D4AC8
:10A900001268914201D13360F6E7BDE87040FFF76D
:10A9100057BF00BF0C480020184800209048002076
:10A92000E0480020DC4800208848002050880108CA
:10A9300004ED00E07C48002038B50D46044620B9FF
:10A9400040F69F310748F8F7FBFF074B2046196890
:10A95000183100F049FD2846BDE838400121FFF7D5
:10A9600019BB00BF508801080C48002070B50E4686
:10A970001446054620B940F6CA310A48F8F7E0FF08
:10A98000094B28461968183100F022FD002C214699
:10A9900008BF3046BDE8704018BF4FF0FF30FFF7EA
:10A9A000F9BA00BF508801080C48002038B5C368C8
:10A9B000DC6824B940F6FA311548F8F7C1FF04F114
:10A9C0001805284600F027FD124B1B68E3B9251D2A
:10A9D000284600F020FD01230F49E26A08689340F1
:10A9E000034314200B6029460C4B00FB023000F09F
:10A9F000EFFC0B4BE26A1B68DB6A9A4285BF0120C1
:10AA0000084B0020186038BD29460748EFE700BF13
:10AA100050880108884800209048002018480020ED
:10AA20000C4800200C490020C8480020034B1B683C
:10AA30000360034B1B684360704700BFC44800209D
:10AA40000849002070B50C46054620B940F665411E
:10AA50001448F8F775FF24B940F666411148F8F735
:10AA60006FFFFEF77FFB104B196823685A1C10D04C
:10AA70000E482E6800686A68864201D08A420FD963
:10AA8000881A83420AD95B1A134423602846FFF7C9
:10AA9000CDFF0024FEF786FB204670BD0023236017
:10AAA0000124F7E75088010808490020C448002025
:10AAB0000122014B1A6070470C49002070B50C460A
:10AAC0001646054608B91B4A156805F1340262604E
:10AAD000EA6A052B22612A6B2560E2616A6CA2603A
:10AAE000EA6C62614FF00002A26119D01149096855
:10AAF000A94209D12273D6B10023296BCA5CA52AC9
:10AB000013D09B08238470BD032B2373F3D1FFF76D
:10AB1000D7FCAB6A0BB102232373FFF777FDEAE79B
:10AB20002846FFF70BFC2073E5E70133E6E72684B0
:10AB3000E9E700BF0C48002008B9064B1868026B13
:10AB40000020135CA52B02D0C0F38F0070470130AA
:10AB5000F7E700BF0C480020014B1868704700BFA2
:10AB60000C480020054B1B6833B1054B1B68002BBC
:10AB70000CBF02200020704701207047DC480020F5
:10AB8000884800202DE9F0410446002836D0234AA9
:10AB9000C36A11681746C96A8B4237D21426826984
:10ABA0001F4D002AA8BF3A6806FB0353A2BFD26A12
:10ABB000C2F10502826142699A4221D100F1040882
:10ABC000404600F028FC174B48B9E06A4643AA59B2
:10ABD0002AB901211A68814022EA01021A603A6802
:10ABE0001968D26AE262012404FA02F0084318608C
:10ABF0001420414600FB025000F0EAFB204603E02F
:10AC00003B68DB6AC3620120BDE8F0811368C06C59
:10AC1000DC6AA0422CBF00200120F5E70C48002090
:10AC20001848002090480020F8B5044608B90020D4
:10AC3000F8BD1F4B1B68834204D040F67A711D4853
:10AC4000F8F77EFE236D23B940F67B711948F8F7BB
:10AC500077FE236DE16AE26C013B91422365E6D009
:10AC6000002BE4D1251D284600F0D5FB124E134AD7
:10AC700050B91421E76A794373582BB9012013683E
:10AC8000B84023EA00031360E36CC3F10501A1613E
:10AC9000E3620124116804FA03F0084310601420F1
:10ACA000294600FB036000F093FB2046C0E700BF8D
:10ACB0000C480020508801081848002090480020C7
:10ACC000F8B50D460446002845D0036D23B940F67B
:10ACD000C9712148F8F734FEE36C9D4238BF1D4628
:10ACE000E36AAB4237D0236D012B34D11B4B1B6879
:10ACF000A34204D140F6E4711748F8F721FE142668
:10AD0000A269E36A002AE562A4BFC5F10505A56151
:10AD1000134D626906FB03539A421CD1271D384626
:10AD200000F079FBE26A0F4C40B95643AB592BB99E
:10AD300001212368914023EA0103236001231420A9
:10AD4000216893400B432360394600FB0250BDE865
:10AD5000F84000F03DBBF8BD508801080C480020C9
:10AD60001848002090480020044B1A681AB119684E
:10AD70000A6D01320A651868704700BF0C48002050
:10AD80002DE9F0411E4C1E4680460F461546FEF743
:10AD9000E9F9236893F85830022B14D00121236875
:10ADA0005A6D22EA08025A65236883F8581056B192
:10ADB0003046FFF7EFF84FF08052124B1A60BFF3A6
:10ADC0004F8FBFF36F8FFEF7EDF9FEF7CBF915B19B
:10ADD00023685B6D2B602368002293F85830022BA8
:10ADE00009BF012500252368596D04BFB943596582
:10ADF000236883F85820FEF7D5F92846BDE8F0818E
:10AE00000C48002004ED00E0F8B50E4617461D463C
:10AE1000044620B941F219212B48F8F791FDFEF7BD
:10AE2000A1F90DB1636D2B60022394F8585084F89A
:10AE30005830EDB2042F16D8DFE807F00A030705F3
:10AE40001100636D1E43666502E0636D0133636547
:10AE5000012D11D00124FEF7A5F92046F8BD022DE1
:10AE6000F1D10024F7E7636D0133F1D041F24A21BB
:10AE70001548F8F765FDEBE7261D304600F0CBFAE4
:10AE80001420124AE36A11689D400D431560104A70
:10AE9000314600FB032000F09BFAA36A23B141F284
:10AEA00059210948F8F74CFD0A4BE26A1B68DB6A36
:10AEB0009A42CFD94FF08052074B1A60BFF34F8FA1
:10AEC000BFF36F8FC6E700BF50880108904800208D
:10AED000184800200C48002004ED00E02DE9F8435C
:10AEE000DDF820800E4691461D46044620B941F209
:10AEF0008C213548F8F724FDFEF70CFAEFF31187A3
:10AF00004FF0500383F31188BFF36F8FBFF34F8F60
:10AF10000DB1636D2B60022394F8585084F85830BB
:10AF2000EDB2B9F1040F16D8DFE809F00A030705FE
:10AF30001100636D1E43666502E0636D0133636556
:10AF4000012D11D0012087F31188BDE8F883022D6F
:10AF5000F1D10020F7E7636D0133F1D041F2CF2149
:10AF60001948F8F7EDFCEBE7A36A23B141F2DA21C7
:10AF70001548F8F7E5FC154B1B6803BB251D284653
:10AF800000F049FA01231249E26A0868934003433A
:10AF900014200B6029460F4B00FB023000F018FA1A
:10AFA0000D4BE26A1B68DB6A9A42CBD90123B8F1E8
:10AFB000000F01D0C8F80030084A1360C2E704F15E
:10AFC00018010748EAE700BF5088010888480020B8
:10AFD00090480020184800200C4800200C49002010
:10AFE000C848002038B5054608B9084B1D6800243C
:10AFF000FEF7B8F895F85830022B04BF85F8584092
:10B000000124FEF7CFF8204638BD00BF0C480020D1
:10B01000F8B50F4CFEF7A6F82568ADB90D4F0E4EEA
:10B02000384600F0C7F9304600F0C4F90B4B2A4609
:10B030001F600B4B0C210A201E60FEF759FB20609D
:10B0400010B10849FEF718FFBDE8F840FEF7AAB8AE
:10B0500044490020184900202C49002010490020B4
:10B060001449002099880108914208B541600061A7
:10B070000AD8D21A83699A420DD2084B011D18686A
:10B0800000F0B2F9002008BD9A4201D2994202D2E2
:10B09000011D034BF3E70120F5E700BF1449002031
:10B0A0001049002007B5FFF7B3FF0C4B1B6843B9ED
:10B0B0000B484FF48971F8F743FC002003B05DF8AA
:10B0C00004FB084BC822019301230749009307485A
:10B0D0000023FEF7DBFF0028EAD0EFE74449002019
:10B0E0009E88010848490020E388010809B2000849
:10B0F0002DE9F04180462C200D4617461E46FEF7EE
:10B1000069F9044688B125B94FF4B6710848F8F7D3
:10B1100017FCFFF77DFF069BC4F80080C4E90657C3
:10B1200026626362201D00F050F92046BDE8F081E0
:10B130009E8801082DE9FF410D4690461F460646B0
:10B1400020B94FF4C3710F48F8F7FAFB0E4C206892
:10B1500078B1052DCDE9015803960DDCFFF702FD0E
:10B16000002302280CBF0A9A1A4601A92068FEF79C
:10B17000E3FA04B0BDE8F08100233A4601A9FEF7E6
:10B1800091FBF6E79E880108444900202DE9F7432A
:10B1900000271A4DDFF86C802B681A6832B9184AFC
:10B1A00011681360296003B0BDE8F083DB68DC68D8
:10B1B0001E6804F10409484600F02DF9636A204630
:10B1C0009847E369012BE7D1A36933449E4206D235
:10B1D000636024614946286800F006F9DCE7002333
:10B1E0000097324619462046FFF7A4FF0028D3D126
:10B1F00040F272314046F8F7A3FBCDE7104900203A
:10B20000144900209E8801082DE9F04F4FF00108F5
:10B21000624D87B0DFF898B1DBF80020136843B3C4
:10B220000024D368D3F80090FFF74AF9FFF750F9EC
:10B230005B4B82461A681F4690425A4E1CD31860D8
:10B24000002C4BD0584B1B681A68B2FA82F2520994
:10B25000A9EB0A013068FEF74BFEFFF7D7F990B96A
:10B260004FF08052514B1A60BFF34F8FBFF36F8F77
:10B2700009E001249946D7E7FFF788FF484BC3F858
:10B2800000A0FFF7C3F9002203A93068FEF7AEFB68
:10B290000028BFD0039B002BF5DB059C636913B12D
:10B2A000201D00F0B8F8FFF713F93B68814698427B
:10B2B00001D2FFF76BFF039BC7F80090092BE2D880
:10B2C00008FA03F313F4047A57D113F0C70F33D1FC
:10B2D0009B06D8D52046FEF709F9D4E7814529D841
:10B2E000FFF794F9DBF80030DB68D3F80CB00BF112
:10B2F000040000F090F8DBF81C30012B15D1DBF8CE
:10B3000018104B46524649445846FFF7ADFE60B10F
:10B31000009423464A4621465846FFF70BFF20B9C2
:10B320004FF4F4712846F8F70BFBDBF8243058464D
:10B330009847A8E722468BE7A169049B4A4619442F
:10B340002046FFF791FE00289DD0636A204698476B
:10B35000E369012B97D1A2690499CDF800A00A44B2
:10B36000534651462046FFF7E5FE00288BD140F2B8
:10B3700001312846F8F7E4FA85E7049BA36123B975
:10B380004FF446712846F8F7DBFAA1694B464A4666
:10B3900049442046FFF768FE75E700BF9E88010814
:10B3A00040490020444900201449002004ED00E0F9
:10B3B000104900204FF0FF3200F108034360C0E95C
:10B3C0000223036100230360704700230361704779
:10B3D00043689A684B608A609A6851609960036814
:10B3E00008610133036070470A6830B5531C0AD105
:10B3F00003695A684A6091608B605960036808610C
:10B400000133036030BD00F108035C682568954294
:10B41000EFD82346F9E70369D0E901128A60516049
:10B420005968814208BF5A60002202611A68013AD5
:10B430001A60186870470000021C18BF0122002122
:10B440000148F9F725B800BF00040240F9F766BCCF
:10B4500038B505460C460020FFF7EEFF45F08000AA
:10B46000FFF7F4FF2046FFF7F1FFBDE83840012069
:10B47000FFF7E2BF08B50120F8F7FCFD0A20F8F756
:10B48000F9FD0B20F8F7F6FD0720F8F7F3FD05208E
:10B49000F8F7F0FDBDE808400420F8F7EBBD000028
:10B4A000204B70B59D780446EDB958B902211E486D
:10B4B000F8F7E8FF23461A460221BDE870401A4813
:10B4C000F8F718BF012805D102211748F8F7D4FF73
:10B4D0002B46F0E7022823D102460146BDE8704022
:10B4E0001148F8F745BF012D14D138B904210E4891
:10B4F000F8F7C8FF002304211A46DEE7012804D12B
:10B5000004210948F8F7B8FFF4E7022808D10246F9
:10B510000421E3E76A21BDE870400448F8F710BA57
:10B5200070BD00BF4C49002000000240EB880108BC
:10B5300008B50020FFF7B4FFF8F7DEFC0120FFF7A5
:10B54000AFFFF8F7D9FC0220FFF7AAFFBDE80840DB
:10B55000F8F7D2BC08B500210120F9F75FFB012004
:10B56000FFF76AFF0023094819461A46F8F7C2FE9A
:10B57000B5214020FFF76CFFA0214120FFF768FFB5
:10B58000BDE8084000210120FFF762BF000402402F
:10B5900010B5FFF76FFF0120FFF74EFF00233A4879
:10B5A0001A461946394CF8F7A5FE00210120F9F793
:10B5B00035FB22787AB1002306211A463248F8F783
:10B5C00099FE06213048F8F757FFF8F795FC192146
:10B5D0005820FFF73DFFFFF7ABFFFFF7BBFF637896
:10B5E0005BB1002304211A462948F8F783FE0023A3
:10B5F0000D211A462748F8F77DFE00220121224836
:10B60000F8F7B6FE00220A211F48F8F7B1FE002223
:10B610000B211D48F8F7ACFE002207211A48F8F765
:10B62000A7FE002205211848F8F7A2FE00220421F7
:10B630001548F8F79DFE0E23022201211248F8F763
:10B6400037FD0E2302220A210F48F8F731FD0E23A1
:10B6500002220B210C48F8F72BFD0E2302220721B2
:10B660000948F8F725FD0E23022205210648F8F7C0
:10B670001FFD094B1B782BB9BDE81040BE210748C0
:10B68000F8F75EB910BD00BF000402404C4900202D
:10B6900000000240000802404F490020EB880108EA
:10B6A00082B00190064B9DF80620BDF804109A70F8
:10B6B00001221980034B1A7002B0FFF769BF00BF67
:10B6C0004C4900204F4900201A4B10B55B78D3B18C
:10B6D0000128194C18D104211848F8F7CDFE0D2186
:10B6E0001748F8F7CFFE23786BB1002304211A46E0
:10B6F0001248F8F7FFFD00230D211A461048F8F70D
:10B70000F9FD0023237010BD40B904210B48F8F760
:10B71000B9FE0D210A48F8F7AFFEE4E70222042142
:10B720000648F8F725FE02220D210548F8F720FE0D
:10B730000123E7E74C4900208C0000200000024074
:10B740000008024008B5FFF795FEFFF7F1FEFFF78E
:10B7500001FFF9F7BFFA012200211F48F8F708FEA0
:10B760000220FFF7B1FF0220FFF79AFE022201211B
:10B770001948F8F7FDFD02220A211748F8F7F8FDED
:10B7800002220B211448F8F7F3FD02220721124888
:10B79000F8F7EEFD022205210F48F8F7E9FD022235
:10B7A00004210D48F8F7E4FD0C4B1B781BB9E2218E
:10B7B0000B48F8F7C5F80B4B1B785BB1002306214B
:10B7C0001A460548F8F796FDBDE8084006210248EC
:10B7D000F8F758BE08BD00BF000402404F490020E2
:10B7E000EB8801084C49002010B5064C0222204687
:10B7F0000021F8F7BDFD2046BDE8104002220121DE
:10B80000F8F7B6BD00140240014BDB68184700BFD3
:10B81000504900200120704701B1096818B1806AC1
:10B82000431A58425841704710B5044618B9D121FF
:10B830000748F8F785F8074B5B689847D4E9062373
:10B84000904271EB0304B4BF101A002010BD00BF7A
:10B850006E8D0108504900202DE9F04188460446CC
:10B8600010B10369012B03D1E6211648F8F768F8F7
:10B87000D4E9062352EA030122D0D4E90867901BD9
:10B8800063EB070107F09EFC05462069013807F0CD
:10B890007FFC0146284607F087FD0546404607F035
:10B8A00077FC294607F0CCFC294607F0BFFB07F0E0
:10B8B000B3FE321847F1000310461946C4E90601E9
:10B8C000BDE8F0816E8D010838B50C4B054618684F
:10B8D00000F0C3FB10B90023184638BD4FF47A744A
:10B8E00003686C431A68A242F6D000F0ADFB002852
:10B8F000F1D003681A689442F6E700BF504900206F
:10B9000041F65832A0F55223A3F61833934224D8B7
:10B91000A0F55423A3F1F902622A1ED96FF45472E0
:10B920009A18C62A19D9A3F21353302B15D9104BE4
:10B93000984214D903F6B833984212D903F5167316
:10B94000984210D903F5167398420ED903F5E173A6
:10B9500098428CBF062005207047002070470120C8
:10B96000704702207047032070470420704700BFD3
:10B97000E8320D00F8B5054618B9F2212148F7F76D
:10B98000DFFF214F386800F068FB002838D0002D19
:10B9900036D003681A79AA422ED11E7B00F054FBE0
:10B9A00008BB6EB3062D03D93F211648F7F7C8FF31
:10B9B000164B53F835400CBBFD211248F7F7C0FF7A
:10B9C0003868744300F049FB0646C8B107683B7904
:10B9D000AB4204D121463846FFF73EFF3C6130467A
:10B9E00000F032FBF0E703681A79AA42D6D11B7B3C
:10B9F000002BD3D00136D1E70026CFE7012CDFD1D1
:10BA0000F8BD00BF6E8D010850490020348901083F
:10BA10002DE9F04F044687B058B3254B00681D69E7
:10BA200007F0B6FB06F09CFF1FA3D3E9002307F045
:10BA300019F9227B06460F462379D4F82890D4F8CA
:10BA40001080D4F808A0BAB1062B98BF194A204636
:10BA500094BF52F823B0DFF868B0FFF7E5FE324636
:10BA60003B46CDE90198CDE903A01348CDF800B0DD
:10BA7000A84707B0BDE8F08F062B98BF0D4A2046B7
:10BA800094BF52F823B0DFF838B0FFF7CDFECDE910
:10BA90000189CDE903A0CDF800B032463B46074806
:10BAA000E6E700BFAFF300800000000080842E4175
:10BAB000504900206C890108558C0108AA8C0108A6
:10BAC000478C010810B5104C206820B923690F4835
:10BAD000BDE81040184700F0C9FA2369014660B17B
:10BAE0000B489847206800F0B8FA044638B9204659
:10BAF00000F0AAFA044610B910BD0648E8E720682D
:10BB0000FFF786FFF3E700BF50490020C88B01080C
:10BB1000E68B0108208C0108F8B5134D06462B7EF4
:10BB20000F4623B940F261111048F7F709FF2C685E
:10BB300024B96B690E4898472046F8BD0D4B204646
:10BB4000002E08BF1E4600F088FA054608B90024FA
:10BB5000F2E7046839462046B0470028ECD1284671
:10BB600000F072FAF1E700BF504900206E8D010825
:10BB7000898B010815B800082DE9F0472F4D814643
:10BB80002B7E0E46904623B940F291112C48F7F7D0
:10BB9000D7FE2C682CB96B692A4898472046BDE827
:10BBA000F087294B2046002E08BF1E4600F055FAAC
:10BBB000824620B96B69254898475446EEE70468E9
:10BBC000237B6BB94FF0FF370024504600F03CFA5E
:10BBD000824690B9B8F1000FE0D0C8F80070DDE7F8
:10BBE000A3684B45EEDB00212046B0470028E9D092
:10BBF0002046FFF719FE0746E7E7DAF800502B7BEF
:10BC0000002BE2D0AB684B45DFDB00212846B04774
:10BC10000028DAD02846FFF707FE6CB187420AD821
:10BC2000D3D1D4E90823D5E90801FBF79BF8002814
:10BC300018BF2C46C9E707462C46C6E750490020E6
:10BC40006E8D0108898B010815B80008AD8B0108BD
:10BC50002DE9FF478946044620B94FF4E971284889
:10BC6000F7F76EFE236923B940F2D3112448F7F7A2
:10BC700067FEDFF894A00027DAF804309847C4E99B
:10BC8000080105462069884607F082FA494607F010
:10BC9000D7FA494607F0CAF906F062FE16A3D3E9BF
:10BCA000002306F0DFFF06F0A7FB07F04BF92D1885
:10BCB00048EB0703C4E906530646206807F068FA14
:10BCC00006F04EFE0CA3D3E9002306F0CBFF04469A
:10BCD00048460D46CDE9026706F042FE2246CDE910
:10BCE00000012B46DAF810100648884704B0BDE87A
:10BCF000F047FFF7E7BE00BF0000000080842E4140
:10BD00006E8D0108888901085049002008B5FFF7A9
:10BD1000F7FD003018BF012008BD000038B50D4DFB
:10BD200004462A7E22B940F20D210B48F7F708FE9F
:10BD300074B1237B63B1002320792373FFF71AFECC
:10BD40002B69064898472046BDE83840FFF760BE9B
:10BD500038BD00BF504900206E8D0108588B010886
:10BD600038B50D4D04462A7E22B940F219210B4800
:10BD7000F7F7E6FD74B1237B63B9012320792373C0
:10BD8000FFF7F8FD2B69064898472046BDE8384084
:10BD9000FFF73EBE38BD00BF504900206E8D010840
:10BDA000718B0108F8B5194D06462B7E23B940F278
:10BDB00025211748F7F7C4FD2C6824B96B6915488D
:10BDC0009847204601E00EB90020F8BD204600F05B
:10BDD00044F904460028F7D023689E420CD13779F5
:10BDE0003046FFF711FD2146286800F04DF938462E
:10BDF000FFF7C0FD0120E8E7204600F025F90446E2
:10BE00000028E9D16B690448DAE700BF50490020F7
:10BE10006E8D0108268D0108488D01082DE9F84333
:10BE2000384D06462B7E8846914623B94FF4F5716E
:10BE30003548F7F785FD3046FFF768FF044630B90F
:10BE40006B693146314898472046BDE8F883304653
:10BE5000FFF73AFD044630B12D482B69314698472B
:10BE60002046FFF79FFF2B7E1BB975212648F7F769
:10BE700067FDAB6830209847044640B96B69254898
:10BE800098476B693146244898470024DCE7302204
:10BE9000002107F0E3FE3046FFF732FD0746207130
:10BEA00038B9EB68204698476B6931461B4898477C
:10BEB000E7E7062803D93F211348F7F741FD184B60
:10BEC000214603EBC70253F83730526823614FF421
:10BED0007A73A2605E4300220023C4E90623012393
:10BEE00026602373C4E90A89286800F097F820794E
:10BEF000FFF740FD2B690B4898472046FFF788FD68
:10BF0000A2E700BF504900206E8D0108408A010859
:10BF1000778A0108AC8A01081D8B0108DA8A0108BA
:10BF200034890108058B010870B50F4C0546237E46
:10BF300023B940F261210D48F7F702FD23685BB198
:10BF40000B4E29463046FFF7E7FD50B923692946D5
:10BF5000BDE870400748184763690748BDE870406E
:10BF60001847FFF751FCECE7504900206E8D01089F
:10BF700019B80008008D0108268D0108014B187EB4
:10BF8000704700BF5049002084B070B504AC84E80D
:10BF90000F00154B1A7E1C462AB1BDE870405B6944
:10BFA000124804B018471D1D04AE0FCE0FC53368EC
:10BFB0002B600BB90E4B636123690BB90C4B2361EA
:10BFC000E3680BB1A36833B923690A4898470A4B61
:10BFD000E3600A4BA36000F013F80123206023768E
:10BFE000BDE8704004B0704750490020CC8901087A
:10BFF000C16E0008058A0108E13B0108D13B010838
:10C0000010B50820FAF7ECFF0446FEF759FA0023B2
:10C01000C4E90034FEF7FAFA204610BD70B50546B3
:10C020000C200E46FAF7DCFF044660B10660FEF70E
:10C0300047FA002363606B68A3601C6004346C6083
:10C04000FEF7E4FA012070BD10B50446FEF738FA99
:10C050006468FEF7DBFA204610BD10B50446FEF713
:10C060002FFA2468FEF7D2FA204610BD10B5044618
:10C07000FEF726FA236800241BB9FEF7C7FA20460C
:10C0800010BD01345B68F7E738B50C460546FEF78E
:10C0900017FAD4E901324BB19A60A2681360FEF737
:10C0A000B5FA2046BDE83840FAF784BF6A60F4E785
:10C0B00010B5084CD4F8D4201AB962210648F7F715
:10C0C0003FFCD4F8D4000023BDE810400322202117
:10C0D000FEF79ABE90000020F992010838B50E4C88
:10C0E0000E4D94F82A30022B11D123680C48984742
:10C0F000062394F8A720D4F8A810012002F03AFAF9
:10C100006B6B00209847042384F8283038BDEB6A15
:10C1100098470123F8E700BF90000020EC85010854
:10C120003993010810B5044601F05CF840B9054B9D
:10C1300005481B6898472046BDE8104001F02AB822
:10C1400010BD00BF90000020D7920108044B1A7F59
:10C1500022B993F82D0080F001007047002070474D
:10C1600090000020F0B591B00C4640220021054619
:10C17000684607F073FD08F0B1FB0746204608F05B
:10C1800089FB002402AE08F0A9FB0134102C06F84C
:10C19000010BF8D1002408AE08F0A0FB0134102CEC
:10C1A00006F8010BF8D100240CAE08F097FB01341F
:10C1B000102C06F8010BF8D1002406AE08F08EFB17
:10C1C0000134082C06F8010BF8D1384608F062FB60
:10C1D0002C466B4610AE1A4603CAB242206061601C
:10C1E000134604F10804F6D1284611B0F0BD000052
:10C1F00084B070B58AB00EAC84E80F00704CB822E1
:10C200002546002104F128000EAE07F027FD0FCED1
:10C210000FC5336813AE2B6004F114050FCE0FC5A4
:10C2200033682B600E9B0BB9664B23600F9B0BB9D9
:10C23000644B2360109B23B940F22B116248F7F73F
:10C240007FFB129B23B940F22F115F48F7F778FB71
:10C25000119B23B940F233115B48F7F771FB636917
:10C2600023B923685948984703236361A3690BB92D
:10C270000A23A361A37F0BB90123A37701F0C2FEB8
:10C28000E37F0BB90123E37701F0B4FE636A0BB9D6
:10C290004F4B636201F0A2FEFBF7B4F8C4F8D00084
:10C2A0000138033004D963684A48984700207EE08B
:10C2B000032200210120FDF71BFAC4F8D80020B9A1
:10C2C0004FF4AE714048F7F73BFB00220421A06910
:10C2D000FDF70EFAE06320B94FF4B0713A48F7F772
:10C2E0002FFB00220421A069FDF702FA206420B987
:10C2F00040F263113448F7F723FB002204210120A8
:10C30000FDF7F6F9606420B94FF4B3712E48F7F7E2
:10C3100017FB082384F8AF30042384F8B0300023DF
:10C3200084F82E30FFF72AFE05AD68B9A3682269AC
:10C330000593236807920893E26863680692009366
:10C3400095E80F00FFF720FE01F082FE2368224EE1
:10C35000079363680496089323690693E36805933B
:10C3600006F15003039303AB93E803008DE8030049
:10C370008C3695E80F0002F045F9019663694FF499
:10C38000CD720093154901231548FDF77FFE012862
:10C39000054611D1002303220421D4F8D400FEF76E
:10C3A00033FD104823689847284684F82C500AB07B
:10C3B000BDE8704004B0704763680B4875E700BF84
:10C3C00090000020C16E0008F9920108588F010802
:10C3D00008E6D333A18F0108D8000020D48F0108CC
:10C3E0008DC50008DC8F0108F98F010810B5154CC8
:10C3F000D4F8D43023B94FF4C9711348F7F7A0FA31
:10C40000042100230322D4F8D400FEF7FDFC0F48DA
:10C410002368984742F21071D4F8D800FDF778FBF2
:10C4200020B940F29B110848F7F78AFA0023D4F8A4
:10C43000D8001A461946FDF77FF923680448BDE87D
:10C440001040184790000020F9920108C49001089C
:10C45000EB90010838B50E4DD5F8D83023B940F22D
:10C46000A3110C48F7F76CFA0021D5F8D800FDF7B6
:10C470004FFB0128044608D10023D5F8D8001A46FE
:10C480001946FDF759F9204638BD0020FCE700BFEA
:10C4900090000020F992010810B5FFF7DBFF0B4C6C
:10C4A00078B1002303220821D4F8D400FEF7ACFCB5
:10C4B000236807489847D4F8D400BDE81040FDF73A
:10C4C0007DBF23680348BDE8104018479000002056
:10C4D0000691010828910108014B5863704700BF7D
:10C4E00090000020002307B50193054B024601A9E7
:10C4F000586CFDF77BFA019803B05DF804FB00BFB0
:10C500009000002070B5FFF7A5FF1B4D044620B139
:10C510006B681A489847002070BDE86BFDF786FCF1
:10C52000AB69834202D22B681548F3E721462046C7
:10C5300002F098F8064610B92B681248EAE7047032
:10C5400000F016FE044618B9304602F0CBF8E2E7D8
:10C550000D4A1368013313605BB91368013313602C
:10C56000636040F2031320462380FFF7DBFD606821
:10C57000D2E71368F4E700BF90000020299001087B
:10C5800055900108879001086C49002001232DE98E
:10C59000F0416E4CDFF8BC816D4E84F828300A23E0
:10C5A0006C4A4FF0FF310020FEF7EAFB012870D102
:10C5B000D8F8000043071DD5337833B1FAF770FE81
:10C5C0000020FAF7C1FE00233370FCF7CBFD23688F
:10C5D00061489847FCF7E6FD022384F828300023E1
:10C5E000D4F8D8001A461946FDF7A6F80020FEF741
:10C5F00039F9D4E710F0080524D0337893B941F223
:10C600008830FAF779FE18B99E215448F7F798F95F
:10C610005348FAF799FE012352483370236898472C
:10C62000FFF75CFD0020FEF7DDFC4FF4FA61D4F863
:10C63000D800FDF76DFA0028B1D1A5214748F7F7DA
:10C640007FF9ACE710F0200053D03378F3B194F8C1
:10C650002830042B1AD1444F2A463946D4F8D0004A
:10C66000FDF706FB012811D13B78072B31D13F485C
:10C6700023689847284600F07BFD38B140F2051248
:10C68000C0E9015505610280FFF74CFD0020FEF76F
:10C69000A9FC3378002B82D000F0BCFD05460028B1
:10C6A0003FF47DAF032384F8283003784168052BDD
:10C6B00098BF2F4A276894BF52F823202D4A2E484E
:10C6C000B8472B78052B3DD8DFE803F0161D1D3148
:10C6D00031392A463946D4F8D000FDF787F90128C8
:10C6E000D4D123683978254898473846FAF732FE7E
:10C6F000CCE7FEF777FC52E7D4211848F7F720F98A
:10C70000FFF7ECFC4BE7FFF721FD38B9284600F0B6
:10C7100095F980B1284600F03DFDF1E723681848FF
:10C7200098472846FFF7FEFCFFF7ECFEE8E72846AF
:10C7300001F0D0FAEDE72846FFF7F4FCE0E700F05F
:10C740009FFCE7E763680F489847E3E79000002005
:10C75000704900207C490020648E0108F99201088C
:10C76000B1C00008878E010874490020B78E010807
:10C77000448E01085C8E0108F38E0108CE8E0108FC
:10C78000118F0108388F0108024B93F8A40001F0C3
:10C790002DBE00BF900000202DE9FF4180460F46CE
:10C7A0001646ADF80430FFF755FE494D044638B142
:10C7B0006B68484898470024204604B0BDE8F081E3
:10C7C000E86BFDF733FBAB69834203D22B68424829
:10C7D0009847F1E7FFF7D8FF8742014605D92B6854
:10C7E00095F8A4203D489847E6E71EB93FB12B686D
:10C7F0003B48DFE7DF2E02D92B683A48E8E73946A5
:10C80000404601F02FFF044610B92B683648DFE799
:10C810009DF80530002B14BF0423022303709DF8FC
:10C82000043033B10D23012203A98DF80C3001F03F
:10C83000C7F995F8292095F82A30934203D195F845
:10C840002B30934217D02023022A18BF00228DF8E4
:10C850000C3094F8583003A90BBF43F0040343F0A5
:10C8600001038DF80D208DF80D20204684F85830F6
:10C87000022201F0A5F96677204600F079FC064611
:10C8800018B9204601F02EFF95E70023174A836070
:10C890001368013313609BB913680133136073602D
:10C8A0000A9B3046336140F20113338000F084FC70
:10C8B000044638B9304600F06DFC6B680C4887E7D9
:10C8C0001368ECE72B6871680A489847746873E747
:10C8D00090000020299001085590010868910108F6
:10C8E000C4910108F6910108389201086C490020B2
:10C8F00073920108A5920108082808BF0120024B85
:10C90000987783F8A400704790000020024BD877F6
:10C9100083F8A500704700BF9000002008B509F01B
:10C9200073FE014B986408BD90000020034630B5AB
:10C93000054C00F11005224618685968083303C2F7
:10C94000AB421446F7D130BDDC000020034630B5C1
:10C95000054C00F11005224618685968083303C2D7
:10C96000AB421446F7D130BDEC0000200246024B2A
:10C970000068516803C370470C0100200246024B57
:10C980000068516803C3704714010020034630B5A6
:10C99000054C00F11005224618685968083303C297
:10C9A000AB421446F7D130BDFC000020014B587754
:10C9B000704700BF9000002030B1044B044A0228A9
:10C9C0000CBF184610467047024870476091010836
:10C9D0005C8E010858910108014B9863704700BFB5
:10C9E0009000002038B50D461446FFF797FF284603
:10C9F000FFF79CFF2046FFF7A9FF0122014B1A77A2
:10CA000038BD00BF9000002038B50D461446FFF732
:10CA1000ADFF2846FFF7B2FF2046FFF7B7FF002221
:10CA2000014B1A7738BD00BF9000002028B1836AFF
:10CA3000012B01D1007B7047002070472DE9F047A2
:10CA4000044686B010B10378012B03D01C217C482A
:10CA5000F6F776FF63691BB91D217948F6F770FF79
:10CA600063691B78042B05D0022B03D01E21744868
:10CA7000F6F766FF4FF00008724E73483368984728
:10CA8000D6E929A903AA714996F8A500CDF80C802A
:10CA9000FFF772F83546074650B933686C48984737
:10CAA000204600F021FC0127384606B0BDE8F0879B
:10CAB000039BABB1FFF706F80399042904D920467C
:10CAC00000F04AFC0027EFE7336862489847039874
:10CAD000614B43434FF47A70B3FBF0F0FDF74AFE2D
:10CAE000A3680133012BA3600FD1D5F8983060699A
:10CAF0000133C5F8983095F8AE30013385F8AE3083
:10CB000000F096FC606901F087F8AB6C60694360E7
:10CB1000D5F89830438195F8AC3033B1002385F8CF
:10CB2000AC30037A43F0040303720026012100F0C5
:10CB3000A9FC05AB019304AB009339464FF4FA63AB
:10CB40004FF47A726069049600F08EF9074610B9C6
:10CB50002B684248A3E7FDF7BBFCE060049848B1AE
:10CB6000314600F08FFC049B1B78052B04BF01238A
:10CB700085F8AC30049800F027FCDDE9040101F0F1
:10CB800059F8049A12B3137A13F0040807D0B84680
:10CB90002B6851893248984795F8B130A360049BBF
:10CBA00033B163691B78022B04BF95F8B130A360E1
:10CBB00000F046FB064640BB7D212148F6F7C0FE4B
:10CBC000284B294A7E211E4806F000FF9046E6E7E2
:10CBD0003146606898476420FDF7CCFD304600F090
:10CBE0003FFB2B6895F8B120A1682048984795F83D
:10CBF000B130A2689A422B6802D31D48984753E788
:10CC00001C489847032333705CE760226169183041
:10CC100006F0FCFF0023049A3366B2672278737231
:10CC2000337095F82D30C6E903A933752369727006
:10CC300086F80880002BCBD1304600F033FBD0E7DC
:10CC40008993010890000020C69301082DCA0008AE
:10CC5000EA9301082494010840420F00519401080E
:10CC600091940108AD9401087B930108B6940108E2
:10CC7000D3940108E79401082DE9F04186B080467D
:10CC80000C468DF80F202BB101220DF10F01002071
:10CC9000FBF702F80025284B20469DF80F109B6AF1
:10CCA0009847264F05AB009304AA2B4629469DF8CA
:10CCB0000F00234ECDE90455FAF7E2FBDDE904232A
:10CCC0009DF80F101F483C68A04740F6B832314627
:10CCD000D7F8D000FCF78AFE38B3FDF7F9FB3378BC
:10CCE0000446012B30461CD1FAF734FB049806F0B9
:10CCF0004FFA01464046FEF7ABFFD8F8000006F0B9
:10CD000047FA05F02DFE0AA3D3E9002305F0AAFF98
:10CD10003D6802460B460C48A847204606B0BDE8D1
:10CD2000F081FAF717FB2C46F7E70446F5E700BF5A
:10CD30000000000080842E41EC8501089000002056
:10CD400080490020DB9601080B9701082DE9F84F78
:10CD50003C4C1F46636B0546884691469847A34660
:10CD6000394E3A4CDFF8FCA04FF47A7202FB05F31F
:10CD700003F5C333A033B3FBF2F23449D6F8D00045
:10CD8000FCF734FE28B9DBF8303098474FF0FF301D
:10CD900036E02378072B0DD1FAF700FF2046FAF78B
:10CDA000D9FA3568FDF794FB01465046A8474FF481
:10CDB0007A65D9E7032BDBF830A023D13568FDF77E
:10CDC00087FB01462248A84765682879296881457C
:10CDD00028BF814640464A4606F018FF366895F956
:10CDE0000830B5F90620A9881A48B0471FB1EB886A
:10CDF0003B802B7ABB701548FAF7ACFAD04748460F
:10CE0000BDE8F88F042B0BD13468FDF761FB0146B8
:10CE10001148A0470D48FAF79DFAD0470020EFE7E8
:10CE2000052B0AD13468FDF753FB01460B48A04798
:10CE30000648FAF78FFAD047A8E7C6210848F6F760
:10CE40007FFDF5E7EC85010890000020884900206F
:10CE5000359501084A9501087F95010897950108C5
:10CE6000AD9501081B9501082DE9F04FC3B0884628
:10CE7000DDE94C97164602A9FF2283469A4601F047
:10CE800051FC704C054630B923686F489847002024
:10CE900043B0BDE8F08F94F8A53094F8A420D8F8FA
:10CEA0000010002001F066FB00232A4602A940463C
:10CEB000FFF7E2FE019010B923686448E6E79BF8AB
:10CEC0005830254613F0050F11D013F0040F0CBF96
:10CED0000020022094F82A30834208D084F82A00E7
:10CEE000D4F800B0FFF768FD01465948D847FF2243
:10CEF000002102A806F0B2FE95F8A42095F8A6300D
:10CF0000D8F8001093429ABFD21AD2B20022062358
:10CF1000012001F02FFB2568FDF7DAFA4FF47A784B
:10CF2000019A0146323A32444A48A84708FB06F1C2
:10CF3000A1F543415039B1FBF8F101A8FDF7DAFB47
:10CF4000D4F800B0FDF7C4FAAAEB0606A6F1640512
:10CF50002A4601464048D847FF223B4602A92846B8
:10CF6000FFF7F4FED4F800A00546FDF7B1FA01463C
:10CF70003A48D0476A1C02D12368394886E7002D19
:10CF800025DD23682946374898470FB10123FB70F8
:10CF90000026B542C9F8006017DDE9B202A801F029
:10CFA00025FF284FC9F800003B682F489847DFF855
:10CFB000CC8002AC3B6814F8011B40460136984710
:10CFC000B542F7D13B6829489847012060E706231E
:10CFD00094F8A720D4F8A810012001F0CBFA256816
:10CFE000FDF776FA08FB06F601462148A847B6FB8E
:10CFF000F8F101A8FDF77EFB2568FDF769FA40F618
:10D00000B83201461448A8473B46FF2202A940F621
:10D01000B830FFF79BFE26680546FDF759FA014632
:10D020000E48B0476B1C02D1236812482EE7002D32
:10D03000AEDD2368294610489847002FA8D0022368
:10D04000A5E700BF9000002097970108B797010857
:10D05000D597010803980108309801084C980108F9
:10D060005D980108869801081B990108BD6F0108A9
:10D07000A8980108CF980108F8980108D79B0108E3
:10D080002DE9F0412E4CC2B023684FF47A612D484F
:10D09000984701ABFF2202A94FF47A60FFF756FED2
:10D0A000061E254649DD23683146274898472368F0
:10D0B000264898470024DFF8B48002AF2B6817F8A1
:10D0C000011B404601349847A642F7D12B682048FF
:10D0D0009847AA6CF1B202A801F098FC044600B38C
:10D0E00003782F68052B20D0032B23D11949627FA9
:10D0F000237F1948B8472B6814489847217FA06CB4
:10D10000F9F748FF2B68124898470021204600F0A5
:10D11000B9F9AB6B5BB92B6810489847204601F012
:10D12000E1FA304642B0BDE8F0810D49DFE7204624
:10D130009847F6E70B48B847F0E723680A48F7E74F
:10D1400090000020EB950108189601081B99010832
:10D15000BD6F0108E8950108319601087C96010829
:10D16000BE6F0108A4960108CA960108D79B010862
:10D1700038B5074B0546DB6818209847044620B1B0
:10D180001422002106F06AFD6561204638BD00BF0B
:10D190009000002010B5044650B1406901F0A2FA99
:10D1A00000236361034B2046BDE810401B6918470C
:10D1B00010BD00BF90000020037807B5052B4FF08D
:10D1C0000003019006481A4601A90CBF006CC06B11
:10D1D000FCF7B2FA431E5842584103B05DF804FB15
:10D1E0009000002007B5037801900948052B4FF007
:10D1F00000024FF0010301A90CBF006CC06BFCF7EB
:10D200009BFA431E5842584103B05DF804FB00BF2F
:10D2100090000020002213B5084C01A9206C019257
:10D22000FCF7E4FB019B33B994F82E201AB901A94D
:10D23000E06BFCF7DBFB019802B010BD9000002012
:10D24000064B10B5DB6880209847044618B1802251
:10D25000002106F003FD204610BD00BF9000002015
:10D2600070B504460C4D0D482B68984794B1236E59
:10D270002BB12B680A4898472B69206E9847A06FFE
:10D2800018B101F02FFA0023A3672B692046BDE8EF
:10D290007040184770BD00BF900000206A970108D9
:10D2A000839701081FB50E4C0190606CFCF7D0FD10
:10D2B000024638B903A9606CFCF798FB10B10398DB
:10D2C000FFF7CEFF002301A91A46606CFCF734FA81
:10D2D00020B940F257110348F6F732FB04B010BDF5
:10D2E00090000020AD950108F8B504234370037841
:10D2F0000546032B0ABF144B04695C6BFFF7A0FFC4
:10D300000646B0B94FF4B3711048F6F719FB104B4D
:10D31000104A40F267110D4806F058FB3146686824
:10D32000A0473046FFF79CFFFA20FDF723FA384666
:10D33000F8BD01272B7807704370002CEED1FFF762
:10D34000B1FF2046F4E700BF90000020AD95010832
:10D350001395010826970108F8B503780646032BB4
:10D3600008BF154B0F460CBF5C6B0469FFF768FFE5
:10D370000546B0B940F27F111048F6F7E1FA104BBC
:10D38000104A4FF4C0710D4806F020FB2946706822
:10D39000A0472846FFF764FFFA20FDF7EBF90120CC
:10D3A000F8BD02230370337847604370002CEDD141
:10D3B000FFF778FF2046F3E790000020AD950108C5
:10D3C000139501084297010837B5164C10B1002398
:10D3D00084F8AE30637F13B394F8AE1094F8AF20A6
:10D3E00091421CD994F8B0308D1A95FBF3F003FBF1
:10D3F0001050A0B90C482568A84700F00BFE20B9D2
:10D4000000F016FE08B900F023FEA37F2568009304
:10D41000E27F94F8A43094F8A5100448A84703B01C
:10D4200030BD00BF9000002050990108A699010866
:10D4300070B5114C0546637FEBB1037A266843F063
:10D440000103037294F8AF2094F8AE1094F8B03052
:10D450000A48B04794F8AE1094F8AF2091420AD928
:10D460002B7A246843F002032B72A446BDE8704077
:10D4700001230348604770BD90000020D599010842
:10D48000159A01082DE9F34105464D4C4D4A0E1EF3
:10D4900023684D494D4808BF1146984723684C48BA
:10D4A0009847696C23684B4898472B784A48072B64
:10D4B00096BF4A4A4A4952F8231027686A78B84703
:10D4C0002368484898472368697F474898472368F6
:10D4D000297F4648984723686989454898472368C3
:10D4E000696844489847297A0B090193C1F3C0033E
:10D4F0000093002E32D0C1F38003C1F340022668AE
:10D5000001F001013C48B0472B7A13F0F00F11D025
:10D5100023683A486FF00B079847DFF8F48005F16D
:10D520000C067F1B297ABA19B2EB111F236810DB96
:10D53000334898472368334898472B7F002B3AD1CC
:10D5400023683148984723682D4802B0BDE8F04170
:10D55000184716F8011B40469847E3E7C1F38003DC
:10D56000C1F34002266801F001012848B0472B7A38
:10D5700013F0F00FDED0236820486FF00B079847B8
:10D58000DFF88C8005F10C067F1B297ABA19B2EB03
:10D59000111F2368CCDA16F8011B40469847F4E7C0
:10D5A000AB6C4046995DB84701362A7FB3B29A42C8
:10D5B0002768F5D8C7E70026DFF85880F5E700BFF1
:10D5C00090000020579A0108509A0108609A0108BB
:10D5D0007C9A0108929A0108A19A010830990108E1
:10D5E0005C8E0108B59A0108C29A0108D89A010810
:10D5F000F79A01080F9B0108289B01086D9B010801
:10D60000BD6F0108BF9B0108CE9B01087D9B0108EF
:10D61000D79B0108D69B0108064A1378FD2BDFBF74
:10D6200000780549C8540133DABF01201370002087
:10D63000704700BF914A00209249002038B100781D
:10D64000032803D0431F58425841704701207047B8
:10D65000084B07B51B680848984705230DF10700DC
:10D660008DF80730FFF7D8FF0448FFF7D5FF03B068
:10D670005DF804FB90000020A2A001089049002062
:10D680002DE9F04F00268FB0CDE90401CDE9062346
:10D690009DF860A0934D564580F07282079B92489A
:10D6A00013F806B09F190BF1FF32D2B21F2A98BFB0
:10D6B0008E492B6894BF51F822208D4A59469847CD
:10D6C000ABF103031D2B00F24D82DFE813F01E00C7
:10D6D000CD012D01EE008E01CD01CD01AF014B0238
:10D6E000D001C100FB01FD014B024B024B024B027A
:10D6F0004B024B024B024B024B024B024B024B02C2
:10D700004B024B024B024B0220020024AAEB060301
:10D71000DBB208938DF82C40089A231D9A4202DD53
:10D720003B5D032B1CD0A4B103230CA88DF8303033
:10D73000FFF772FF0BA8FFF76FFF9DF82C102F6803
:10D7400001F001030093C1F38002C1F34003694873
:10D75000B8473444E2B2964200F00B8216469AE78C
:10D7600007EB040999F80180A01C4FEA181138440E
:10D77000099108F054FF99F804900999C9F302132C
:10D780000534062908F00F080290039309F00F09E9
:10D79000E4B235D90F2939D19DF82C3043F002037A
:10D7A0008DF82C3008F1FF32042A2B6832D9B8F1F9
:10D7B0000F0F37D19DF82C3043F004038DF82C3037
:10D7C000B9F1000F07D02B684A4695F8B1104A48C6
:10D7D000984785F8B190039A2B683ABB029947485D
:10D7E0009847029800F004FD9DF82C3043F00103A7
:10D7F0008DF82C302B68DDE90221414898478BE7F2
:10D8000085F8A4102B683F489847C5E72B683E4829
:10D810009847C7E7424695F8A5103C48984785F8D1
:10D82000A580C7E741463A489847C9E7039A062AC0
:10D83000E0D14FF6FF71314898474FF6FF7000F086
:10D84000D7FC9DF82C3043F001038DF82C3063E7B2
:10D85000AAEB0603DBB2052B40F282813B780D2B4D
:10D8600040F07E81781C08F0CDFE002197F905304C
:10D87000002BACBF274B284BC418069B41F1000777
:10D88000012B0DD1013447F1000704992B68224682
:10D89000096D22489847049BC3E9144706221EE0FD
:10D8A000069B022BF1D10234EDE73B78062B40F0CA
:10D8B00057810BA88DF82C30FFF7AEFE059B95F82D
:10D8C000B21003F01F028DF8302015482C68A047D5
:10D8D0001448FFF7A1FE0CA8FFF79EFE0122324478
:10D8E000C3E000BF90000020189D0108909C010833
:10D8F000109D0108089E0108AB9D0108C49D010808
:10D90000DD9D0108399D01085A9D0108779D010898
:10D91000909D01086E3DD5126F3DD5123E9E0108C7
:10D920005C9E010842010020AAEB0603DBB2042B37
:10D9300059D93C78052C56D1D7F801202B680C9288
:10D9400095F8A610C2F302128F4898479DF8302030
:10D950008E4FC2F3021385F8A6303B7802F00F0217
:10D9600043F00403052A3B702B682DD895F8A710C7
:10D97000874898479DF83030C3F3030385F8A730F4
:10D980003B7843F002030DF131003B704FF0640827
:10D9900008F03DFE08FB00F84046FAF701F92B6855
:10D9A0008146C0B14246D5F8A8107A489847774AD0
:10D9B000C5F8A880137843F0010313700122764B59
:10D9C0001A70FFF745FEC4E61146744898473B7845
:10D9D0006FF34103D7E74146714898473B7869F3B5
:10D9E00000033B70EAE70024B3E6AAEB0603DBB2D0
:10D9F000052B40F2B5803C78072C40F0B1806421C3
:10DA000057F8010F030A3A790C905943C0B28DF8C8
:10DA1000342000F06FFB8DF828000BA88DF82C4007
:10DA2000FFF7FAFD0AA8FFF7F7FD37E7AAEB0603B1
:10DA3000DBB2042B40F294803C780A2C40F09080BA
:10DA40006421D7F80100030A5943C0B200F09AFBE1
:10DA50008DF82C000CA88DF83040FFF7DDFD0BA8E9
:10DA6000FFF7DAFD05223AE7B21CD2B273E6AAEB61
:10DA70000603DBB2012B73D097F80080B8F10C0FCE
:10DA80006ED14FF001097C782B68270909FA07F756
:10DA900004F00F043A4695F8AF10424809FA04F929
:10DAA0009847414885F8AF702B684A4695F8B01002
:10DAB000984785F8B0908DF830800CA8FFF7ACFD42
:10DAC00002220CE7F21CD0E7AAEB0603DBB2012B23
:10DAD00046D097F80080B8F10F0F41D1AB687C7841
:10DAE0009847012223090A33C5E92E0102FA03F3FC
:10DAF00004F00F040CA8C5F8C030C5F8C4408DF878
:10DB00002C208DF83080FFF787FD0BA8D6E7AAEB15
:10DB10000603DBB2012B23D03B78202B20D17C786D
:10DB20000CB1022C1CD120462F68FEF745FF0146A0
:10DB30001E48B84795F82B00844203D12B681C4837
:10DB40009847BDE72F68FEF737FF80462046FEF76F
:10DB500033FF414602461748B84785F82B40AFE7E8
:10DB60000022BCE6AAEB06022B68594612489847E9
:10DB70003246124BAAEB02021B6859460E489847E0
:10DB80000FB0BDE8F08F00BF809E010890490020D3
:10DB9000AF9E0108FD9E010891490020DB9E01080F
:10DBA0002A9F0108519F0108769F01089B9F010849
:10DBB000C69F0108E99F010810A0010890000020FD
:10DBC000037A70B51B09D61804460F2E00F10C001D
:10DBD000154618440D4E0BDC06F018F8237A0C4855
:10DBE00065F307132372294633689847012070BDF7
:10DBF000C3F10F0206F00AF8237A064843F0F00357
:10DC000023722946336898470020F0E790000020EF
:10DC100048A001086CA0010810B5044C227822B17C
:10DC20000349FFF7CDFF0023237010BD914A002068
:10DC30009249002030B585B003910446174B30B9A6
:10DC40001B78FBB105B0BDE83040FFF701BD0025F2
:10DC50009DF90E109DF80F201D70FFF7EFFC88B1A5
:10DC60000F48237A457F2DB113F0010518BF012518
:10DC700080F8AD501B0907D0009304F10C03204637
:10DC8000FFF7FEFC05B030BD637F002BFAD1237F88
:10DC9000002BF7D00093A36CF1E700BF914900205F
:10DCA0009000002010B5044678B1836A012B0CD196
:10DCB000C36A1BB910210648F5F742FEE36A58789B
:10DCC00002288CBF0020012010BD0020FCE700BF0F
:10DCD0007CA101082DE9F047054686B018B103780C
:10DCE000033B012B03D922219348F5F729FE6B69E9
:10DCF0000BB11B781BB123218F48F5F721FE4FF0A4
:10DD0000000A8E4E8E4833689847D6E9299896F8CF
:10DD1000A54000F06FF900F075F9204603AA894983
:10DD2000CDF80CA0FDF728FF3446074638B98648E1
:10DD3000336898472846FFF7D7FA01270AE0039B84
:10DD4000C3B1FDF7BFFE0399042907D92846FFF7A1
:10DD500003FB5746384606B0BDE8F08733687B487A
:10DD6000984703987A4B43434FF47A70B3FBF0F033
:10DD7000FCF700FDAB680133012BAB6009D1D4F88F
:10DD800098300133C4F89830724B5B699847A4F817
:10DD90008C00B4F88C3094F8A7600133A4F88C3070
:10DDA000002384F8A730049305AB019304AB0093E0
:10DDB000394641F2707341F288326869FFF754F8CE
:10DDC000074658B92368644898472846FFF78CFAF5
:10DDD000049800F087FC84F8A760AEE7049A84F802
:10DDE000A760236812B11278012A08D05B489847CF
:10DDF0002846FFF779FA049800F074FCAAE758481F
:10DE00009847236857489847049BA16CDA6856489E
:10DE1000A26423689847049BDFF870E103F13202A3
:10DE2000944603F1420A764610685168083203C6E8
:10DE30005245B646F7D14D4E2233324618685968DE
:10DE4000083303C263451646F7D10026236894F8C9
:10DE50006B2094F85C1046489847236894F85B2040
:10DE600094F84C1043489847049B216B9A684248A9
:10DE7000226323689847049B94F8A7101A7C3F48B4
:10DE8000C2F3030284F8A720236802F00F02984728
:10DE9000049B94F8A6101A7C3948C2F3021284F845
:10DEA000A620236802F007029847D4F89810C4E926
:10DEB0002766C4F898602368324898472368324838
:10DEC000984794F82930049813F0FD0F668500F107
:10DED000120018BF84F8296000F0C6F923682048B2
:10DEE0009847FDF7EFFD012384F82D30FFF7A8F9DF
:10DEF000602206466969183005F088FE0023049AFE
:10DF00003366B26794F82D20737233702B783275B4
:10DF10007370636BC6E903984BB1314668689847E4
:10DF20006420FCF727FC3046FFF79AF912E73046E9
:10DF3000FFF7B8F90EE700BF7CA1010890000020B0
:10DF4000B7A10108A5DC0008D7A1010824940108A5
:10DF500040420F00EC8501080DA2010847A201080C
:10DF60007DA20108C5A20108ECA20108DC00002086
:10DF700018A3010856A3010894A30108C1A301082E
:10DF8000EFA3010820A4010850A40108EC00002020
:10DF9000437882781B02007843EA024303430A2055
:10DFA000B3FBF0F07047000038B5044681B10D783E
:10DFB00084B1A36A012B0DD1E36A1BB95421064831
:10DFC000F5F7BEFCE36A5878431B5842584138BD08
:10DFD000FF25EDE70020FAE7CCA40108044B93F8F5
:10DFE000202083F8A7205A6AC3F8A820704700BFF2
:10DFF00090000020024BDA7F83F8A520704700BF15
:10E0000090000020024B9A7F83F8A420704700BF45
:10E0100090000020054BDA7F93F8A51091423ABF9B
:10E02000012083F8A5200020704700BF9000002049
:10E03000064A92F8A430917F99423DBF03F1FF3325
:10E04000012082F8A4300020704700BF900000201B
:10E0500010B5FFF7C3FF0120FDF766FF5023164CF4
:10E06000012123700023224614486370FDF7D6FE79
:10E0700018B932211248F5F763FC50230121114AE7
:10E080001148A370E170FDF7C9FE18B936210C489C
:10E09000F5F756FC5023237102230C4A01210C484A
:10E0A0006371FDF7BBFE28B9BDE810403A21044872
:10E0B000F5F746BC10BD00BF784E0020043F0D00B0
:10E0C000CCA401087A4E0020CC3F0D007C4E0020ED
:10E0D00094400D0007B58DF807000DF107010448C5
:10E0E000FDF71AFD08B1FDF75DFE03B05DF804FB16
:10E0F000A9DF00082DE9F8431746C7F30312052AE4
:10E10000044689464FF000052FD91A4B07F00F013E
:10E110001B68194898474FF000084FF47A76B9FB0E
:10E12000F6F63046FDF7F2FD08B10F2C20D9114B61
:10E1300049461B6811489847002368F3000563F3BC
:10E14000410505F00303032B0CD12046FFF7C2FF66
:10E150000B4B012103EB4402547003F8147030465A
:10E16000FDF75CFE2846BDE8F8834FF00108D4E7D0
:10E170000123E2E7900000204EA501086EA50108EA
:10E18000784E00200F282DE9F04105460F461FD894
:10E19000164B03EB40035C78231A5C425C414FF45E
:10E1A0007A78B7FBF8F0FDF7B1FD4FF0000360F3AC
:10E1B000000364F3410303F00303032B064609D075
:10E1C0004FF0000066F3000064F34100BDE8F08109
:10E1D0000024E4E72846FFF77DFF044A012102EB13
:10E1E000450208FB07F0FDF719FEE9E7784E00202D
:10E1F0002DE9F743174D01462B680446164898470A
:10E200000023164E164FDFF85C808DF807300DF1B5
:10E2100007013046FDF780FC814648B1E2072B68D4
:10E220009DF8071010D5404698474846FDF798FDE1
:10E230009DF8073064080133DBB20F2B8DF80730EF
:10E24000E5D903B0BDE8F083384698474846FDF766
:10E2500065FDEDE79000002009A50108A9DF000891
:10E2600036A501081FA5010838B504460320FFF7AD
:10E2700031FF0420FFF72EFF0520FFF72BFF0620BC
:10E28000FFF728FF0720FFF725FF2046FFF780FE56
:10E290000546FDF73BFD48B15023294A0121937102
:10E2A0000323063253702846FDF7B8FDE01CFFF744
:10E2B0006FFE0546FDF72AFD48B15023204A012193
:10E2C00013720423083253702846FDF7A7FDA01DE2
:10E2D000FFF75EFE0546FDF719FD48B15023184AC9
:10E2E0000121937205230A3253702846FDF796FDEB
:10E2F00004F10900FFF74CFE0546FDF707FD48B1A4
:10E3000050230F4A0121137306230C325370284601
:10E31000FDF784FD04F10C00FFF73AFE0446FDF71B
:10E32000F5FC58B15023064A204693730723D37354
:10E330000121BDE838400E32FDF770BD38BD00BF89
:10E34000784E00200738C0B205289ABF014B185CF0
:10E35000082070478BA4010806289ABF014B185C5F
:10E360000020704791A40108052804D90628034815
:10E3700018BF002070470248704700BF90D00300CC
:10E3800048E80100052810B5044604D94FF49C71F3
:10E390000348F5F7D5FA034B13F9240010BD00BF6D
:10E3A000CCA4010898A40108142808B506DD0E487D
:10E3B00040F23D11F5F7C4FA062008BD06280ADD33
:10E3C00008280ADD0A280ADD0C280ADD0E28CCBF41
:10E3D00000200120F1E70520EFE70420EDE703200E
:10E3E000EBE70220E9E700BFCCA4010808B50F283D
:10E3F0000DD8DFE800F0181818081A1A1A0A0A0CC3
:10E400000C0C0C0C0C0A732008BD0020FCE740F239
:10E410006F110748F5F794FA064B074A4FF4B871A5
:10E42000034805F0D3FA3320EEE7DE20ECE700BF27
:10E43000CCA40108B6760108B0A4010800000000D1
:10E440002DE9F04F8DB01E46169F434B81469F42EB
:10E450008A46934608D0414B9F4203D0A6214048AC
:10E46000F5F76EFA002100E001213E4D0B91EB6AB9
:10E470009847EB6850469847B9F1010F4FF00004F8
:10E480000A95DFF8EC800B9933D108230A22CDE9F5
:10E490000132AB6932461D4602204B46CDE9089950
:10E4A000CDE90644CDE9044403940094A8472146ED
:10E4B000FF20F8F7C9FF504604F06AFE04F050FA56
:10E4C00023A3D3E9002304F0CDFBD8F80030CDE935
:10E4D00000013A463146244898470820F8F7AAFF39
:10E4E000342139200A9B1B6C0A930DB0BDE8F04F14
:10E4F00018474FF47A634FF00109CDE90743082329
:10E50000CDE901930A9B2246DB69CDE905441D460E
:10E51000CDE903490B46009659460220A8474946D3
:10E52000FF20F8F791FF5046CDF808B004F030FE18
:10E5300004F016FA06A3D3E9002304F093FBD8F8FD
:10E540000030CDE900013A46314608489847C4E713
:10E550000000000080842E4190D0030048E80100B4
:10E5600094A50108EC850108CEA5010802A60108C2
:10E57000900000202DE9F7430546104614460F464B
:10E580009946FFF7F1FE80462046FFF7E5FEC6B24A
:10E590001EB9C9210C48F5F7D3F995B94846FFF7DC
:10E5A000F1FE0246334639462846CDF80080FFF793
:10E5B00047FF2146054B06481B6803B0BDE8F04302
:10E5C00018470022EEE700BF94A501089000002044
:10E5D00087A501080068704782B0034668B16A46A3
:10E5E0005968006803C25A1E0DF10701073311F87C
:10E5F000010902F8010F9A42F9D102B070470FB435
:10E6000004B0704730B585B06D4685E80F00104CFA
:10E6100095E80F0084E80F0004F1100208A903C96F
:10E6200082E803000BB90B4BE360A3680BB9094BFD
:10E63000A36063680BB1236833B9A36806489847A1
:10E64000064B6360064B23600123237605B030BD83
:10E65000944A0020FFE50008A1A60108E13B01085B
:10E66000D13B01082DE9F041194E8046337E0D461D
:10E670002BB96A21174B184A184805F0A7F9DE296B
:10E6800003D9174B144A6B21F6E73368602098478B
:10E69000044680B16022002105F0E0FAB8F1000FD5
:10E6A00012D08DB1336828469847074630B92046C6
:10E6B000736898473C462046BDE8F0812A464146AB
:10E6C00005F0A4FA2577A76400236370F3E700BF81
:10E6D000944A002041A6010841A901084EA601085C
:10E6E00093A6010870B50B4C0546237E2BB90A4B47
:10E6F0000A4A86210A4805F069F950B1806C18B1C0
:10E70000636898470023AB6463682846BDE870409F
:10E71000184770BD944A002041A6010853A901087A
:10E720004EA601082DE9F0431746B34A91B0137E77
:10E7300005460C4690462BB99E21B04BB04AB148D5
:10E7400005F044F9032F04D80026304611B0BDE887
:10E75000F0830178437843EA411323700378022B56
:10E7600001D0042B68D10023042F8DF81630EBD094
:10E770006B6863706B681B0AA370EB88E370EB79BE
:10E7800023716B68CDF812309DF81630002B40F0E5
:10E79000FF80052FD8D02A7AC2F3400302F001018E
:10E7A0009B0143EAC11343EA1213C2F3800243EA16
:10E7B0004213062663712A7A1209731C9F42C3DD35
:10E7C0006989DBB2A15569890236090AE1546B896E
:10E7D000069352B106EB02094F45B5DBA01905F1CE
:10E7E0000C0105F013FA5FFA89F62B7F002B00F07D
:10E7F000EF80BE42A8D26A7F06F101095FFA89F96B
:10E80000A255D8F81430002A40F0E0800433029377
:10E81000AB6C02A903932B7F04EB0900ADF8103019
:10E8200000F07FFB4844C6B2B74280F0D180764BFF
:10E83000734A40F2571182E7032B01D0052B01D117
:10E84000012391E7C3BB082F7FF67EAF5669601C9A
:10E85000324652F8343FC4F8013053684360FFF742
:10E86000BBFE102F7FF670AF324652F83C3F04F1EA
:10E870000900C4F8093053684360FFF7ADFE122F5A
:10E880007FF662AFB6F8443002A96374B6F844303C
:10E8900001A81B0AA37413232436CDE90264ADF842
:10E8A000103000F0EAFA162F7FF64EAF019B1726C4
:10E8B000C4F813306B6448E7012B7FF445AF43681D
:10E8C000637043681B0AA370C388E3708368237175
:10E8D00083681B0A63714389A371C368E371C368CA
:10E8E0001B0A2372C3896372C37BA372037C03F088
:10E8F0007002C3F303031343E372437C237390F862
:10E900002130002B42D0034633F8122F1C26A4F8E6
:10E910000D209B78E373034633F8152F22829B78F2
:10E92000A374034633F8182FA4F813209B7863755B
:10E93000034633F81B2FE2829B78237635F81E3F7F
:10E94000A4F81930AB78E376D8F8143002A9243350
:10E9500001A8CDE90234ADF8106000F08EFA019BF9
:10E9600002A9A351D8F81430043624330293013499
:10E97000731E07A80394ADF8103000F096FABDF8A6
:10E98000102007A9204605F041F9DEE60D26DBE759
:10E990002B78032B01D0052B15D1052F3FF4D4AED6
:10E9A0002A7AC2F3400302F001019B0143EAC1133A
:10E9B00043EA1213C2F3800143EA4113C2F3C002D7
:10E9C00043EA0213F5E600220526F6E614331EE7B5
:10E9D000F31C9F427FF7B8AED8F8143002A9043375
:10E9E00001A8CDE90234ADF8106000F002FA019BF5
:10E9F000A3510436F6B2A8E6944A002041A60108C5
:10EA000068A901084EA601084ABD01082DE9F04F8A
:10EA1000DFF8A09295B099F8188006460F46924606
:10EA20004D46B8F1000F06D1944B954A40F2731150
:10EA3000944804F0CBFF022922D9D9F80030602095
:10EA40009847044638B9D9F80C308F489847204683
:10EA500015B0BDE8F08F6022002105F0FFF8337893
:10EA60005B0923703278072B02F00302627009D130
:10EA7000D9F80C3085489847D9F804302046984793
:10EA80000024E4E7052B00F2A781DFE813F075010D
:10EA9000BC000600060006000600701CFFF79AFD89
:10EAA00001466060BAF1000F08D0504506D0D9F891
:10EAB0000C305246764898476B68DFE7F079B279B8
:10EAC00096F805A042EA00226869A7F1040904301B
:10EAD000042B6281CDE90606CDF82210ADF8209016
:10EAE00029694FEADA1BCAF3401ECAF3001C0AF078
:10EAF0000F0001D0022B31D100238DF82630237A6C
:10EB00004FEA9A1A6BF300036AF341036EF3820330
:10EB10006CF3C30360F30713096823720B0C89B20B
:10EB2000914284BF01339BB202EB034206EB090022
:10EB30000A92FFF74FFD06A9606401A800F059F999
:10EB4000019B626C93421AD052485349EE68B8F167
:10EB5000000F18BF01465148B047ADE701238DF8BB
:10EB60002630237A49686BF300036EF382036CF35B
:10EB7000C30360F3071323724FF00008CEE794F845
:10EB8000088006F108014FEA1818424604F10C000B
:10EB900005F03CF808F10C039F4230D908F1080257
:10EBA000B25C08F10D039F42627704D100233C4818
:10EBB0002377EB684AE708F10908A9EB0800C0B21F
:10EBC00020776B696AB90433464406930796ADF81B
:10EBD00020002B689847A06428B9EB683148984713
:10EBE0006AE71433F0E706A900F09BF900283FF725
:10EBF0002EAFEB682C4898476B68A06CEFE70023BA
:10EC00002377A36423E7112F1BD1002384F821303D
:10EC10006B691FFA87F824330693731C079308F176
:10EC2000FF33ADF82030337806A90DF12D008DF8B3
:10EC30002C3000F058F900280BAE07DCEB681B48BD
:10EC4000CDE7212F40F09A800123DFE7381F3044C1
:10EC5000FFF7C0FC6B6960642433A8F1040806A9BF
:10EC600001A8CDE90636ADF8208000F006F9636C06
:10EC7000019A9A4220D0EB680D48B0E741A60108FE
:10EC80007EA901084EA60108D7A60108EFA6010833
:10EC90001DA70108A77B0108CEA6010857A70108F8
:10ECA0009CA70108D0A7010802A8010878A80108BC
:10ECB0009CA80108944A00209DF82F109DF82E3042
:10ECC000090441EA03219DF82D300DF13300194369
:10ECD00061609DF832309DF831201B0443EA022325
:10ECE0009DF830201343A360FFF774FCE0609DF8AB
:10ECF0003700227CC60966F3C712061166F30612B6
:10ED000060F3030222749DF83820627494F8212085
:10ED100002B3BDF8392062829DF83B20BDF83C006B
:10ED200022759DF83E20A4F81500E275BDF83F203D
:10ED300022839DF84120A276BDF84220A4F81B2032
:10ED40009DF844206277BDF84520E2839DF8472076
:10ED500084F820206A69049302F12400B2F8443058
:10ED6000CDE9020102AA04F1320104F12200ADF85A
:10ED7000143000F038F96AE6172F02D0EB68184813
:10ED80002DE706F11300FFF725FCD9F81430606475
:10ED90002433CDE90636132306A901A8ADF82030A7
:10EDA00000F06BF8636C019A9A4203D0D9F80C30EA
:10EDB0000C4814E7324652F8013F6360536832460C
:10EDC000A36052F8093FE36053682361B27C737C0F
:10EDD00043EA0223A3823AE6D9F80C300248FEE661
:10EDE00028A80108D1A8010807A901080022FFF7F7
:10EDF0000DBE70B51025CEB00C4606462A46002141
:10EE0000684604F02BFF49238DF80030A37B62890C
:10EE10008DF80530D4F80A30ADF8062023FA05F253
:10EE20001B0E8DF808208DF80930228A2369ADF871
:10EE30000A2023FA05F21B0E8DF80D30238908A84D
:10EE40008DF80F308DF80C2000F0C8FC216808A860
:10EE500000F0D4FC2A46694608A800F0D5FC2289B7
:10EE6000616808A800F0D0FC08A90DEB050000F0CF
:10EE700032FD049B33604EB070BD30B50C46CBB054
:10EE8000054604A800F0AAFC216804A800F0B6FC1E
:10EE90002289616804A800F0B7FC04A9684600F064
:10EEA0001AFD009B2B604BB030BD70B50C89BEB015
:10EEB00006460D46A4B114F00F0411D101AA102189
:10EEC000286800F0F1F82889A04201DC3EB070BD4E
:10EED00068683119204401AA00F0D4FA1034F2E72E
:10EEE0004FF0FF30F2E770B50C89BEB006460D4614
:10EEF000A4B114F00F0411D101AA1021286800F068
:10EF0000D3F82889A04201DC3EB070BD6868311991
:10EF1000204401AA00F042F91034F2E74FF0FF302C
:10EF2000F2E72DE9F0430B89C7B080460D46002B70
:10EF300056D00124102203F00F0900211B0901A85B
:10EF40005F1C04F08BFEAB7B6A898DF80930D5F825
:10EF50000A30ADF80A201A0C1B0E8DF80C208DF823
:10EF60000D302A8A2B696E68ADF80E201A0C1B0E24
:10EF70008DF804408DF810208DF81130013EBC4210
:10EF800003DD288947B0BDE8F08309AA102128686D
:10EF90008DF8134000F088F809AA05A901A800F02F
:10EFA000FDF8BC4211DBB9F1000F14BF4B46102332
:10EFB0003046424643440DF1140C934207D80134C5
:10EFC000A4B208F110081036D9E71023F0E710F8C2
:10EFD00001EF1CF8011B81EA0E0102F8011BECE7AE
:10EFE0004FF0FF30CEE770B5C2B0144606460D466E
:10EFF000F122002105A804F031FE0023CDE90333FE
:10F00000636810218DF805301A0A1B0C8DF8073043
:10F0100023898DF80620ADF80830638905AA8DF89C
:10F020000A30A38920688DF80B301B0A8DF80C304C
:10F0300001238DF8043000F037F805AA314601A805
:10F0400000F0ACF8022305AA102120688DF80430E6
:10F0500000F02AF805AA294601A800F09FF842B05E
:10F0600070BD0A680368534003604A6843685340B0
:10F0700043608A68836853408360CA68C3685340AA
:10F08000C36070470B6810B5146863400360546830
:10F090004B686340436094688B6863408360CB68CF
:10F0A000D2685340C36010BDA1F11003DBB2102B36
:10F0B0002DE9F0470C46154608D84FF0010909FA2A
:10F0C00003F303F0013323F080732BB90023FF20F7
:10F0D00085F8F030BDE8F0870A460146284604F07E
:10F0E00095FD04F11C0E4FEA8E0E5FFA8EFE4FEA7C
:10F0F0001E13013B85F8F03023462749B3FBF4F299
:10F1000004FB1232E81812F0FF0210F804AC10F8F9
:10F1100003CC10F8027C10F8016C32D111F80C808D
:10F120004FEAD91289EA080811F807C08F5D11F873
:10F130000A604FEA420A5244C24602EBC20282EA25
:10F1400049025FFA82F91A1BD2B215F802802A44EA
:10F150008AEA080A05F803A092F8018004338CEAD1
:10F16000080C80F801C092F802C0DBB287EA0C07F5
:10F170008770D2789E4586EA0206C670BED8002007
:10F18000A8E7182CDFD9102A01BF11F80AA011F83E
:10F190000CC0CF5D8E5DD6E799B001082DE9F04F28
:10F1A00092F8F03097B00D910B92002B00F0628135
:10F1B00001460EA8FFF766FF0127AF4CAF4DB04EDA
:10F1C0000B9B03EB07130C930B9B93F8F030BB42A4
:10F1D00059D8A94B9DF838209DF83D109A5C595C90
:10F1E0008DF838209DF83C209A5C8DF83C209DF8E5
:10F1F00040209A5C8DF840209DF844209A5C8DF860
:10F2000044209DF839208DF839109DF841109A5C02
:10F21000595C8DF83D109DF845108DF84520595CDE
:10F220009DF83A208DF841109DF842109A5C595C87
:10F230008DF842208DF83A109DF846109DF83E203A
:10F24000595C9A5C8DF83E109DF843108DF846206D
:10F25000595C9DF847208DF847109DF83F100D9898
:10F26000595C8DF843109DF83B10595C9B5C8DF800
:10F270003F100C9A0EA98DF83B30FFF703FF0020DA
:10F2800017B0BDE8F08F0DF1580C0EAB0FCB0CE9A9
:10F290000F009DF849309DF848E002939DF84A30F0
:10F2A0009DF84D9001939DF84B309DF84C100393C1
:10F2B0009DF84E309DF8560004939DF84F3005930D
:10F2C0009DF8503006939DF8513007939DF85330C8
:10F2D00008939DF8543009939DF855300A939DF892
:10F2E00052809DF857C015F80E2016F809B014F892
:10F2F00008A014F80C3082EA0B028AEA02025A4093
:10F300008DF8382014F80E2015F809B053408BEA18
:10F31000030316F808B015F8088083EA0B038DF88C
:10F32000393014F809305A4082EA080216F80C8085
:10F330008AEA030A16F80E3082EA08028DF83A20AB
:10F3400083EA0A0A079A15F80C3015F8018016F8B6
:10F3500002E08AEA030A039B14F800C0E35C88EA2F
:10F360000E028CEA02025A408DF83C20625C8DF855
:10F370003BA083EA0208079B15F803E08EEA080326
:10F3800016F800E083EA0E038DF83D30079BE35C3E
:10F39000285C5A408CEA030C735C4240039883EA71
:10F3A0000C0C039B305CEB5C42408CEA030C8DF848
:10F3B0003E20019B069A0A98E15C305C059BAA5CA2
:10F3C000E35C42404A405A408DF84020069A0A9831
:10F3D000A25C285C5340434001988DF83FC0305CEC
:10F3E00043408DF841300A9B0198E35C285C5A4009
:10F3F000424005985940305C069B42408DF84220BF
:10F40000F35C059A4B40A95C02984B408DF8433061
:10F41000049B305CE15C089BE25C099BEB5C434035
:10F420004B4053408DF84430099B0298E35C285CC4
:10F430005A4042400498305C42408DF84520029A80
:10F440000498A25C285C5340434008984A40305CD2
:10F4500043408DF84630099B0EA8F15C089B514053
:10F46000EB5C59408DF847100C99FFF7FAFD7B1CB7
:10F47000DFB2A5E6FF2003E799B0010899A90108CA
:10F4800099AA01082DE9F04F924692F8F02095B024
:10F490000B91002A00F09B810AEB021201460CA896
:10F4A000FFF7F0FD324C9DF830309DF83920E35CD9
:10F4B000A25C8DF830309DF834302E4DE35C2E4E3A
:10F4C0008DF834309DF83830E35C8DF838309DF895
:10F4D0003C30E35C8DF83C309DF83D308DF83D20AC
:10F4E0009DF83520E35CA25C8DF839209DF8312031
:10F4F0008DF83130A25C9DF832308DF835209DF8C2
:10F500003A20E35CA25C8DF83A308DF832209DF809
:10F510003E209DF83630A25CE35C8DF836209DF8E5
:10F5200037208DF83E30A25C9DF833308DF83320C3
:10F530009DF83B20E35CA25C8DF837209DF83F20CE
:10F540008DF83F309AF8F030A25C013BDBB28DF8C9
:10F550003B200AEB0318D0450CAF0FD10B98424665
:10F560003946FFF78FFD002015B0BDE8F08F00BFD2
:10F5700099AF010899AE010899AC01084146384697
:10F58000FFF76FFD97E80F0014AF07E90F009DF834
:10F5900046309DF844C001939DF847309DF8457072
:10F5A00002939DF848309DF8419003939DF84930AF
:10F5B000884A04939DF84A30A8F1100805939DF8F5
:10F5C0004B3006939DF84C3007939DF84D300893CF
:10F5D0009DF84E3009939DF84F300A939DF84030C6
:10F5E00018469DF84230295C009316F809309DF8C2
:10F5F00043E05940009BD35C5940774B13F80EB061
:10F6000081EA0B01615C13F800B08DF8301015F839
:10F6100009108BEA010B0099715C8BEA010112F869
:10F620000EB081EA0B01615C12F800B08DF8351064
:10F6300013F8091012F809908BEA010B0099695C24
:10F640008BEA010116F80EB081EA0B01615C8DF8BE
:10F650003A10315C009881EA090113F8009081EAC0
:10F66000090115F80E9015F80CE081EA0901615CBA
:10F670008DF83F10F15D02988EEA010E0199515C00
:10F680008EEA010113F800E081EA0E01615C13F8D3
:10F690000CE08DF83410E95D8EEA010E0199715C81
:10F6A0008EEA010112F800E081EA0E01615C12F8B5
:10F6B0000CE08DF83910D95DD75D8EEA010E019905
:10F6C000695C8EEA010116F800E0019881EA0E01FA
:10F6D000615C8DF83E1016F80C1079401F5C0298A2
:10F6E00079402F5C7940615C8DF833100399685C38
:10F6F0000499715C48400599515C41400698185C3A
:10F700004140615C8DF838100399585C0499695C3C
:10F7100048400599715C41400698105C4140615C2D
:10F720008DF83D100399505C0499595C4840059947
:10F73000695C41400698305C4140615C04988DF8FA
:10F7400032100399105C715C41400598185C484088
:10F750000699695C4840215C08988DF83710079934
:10F76000305C695C41400998105C41400A98185C23
:10F770004140615C08988DF83C100799285C595C01
:10F7800041400998305C41400A98105C4140615CFE
:10F7900008988DF831100799185C515C4140099820
:10F7A000285C41400A98305C4140615C08988DF8C3
:10F7B00036100799125C715C4A4009995B5C5340B2
:10F7C0000A9AAA5C5340E35C8DF83B30C3E6FF2005
:10F7D000CAE600BF99AD010899AB010810B5102227
:10F7E00004460021F13004F039FA00212046C4F823
:10F7F0001411F022BDE8104004F030BA0B46024666
:10F8000010211846FFF750BC2DE9FF470446D0F8F9
:10F8100014018846154604F2011910B3C0F110070F
:10F8200097423E4628BF16464844324604F0EEF959
:10F83000D4F8143133440F2BC4F814311CD9AF421F
:10F840001AD204F1F10319461A78187C424003F8E1
:10F85000012B4B45F8D122460846FFF79FFCB044E8
:10F86000AD1B0DF1100A102D09D82A464146484615
:10F8700004F0CCF9C4F8145104B0BDE8F08704F1E9
:10F88000F1031E4608F1FF311A7811F8010F4240CA
:10F8900003F8012B4B45F7D16A4633461746944689
:10F8A000186859680833ACE803004B456246F6D146
:10F8B000224639463846FFF771FC33463A4603CABA
:10F8C000524518605960174603F10803F6D108F154
:10F8D0001008103DC7E7F0B50C4689B01022002192
:10F8E0000546684604F0BAF9224669466846FFF7BD
:10F8F00055FC9DF900306A46002B4FF000013EDABE
:10F90000537810780131DB0943EA40030F2902F8EC
:10F91000013BF5D19DF80F305B0083F087038DF834
:10F920000F30D4F81431102B37D1694604F201138B
:10F9300004F211101A7811F8016B724003F8012BD0
:10F940009842F7D104F1F102134604F2011711783D
:10F95000107C414002F8011B9742F8D104AA94465A
:10F96000164618685968083303C6BB423246F7D1B9
:10F97000224629466046FFF711FC09B0F0BD5378D6
:10F9800010780131DB0943EA40030F2902F8013BFB
:10F99000F5D19DF80F305B00C1E79DF90020694665
:10F9A000002A4FF0000028DA4A780E780130D20998
:10F9B00042EA46020F2801F8012BF5D19DF80F20ED
:10F9C000520082F0870280218DF80F20E21882F821
:10F9D0000111002104F2011201330F2B1BD9C4F8CD
:10F9E00014316B4604F21110117813F8016B714059
:10F9F00002F8011B9042F7D1A4E74A780E78013053
:10FA0000D20942EA46020F2801F8012BF5D19DF8F0
:10FA10000F205200D7E7D154DEE710B1012101F0E9
:10FA200081BE704708B1F7F7DBBA7047806870474E
:10FA3000406870474368012B08D1D0E904329342F3
:10FA400004D01878003018BF01207047002070479C
:10FA50004B6870B5042B04460E464FF0000304D0EB
:10FA6000C0E900338360204670BDD1E90425AD1A9A
:10FA7000C0E9003383602846FFF7D4FFC4E90000E3
:10FA80000544A560D6E9041305460A46934204D00E
:10FA900012F8016B05F8016BF8E75B1A1844606017
:10FAA000E1E742680346022A06D1D3E904031B1AA0
:10FAB000032B01D906F0A4BD002070474368032B37
:10FAC00006D1D0E904329A4208BF00231846704795
:10FAD0000023FBE7037870B581680446B3B1284A78
:10FAE0002848F7F7F1F96368022B12D12046FFF797
:10FAF000D8FF01462448F7F7E7F9E1680B78002BB7
:10FB00003CD02248BDE87040F7F7DEB9204A2148D2
:10FB1000E7E7032B05D12046FFF7D0FF01461E483B
:10FB2000E9E7042B0ED100251C4ED4E90431C91A93
:10FB30008D4205D2595D3046F7F7C6F90135F4E735
:10FB40001748D8E7012B08D12046FFF773FF154966
:10FB5000154B002808BF1946E1E700250F4ED4E9F0
:10FB600004239B1A9D4205D2515D3046F7F7ACF94C
:10FB70000135F4E70D48F7F7A7F9BEE70C48C1E7F0
:10FB80001F680108FBB101080FB2010831B201087A
:10FB9000BE6F010805B2010849780108D79B01082A
:10FBA00019B20108F6B10108B67601081FB20108C2
:10FBB000BD6F0108B1F5705F2DE9F84304460F46AB
:10FBC00002D9164801F084FD056883685B1B9942E1
:10FBD00018D9D0F804900846FFF724FF06460346DC
:10FBE000A9EB0508A94504D015F8012B03F8012B52
:10FBF000F8E72068FFF711FF06EB080326603E4494
:10FC00006360A66025683DB92846C4E90155FFF741
:10FC100004FF2846BDE8F8830120FBE799B10108FD
:10FC20002DE9F0410368561A904682680446D21ABC
:10FC300096420D4614D93046FFF7F4FE07460346B8
:10FC4000A84504D015F8012B03F8012BF8E720682C
:10FC50003E44FFF7E2FEC4E901662760BDE8F0819B
:10FC60004768481EFF1ABE4211D81A469D19A91AA4
:10FC7000002904DD10F8011F02F8011BF7E7002E30
:10FC8000A8BF9B1962689A42E8D06360E6E73D44EA
:10FC90001F44FA1A002A04DD10F8012F03F8012B83
:10FCA000F7E7636828461A46804504D010F8011B20
:10FCB00002F8011BF8E7A8EB05084344E5E708B59F
:10FCC00009C81B1AC3F57050884202D2104601F0D1
:10FCD000FFFC994238BF1946C81805D2B0F5705FCD
:10FCE00028BF4FF4705008BD4FF47050FBE7000080
:10FCF0002DE9F8430C46591C204615461E46FFF7D1
:10FD000059FF804678B14FF00003AA1929462046D2
:10FD1000FFF786FFD4E901639E4207D000233370CA
:10FD20006368013363604046BDE8F883104A0121EF
:10FD30002046FFF7C4FF27688146FFF773FE0022C5
:10FD4000F31BC25405463A46411EB24202F101037A
:10FD500004D010781A4601F8010FF6E7DB1BEE1805
:10FD60003846FFF75AFEC4E900564D44A560DAE76D
:10FD7000B4B101081346426810B5032A06D1BDE8A4
:10FD800010400A4600F11001FFF7B2BF8168024837
:10FD9000F7F79AF8002010BD38B201082DE9F041BC
:10FDA000D0E900239E1AB14204460D462ED9891B84
:10FDB0000AD08268D21A914208D80022194403F866
:10FDC000012B8B42FBD16360BDE8F081124AFFF743
:10FDD00076FF8046FFF726FE0023074606440544CB
:10FDE00006F8013BB542FBD1D4E900303A468342E4
:10FDF00004D013F8011B02F8011BF8E72068FFF795
:10FE00000CFEC4E900754744A760DDE7DCD2154469
:10FE10009D4218BF4560D7E71CB3010870B50C467A
:10FE2000012120461646FFF7C5FE054628B10121EF
:10FE30002046FFF7B3FF23681E70284670BD000000
:10FE4000426808B5012A06D1BDE808400A4600F11B
:10FE50001001FFF7E3BF81680248F7F735F800208B
:10FE600008BD00BFABB2010810B50C1A134605D08F
:10FE700001462246184603F0D7FE0346181910BD66
:10FE80002DE9F0418368A2EB010817460268044699
:10FE90009B1A98450D4614D94046FFF7C3FD064608
:10FEA0000346AF4204D015F8012B03F8012BF8E705
:10FEB0002068FFF7B2FD26604644C4E90166BDE84C
:10FEC000F0814668B61AB04508D839462846FFF78B
:10FED000CBFF63688342F2D06060F0E70E443146A6
:10FEE0002846FFF7C1FF636832461946974204D09F
:10FEF00012F8010B01F8010BF8E7BE1B1E44666007
:10FF0000DDE7000070B5D0E9043100F110060446C9
:10FF1000C91A3046FFF74EFE054640B1D4E9071234
:10FF2000914206D1A1680648F6F7CEFF0025284683
:10FF300070BD4FF000033046FFF7A2FFF7E700BFA8
:10FF4000CEB101082DE9F0418368A2EB0108164605
:10FF5000026804469B1A98450F4614D94046FFF79D
:10FF600061FD05460346BE4204D017F8012B03F895
:10FF7000012BF8E72068FFF750FD25604544C4E9F0
:10FF80000155BDE8F0814568AD1AA84508D831464D
:10FF90003846FFF769FF63688342F2D06060F0E79C
:10FFA0000D4429463846FFF75FFF63682A46194625
:10FFB000964204D012F8010B01F8010BF8E7751B0B
:10FFC0001D446560DDE737B50D4601A8114606F012
:10FFD0002BFB04212846FFF7EDFD044630B14FF01E
:10FFE000000302AA01A92846FFF7ACFF204603B090
:10FFF00030BDFFF7E8BF0000426808B5022A06D10D
:020000040801F1
:10000000BDE808400A4600F11001FFF7DCBF816837
:100010000248F6F759FF002008BD00BFE3B201080F
:10002000FFF7EABFF7B50E4604461046154604F042
:10003000FFFC00237268C4E90033013AA360032A7D
:1000400012D8DFE802F0022A393F2C49284604F092
:10005000DDFC20B12A49284604F0D8FC38B9012239
:1000600021463046FFF7DAFE204603B0F0BD2549B1
:10007000284604F0CBFC20B12349284604F0C6FCF6
:1000800008B90022ECE7002201A92846019204F0F9
:10009000E3FD021C18BF0122E2E7002201A9284665
:1000A000019304F0D9FD019B0246AB42DCD021460E
:1000B0003046FFF788FFD7E72A462146304600F052
:1000C00025F8D1E710F00106CED147083946204681
:1000D000FFF770FD0028C7D039462046FFF75EFEC7
:1000E000B742C1D0022105EB460006F072FA0028A3
:1000F000BADB236898550136F2E700BFF6B1010874
:10010000A9B10108B6760108AEB10108F0B543689F
:1001100085B0032B0D46164615D0014601A8FFF702
:1001200081FFDDE901128A420BD04FF0000328461F
:10013000FFF7A6FE01240198FFF76FFC204605B0EB
:10014000F0BD0024F7E7104604F072FC471C394666
:100150002846FFF72FFD04460028EFD04FF000039C
:10016000F21931462846FFF75BFDE7E70A4600F142
:100170001001FFF7CBBFF8B50D46194628461646C5
:100180001F46FFF717FD044630B14FF00003F21988
:1001900031462846FFF7D6FE2046F8BD1346426892
:1001A00010B5042A06D1BDE810400A4600F110013E
:1001B000FFF7E1BF81680248F6F786FE002010BD18
:1001C00072B2010810B10C2101F0ACBA704710B145
:1001D000012101F0A7BA704710B5044638B1EFF716
:1001E000EBFF2046BDE81040282101F09BBA10BD6E
:1001F00070B50446006AFFF7E5FFD4E90556AE4244
:1002000004D02846EFF7D8FF2835F8E7656935B1FF
:100210002846EFF7D1FF2821284601F083FA20462F
:1002200070BD0000F8B5054600242826074FD5E923
:1002300005031B1ADB107B439C4205D206FB04001E
:10024000FFF760FE0134F2E7F8BD00BFCDCCCCCCA7
:10025000F8B504462248F6F737FE2248F6F734FE92
:10026000D4E90531994218D0C91A1F4EC9107143FB
:100270001E48F6F729FE00252827D4E905031B1A96
:10028000DB1073439D4205D207FB0500FFF722FCFC
:100290000135F2E71648F6F717FED4E90831154E96
:1002A000C91A891071431448F6F70EFE00250C2771
:1002B000D4E908031B1A9B1073439D4205D207FB28
:1002C000050000F0F3FE0135F2E70C48F6F7FCFDFF
:1002D0000B48F6F7F9FDBDE8F8400A48F6F7F4BD1B
:1002E000FCB30108386E0108CDCCCCCC06B40108B3
:1002F00018B40108ABAAAAAA51B40108BD6F01083D
:1003000061B40108E46A01082DE9F043002487B0D4
:1003100006466846CDE90044029400F0E5FF6846D1
:1003200001F07AF84FF028082F4F304DD6E9052319
:100330009B1ADB107B439C424ED208FB04F302EB7A
:100340000309D35C002B43D14846FFF76FFB0146FE
:10035000684601F053F84846FFF76AFB042837D88F
:10036000DFE800F03803101A24004846FFF762FB6C
:100370000146684600F0F8FF50BBC1212846F3F75C
:10038000DFFA25E04846FFF78CFB0146684600F09F
:10039000D1FFE8B9C521F1E74846FFF78FFB0146D9
:1003A000684601F02BF898B9C921E7E7494603A848
:1003B000FFF74EFBDDE903126846521A00F0F6FF24
:1003C00018B9CE212846F3F7BBFA0398FFF7FFFED2
:1003D0000134ABE7D221D1E7684601F045F8029835
:1003E00007B0BDE8F08300BFCDCCCCCC51B3010841
:1003F0002DE9F04305460E4600244FF028081A4F19
:100400008DB0D5E905239B1ADB107B439C4224D297
:1004100008FB042931461822684604F023FB4846AD
:10042000FFF704FB182201460DEB020004F01AFB53
:10043000684606F007F9684606F014F906A806F0C3
:1004400001F906A806F00EF9182268460DEB020124
:1004500004F0F6FA18B10134D3E74FF0000948462A
:100460000DB0BDE8F08300BFCDCCCCCC2DE9F04F72
:1004700006460F4600244FF00C09DFF86C808DB063
:10048000D6E908535B1B9B1008FB03F39C4224D264
:1004900018223946684604F0E5FA182209FB04FBE5
:1004A0000DEB020055F80B1004F0DCFA684606F07C
:1004B000C9F8684606F0D6F806A806F0C3F806A8FC
:1004C00006F0D0F8182268460DEB020105EB0B0A86
:1004D00004F0B6FA18B10134D2E74FF0000A5046E2
:1004E0000DB0BDE8F08F00BFABAAAAAA10B51446A4
:1004F000FFF77EFF20B12146BDE81040FFF736BE72
:1005000010BD0000F8B50C46064640F2011200216D
:10051000224803F0A3FB4FF4807221461F4803F0EA
:1005200075FB1E491E48F6F7CFFC1E491B4804F018
:10053000C3FA1C490546002004F0BEFA29460746C6
:100540003046FFF755FFC8B929463046FFF78EFF02
:10055000044600B301681448F6F7B6FCA3683846B1
:10056000984701242046F8BD1048F6F7ADFC104826
:10057000F6F7AAFC3046FFF76BFEF3E73A4629464A
:100580003046FFF7B3FF04460028EDD1394609484D
:10059000F6F79AFCE6E729460748F9E7344C0020CD
:1005A000CA7201087AB401087CB4010891B4010848
:1005B000BD6F0108A5B40108BEB4010810B54FF421
:1005C00080720649044600F0D3FF002805DD20466E
:1005D000BDE810400149FFF795BF10BD344B002026
:1005E00038B514461D46FFF703FF28B12A462146B9
:1005F000BDE83840FFF7BEBB38BD10B51446FFF765
:10060000F7FE20B12146BDE81040FFF7F5BC10BD54
:1006100010B51446FFF7ECFE10B12146FFF710FCB1
:10062000002010BD38B514461D46FFF7E1FE28B185
:100630002A462146BDE83840FFF7B0BD38BD00006E
:100640002DE9F04700248CB0074603A8CDE9034408
:10065000059400F049FE214603A8009400F060FFD5
:100660000146002834D0214603A800F0E2FE40F203
:10067000E7330446009300263546DFF8F4A0009BDC
:10068000B34271D9214603A800F005FF8146002836
:100690006AD1182321460DEB030203A800F08CFE5B
:1006A0000444214603A800F004FF8046B0B121466F
:1006B00002AA03A8CDF8089000F01CFE029A044498
:1006C00006A93846FFF799FF00B101350136D6E794
:1006D0006A4603A800F0B4FE0446CCE7214603A80E
:1006E00000F031FF70B102AA214603A88DF80880FE
:1006F00000F02AFE9DF80820044406A93846FFF7BA
:1007000087FFE1E7214603A800F0EEFE804668B1CE
:1007100002AB01AA214603A800F05FFEDDE9012338
:10072000044406A93846FFF75BFFCDE7214603A83E
:1007300000F0CCFE80B102AB01AA214603A8CDE9AE
:10074000018800F022FE9DF808300444019A06A9B1
:100750003846FFF767FFB7E7039B5046195D01F086
:10076000E001F6F7B1FBB1E728460CB0BDE8F08731
:100770008BB3010808B5FFF73BFE18B1BDE8084090
:10078000FFF758B908BD10B5044608461146FFF7F3
:100790002FFE014620B9C4E90000A060204610BD2C
:1007A0002046FFF755F9F9E708B5FFF721FE18B124
:1007B000BDE80840FFF775B908BD08B5FFF718FE9A
:1007C00018B1BDE80840FFF779B908BD002370B53E
:1007D000D1E90025AD1A0446C0E9003383600E4616
:1007E000284601D0F6F7FCFBC4E900000544A560EB
:1007F000D6E9001305460A46934204D012F8016B6D
:1008000005F8016BF8E75B1A18446060204670BD7C
:1008100038B504460D460B78103000F8103C4B6894
:10082000103140F80C3C51F8083C40F8083C51F8B5
:10083000043C40F8043CFFF7C9FF05F11C0104F13A
:100840001C00FFF7C3FF204638BD00002DE9F84F1C
:10085000D0E90075EC1BA310304C06465C43B4F5A0
:10086000705F8946934602D12D4800F031FF002C7D
:1008700014BF23460123E418A1EB070A19D2B4F5EB
:10088000705F16D8C4B10C206043F6F7A9FB804610
:100890009BE8070008EB0A0383E807000023DA1946
:1008A00091450BD007CA08EB030C8CE807000C330A
:1008B000F5E74FF47054E6E7A046E9E70C22194942
:1008C0004FF000098C464FEA9A034B4323F0404314
:1008D00002FB037E03FB0223434409EB0E02954215
:1008E00007D007CA03EB090A8AE8070009F10C09D7
:1008F000F3E74FF00C09A5EB0E05AD080CFB05F571
:1009000025F0404509FB053509FB04843846FFF70F
:1009100059FCC6E90085B460BDE8F88FABAAAAAA65
:10092000B4B10108ABAAAA2A2DE9FF47044608463C
:100930000D4617461E4604F07BF8172803D981217F
:100940002C48F2F7FDFFD4E9089A2B4AAAEB0908D4
:10095000CDE901574FEAA80555430135B5F5705F5C
:10096000039602D9254800F0B3FEA36AA3EB09035E
:100970009B1053439D4229D90C266E437DB13046CE
:10098000F6F72EFB0746002309EB0302924508D039
:1009900007CA07EB030C8CE807000C33F4E72F467B
:1009A000F1E7206AFFF70EFC07EB08036362124BC6
:1009B00027623744B6105E43B542A76206D9104895
:1009C000F6F782FA8B210B48F2F7BAFFD4E9093225
:1009D000934201AA07D007CA83E807000C33636279
:1009E00004B0BDE8F087194604F12000FFF72EFFA0
:1009F000F6E700BF51B30108ABAAAAAA99B1010852
:100A000036B30108002310B50446C0E90533C0E938
:100A10000733C0E90933064B8021036100F0A1FDD3
:100A20002046044B044A0549FFF77EFF204610BDCF
:100A3000B44A0020790A0108E1B40108EDB40108C4
:100A400010B5084C2368DB0709D40748FFF7DAFF25
:100A50000123064A06490448236001F0C8FC024805
:100A600010BD00BFB04A0020384D0020000000201B
:100A7000F1010108FFF7E4BF08B5FFF7E1FFBDE8AA
:100A80000840FFF7E5BB0022C0E90022826010B5F4
:100A90000C6804600A6042684C6844604A6082687E
:100AA0008C6884608A6010BDF8B50F46154600F169
:100AB0001004A4F110039F4205F128061AD014F87F
:100AC000103C214606F8283C54F80C3C05F1100077
:100AD0006B6054F8083CAB6054F8043CEB60FFF7E3
:100AE000D2FF04F10C0105F11C00FFF7CCFF283404
:100AF0003546DEE72846F8BD2DE9F84FD0E9006716
:100B0000BC1BE310224C05465C43B4F5705F88467D
:100B1000924602D11F4800F0DBFD002C14BF234693
:100B20000123E418A1EB060B22D2B4F5705F1FD8A5
:100B30000CB328206043F6F753FA8146514609EB7F
:100B40000B00FFF765FE41464A463046FFF7ACFF13
:100B5000394600F128024046FFF7A6FFB04682461C
:100B6000B8450AD04046EFF727FB08F12808F7E719
:100B70004FF47054DDE7A146E0E73046FFF72CFB69
:100B8000282303FB0494C5E9009AAC60BDE8F88F04
:100B9000CDCCCCCCB4B101082DE9F04FD0E905564D
:100BA000044688463B4F8BB0AE421BD02946684670
:100BB000FFF72EFE6846FEF739FF81464046FEF7F6
:100BC00035FF0146484605F073FD30B14046FEF75B
:100BD0002DFF01463846F6F777F96846EFF7ECFA4D
:100BE0002835E1E7D4E905AB2B4AABEB0A094FEA1C
:100BF000E90555430135B5F5705F02D9274800F086
:100C000067FDE369A3EB0A03DB1053439D422CD934
:100C100028266E4395B13046F6F7E2F90746594665
:100C200050463A46FFF740FFD4E905ABD34507D01D
:100C30005046EFF7C1FA0AF1280AF7E72F46EEE728
:100C40006069FFF7C9FA07EB0903A361124B6761FB
:100C50003744F6105E43B542E76106D91048F6F70F
:100C600033F976210F48F2F76BFED4E90603984278
:100C700008D04146FFF7CCFDA3692833A3610BB030
:100C8000BDE8F08F0146424604F11400FFF734FF3F
:100C9000F5E700BFABB30108CDCCCCCC99B10108CE
:100CA000DDB3010851B3010808B50848F6F70CF99F
:100CB000FFF7C6FEFFF7B6FA0548F6F705F9FFF7A6
:100CC000BFFEBDE80840FFF7C3BA00BFBFB60108CA
:100CD000D7B6010873B505464FF40070F6F780F9F2
:100CE000044618B928211848F2F72AFE4FF400727A
:100CF0000021204602F0B2FF4FF400722146284640
:100D0000FFF702FB114D124E014601901148F6F714
:100D1000DBF87368294604226868984704226868EB
:100D20000DEB020173681044984768687368019A74
:100D30002146083098470848F6F7C6F82046F6F7E7
:100D400039F902B070BD00BF88B50108744D0020AC
:100D5000684D0020D0B50108EBB501082DE9F74F2B
:100D6000FFF76EFE2E4F06462E48F6F7ADF8B84652
:100D7000DFF8CC90DFF8CCA0F9F7AAFB2A4D386059
:100D80002B68AB46294C002B37D003F56A43603300
:100D9000984232D223782BB92548F6F795F82548A2
:100DA000F6F792F8012330462370FFF707FC41F273
:100DB000883352464FF0FF310020F9F7E1FF0190F0
:100DC000F9F786FB019BC8F8000023B9237813B11B
:100DD0003046FFF7F3FBDAF80030DA0744BFD8F803
:100DE00000202A609B07C7D50023CBF80030D9F834
:100DF0000830002BBED09847BCE7237863B130465B
:100E0000FFF768FF0C48F6F75FF80C48F6F75CF858
:100E1000D9F8083003B19847002323702B60C6E748
:100E2000884D00202FB60108844D00207C4D002005
:100E300044B6010867B601088AB601089CB60108E5
:100E4000684D0020804D002010B5FFF7F9FD0446E5
:100E5000FFF740FF2046FFF7FBF9BDE810400348CD
:100E60000023012202210068F9F7CEBF644D002063
:100E700010B5FFF7E5FD0446FFF72CFF2046BDE85F
:100E80001040FFF7E5B900002DE9F3410024154DAE
:100E9000154E042207468846009469463368686800
:100EA00098472A6800998A4204D01048F6F70CF84F
:100EB000204613E0042268680DEB020110443368F9
:100EC000984701990A48F5F7FFFF019A9045EFD33B
:100ED00068683368394608309847019802B0BDE821
:100EE000F08100BF744D0020684D0020FAB5010864
:100EF00015B6010882B0F0B587B003AC84E80700EE
:100F00000D93049B1BB9F1215648F2F719FD039B81
:100F10001BB9F2215348F2F713FD94E80700524B36
:100F200083E80700514B0DAA92E8030083E8030011
:100F3000FFF786FD06464E4B4E4A4F49FFF7F4FC3D
:100F40004E4B4F4A4F493046FFF7EEFC4E4B4F4A4F
:100F50004F493046FFF7E8FC4FF40070F6F740F8D1
:100F6000044670B14FF40072002102F077FE4FF496
:100F700000712046FFF788FF024660B92046F6F769
:100F800019F84448F5F7A0FF3046FFF74BF94248FF
:100F9000F5F79AFF06E021463046FFF751FB204661
:100FA000F6F708F84FF40070F6F71AF805464FF414
:100FB0000072002102F052FE4FF400712846FFF744
:100FC00063FF0746F8B9F5F7F5FF2846F5F7F2FF96
:100FD0003248F5F779FFFFF733FDFFF77BFE304B23
:100FE000FA22019301232F4900932F480023F9F798
:100FF0004DF890BB4FF486711A4807B0BDE8F04039
:1010000002B0F2F79DBC4FF40070F5F7E9FF04461B
:1010100018B968211348F2F793FC4FF400720021CD
:10102000204602F01BFE4FF4007221463046FFF7C7
:101030006BF908B92046C6E78742FBD10023E15C83
:10104000EA5C9142F6D101339842F8D12046F5F797
:10105000B1FF2846F5F7AEFFC1E707B0BDE8F040A5
:1010600002B0704788B50108684D0020744D00201B
:10107000710E0108F1B40108FDB40108A90C0108C2
:1010800002B501081DB50108490E010825B5010882
:101090003DB5010842B50108D7B6010866B501089B
:1010A000644D00207DB501085D0D010810B50446B2
:1010B00001680748F5F708FF616831B10B7823B183
:1010C0000448BDE81040F5F7FFBE0348F9E700BF4C
:1010D000EFB6010831B20108BD6F010870B508B95B
:1010E000002070BD002346684D1CB5421360F7D840
:1010F00003685C185B5C03F01F03A3F1180103296C
:101100000DD81449194411F8180C0544AE42E7D320
:10111000042819D8DFE800F003070B18120000209C
:1011200013600130DDE7637801201360F9E7B4F85C
:10113000013002205BBA9BB21360F2E7D4F80130B1
:1011400004201BBA1360ECE7D4F801301BBA13601B
:10115000E7E700BFF4B60108F7B51F464368164637
:101160004A1C9A4205460C4617D803685B5C03F09C
:10117000C003402B11D196B101AAFFF7AFFF50B1C8
:10118000019A04446B68A118994206D82968104452
:101190000C4434603A6003B0F0BD0020FBE73046F9
:1011A000F9E72DE9F7439946436817464A1C9A42E6
:1011B00080460D4624D803685B5C03F0C003402BD7
:1011C0001ED1FFB101AAFFF789FF0446A0B1019E1D
:1011D00009F10109B14513D30544D8F80430721957
:1011E0009A420DD8D8F8001032462944384602F009
:1011F0000DFD00233444BB55204603B0BDE8F08309
:101200000024F9E73C46F7E7F0B581B3172A1CD86C
:10121000D3B2A3F11804032C8CBF0024154C8D68A5
:101220009CBFE41814F8184C6F1C4E6804EB070CB4
:10123000B4451CD20E6818438F60E3007055083B1C
:1012400013F1080F0BD1601CF0BDFF2A05D9B2F5D0
:10125000803F34BF19231A23DBE71823D9E78868B6
:101260000D68461C8E6022FA03F62E54E7E7002034
:10127000EAE700BFF4B60108172BF8B50D4616468D
:101280001C4612D8DBB2A3F11802032A8FBF00223A
:10129000144A9B1813F8182CAB68013223441344EA
:1012A0006A6893420BD30020F8BDFF2B05D9B3F534
:1012B000803F34BF19231A23E5E71823E3E72246CA
:1012C0002946FFF7A1FF07460028ECD02868AB6845
:1012D0003146184402F09AFCAA68E0192244AA6038
:1012E000E2E700BFF4B6010818B10023C0E900121C
:1012F00083607047436873B514464A1C9A42064699
:101300000D4602D9002002B070BD03685B5C13F08B
:10131000C00FF7D1002CF5D001AAFFF7DFFE00289F
:10132000F0D03268019B525D12F0E00F18BFDB4332
:101330002360E8E70A1EABBF014601460020D24306
:10134000B8BF2020FFF760BF03685B5C03F0E001DB
:10135000E02907D132B1A3F1F5014B424B411370A3
:101360000120704700207047836810B544685A1CFC
:10137000A24208D2002914BFF524F4240168826037
:101380000120CC5410BD0020FCE7F0B446684F1C8F
:10139000B74208D805686C5C04F0E004402C02D128
:1013A000F0BCFFF7D9BE0020F0BC704713460A46D8
:1013B00001464020FFF760BFF0B446684F1CB742BB
:1013C00008D805686C5C04F0E004602C02D1F0BC25
:1013D000FFF7E7BE0020F0BC7047F0B446684F1C32
:1013E000B74208D805686C5C04F0E004602C02D1B8
:1013F000F0BCFFF7B1BE0020F0BC704770B50546E9
:1014000008460C4603F014FB224603462946BDE875
:1014100070406020FFF730BF836841685A1C8A42E1
:101420003FBF8260BF220168012034BFCA54002040
:1014300070470368585CA0F1BF0358425841704799
:1014400013B5036814465B5C03F0E003A02B07D1DF
:1014500042B101AAFFF742FE019B236002B010BD1A
:101460000020FBE71046F9E7836841685A1C8A426E
:101470003FBF8260FF220168012034BFCA540020B0
:10148000704730B18068013888428CBF002001204D
:1014900070470120704708B50246FFF7F2FF30B9E8
:1014A0001268505CA0F1FF035842584108BD01206A
:1014B000FCE743688B4207D903685B5C13F0C00FFD
:1014C0000CBF0120002070470020704743688B420A
:1014D00008D90368585C00F0E000A0F140035842CE
:1014E000584170470020704743688B4208D9036811
:1014F000585C00F0E000A0F160035842584170478A
:101500000020704743688B4208D90368585C00F09C
:10151000E000A0F1A00358425841704700207047F6
:1015200010B50446FFF7EEFF50B163688B4208D94F
:101530002368585C00F01F00A0F11F035842584177
:1015400010BD0020FCE743688B4208D90368585C53
:101550000C30C0B201288CBF002001207047002051
:1015600070470023C0E9013303690160C36070471D
:10157000F8B503680446002B0D46164603DC3621F9
:101580002948F2F7DDF932460021284602F066FBD1
:10159000D4E90170B8420CD00021236801EB070C9C
:1015A0009CFBF3F203FB12C2904205D1002088425B
:1015B00004D14FF0FF3031E00131EFE7C21992FB67
:1015C000F3FE03FB1E2ED4F80CC01CF80EE0BEF197
:1015D0000A0F26D128B3013A92FBF3F103FB112243
:1015E000002106F1FF3E71450ED2E7686368FB5C9F
:1015F0006B5467682668013797FBF6F306FB137791
:10160000013188426760EEDA1CF802300D2B4FF092
:10161000000304D1054405F8013C0138F8BD2B5402
:10162000FCE70130C3E700BFF8B6010810B5044677
:101630000846C4E900120021A160217302F00EFBEC
:10164000204610BD38B51546D0E901230446581987
:10165000904202D9257B55B1D51A20682A461844F4
:1016600002F0D4FAA3681D44A560012503E01B2104
:101670000248F2F765F9284638BD00BF40B70108B7
:1016800007B501228DF807100DF10701FFF7DAFF0A
:1016900003B05DF804FB006870478068704713B5BD
:1016A000044601A804F0C9FF022201A92046FFF761
:1016B000C9FF02B010BD13B5044601A804F0BDFF78
:1016C000022201A92046FFF7BDFF02B010BD0000B5
:1016D000014608B50348F5F7F7FB0C210248F2F77D
:1016E0002FF900BF78B7010896B7010808B504487C
:1016F000F5F7EAFBBDE808401E210248F2F720B9E1
:10170000E7B7010814B80108F5F76ABC10B9024838
:10171000F5F7DABBF5F74EBCD2B70108F5F760BCB8
:10172000FFF7F4BFFFF7F2BF73B50E4C8DF807005B
:1017300023690E469847054620B9636998472846AD
:1017400002B070BD6368D02201210DF107009847F7
:10175000A368D02201213046984763699847012544
:10176000EDE700BF70010020002337B50A241D46B5
:101770008DF803300DF103010F20FFF7D5FF9DF821
:1017800003305B070ED549F6FE720195019B93422B
:1017900004DD013CEED1204603B030BD019B013396
:1017A0000193F3E70120F7E7F7B50B4C07462369F0
:1017B0000E469847054620B963699847284603B006
:1017C000F0BD8DF804708DF805602368D0220221E9
:1017D00001A898470546EFE77001002010B50C4CB2
:1017E000A37F0BB9637F7BB9E3685A1E03320CD821
:1017F000984728B95C21BDE810400648F2F7A0B828
:10180000012363770023A37710BD6221F3E700BFB4
:101810007001002050B8010807B5FFF7DFFFFFF7A0
:10182000A3FF40B10DF107010E20FFF77DFF30B996
:101830000122094B9A77002003B05DF804FB9DF864
:1018400007100E2041F080018DF80710FFF7ACFF64
:101850000028F0D1ECE700BF7001002084B073B520
:1018600006AC84E80F002D4C06AE25460FCE0FC502
:1018700096E80700002385E807006377A3690BB9A2
:10188000274BA36163682BB1A3681BB123680BB11D
:10189000E3684BB9A0212348F2F752F8002002B0C8
:1018A000BDE8704004B0704723691BB9A4211D48EE
:1018B000F2F746F863691BB9A5211A48F2F740F818
:1018C000FFF78CFF04210E208DF80710FFF76CFF47
:1018D00020B90123A377FFF781FFDFE7FFF744FF7C
:1018E0000028F6D000250DF107010F208DF80750D4
:1018F000FFF71AFF30B19DF90730AB42B6BF0123A5
:101900002577237700210F20FFF74EFF18B9C52157
:101910000448F2F715F801206077C0E77001002055
:10192000C16E000850B80108024B0A465B680146C8
:10193000302018478C4D0020024B0A461B68014698
:10194000302018478C4D00202F4B10B51B7823B941
:1019500040F201112D48F1F7F3FF2D4CA368984791
:1019600000211F20FFF7E8FF20B94FF482712748BC
:10197000F1F7E6FF90211E20FFF7DEFF20B94FF4BC
:1019800083712248F1F7DCFF00212020FFF7D4FF0C
:1019900020B940F207111D48F1F7D2FF00212120A4
:1019A000FFF7CAFF20B94FF484711848F1F7C8FF58
:1019B00000212220FFF7C0FF20B940F2091113488F
:1019C000F1F7BEFF00212320FFF7B6FF20B94FF447
:1019D00085710E48F1F7B4FF00212420FFF7ACFF1A
:1019E00020B940F20B110948F1F7AAFF0021252088
:1019F000FFF7A2FF20B94FF486710448F1F7A0FF6A
:101A0000E368BDE810401847A44D0020FDB8010868
:101A10008C4D002084B073B506AC84E80F002C4CCC
:101A200006AE25460FCE0FC596E8030085E80300F5
:101A300063690BB9274B63616369274898476368FB
:101A400023B940F27D112548F1F77AFF236823B9C5
:101A50004FF4BF712148F1F773FFA36823B940F237
:101A60007F111E48F1F76CFFE36823B94FF4C07192
:101A70001A48F1F765FF236923B940F2811117482D
:101A8000F1F75EFFA36898470DF107010F20FFF7FC
:101A90004BFFE368984763699DF807101048984723
:101AA0009DF80730332B08D00E4863699847002013
:101AB00002B0BDE8704004B0704701250A4B1D70AC
:101AC000FFF742FF0948636998472846F0E700BFDF
:101AD0008C4D0020C16E00088FB80108FDB80108C8
:101AE000A2B80108C7B80108A44D0020DBB801085E
:101AF00000BF7047184B37B51B781BB93C211748FE
:101B0000F1F71EFF0021012000F011FAE8B9144C92
:101B10006420E3689847322500F01FFA01280CD0B2
:101B200000230DF106010F48ADF8063000F01DFA54
:101B300070B9BDF9060003B030BDE36819209847BD
:101B4000013DE9D147F6FD70F5E747F6FF70F2E792
:101B500047F6FE70EFE700BFAD4D002065B9010804
:101B6000984E0020A54D0020F8B5144B05461B7873
:101B70001BB957211248F1F7E3FE0021012000F0C4
:101B8000D6F933240F4E00F0E8F940B904466E1C34
:101B900005F581772B78A34208DC0120F8BDF368B6
:101BA00019209847013CEED12046F7E739463046E8
:101BB00000F0DBF9013408360237EBE7AD4D0020C9
:101BC00065B90108984E0020F0B5244B85B01B780C
:101BD00004461BB99D212248F1F7B2FE214EFF2594
:101BE000B3699847002347F6FF70A4EB8402CDE960
:101BF00001338DF80C3004F5A17104F58173A2F264
